:100000000C94AA290C94A42C0C94CF2C0C94FA2CAC
:100010000C94252D0C94502D0C947B2D0C94A62D16
:100020000C94D12D0C94DB290C94DB290C94DB2946
:100030000C94DB290C94DB290C94DB290C94DB2930
:100040000C94DB290C94D2AB0C94DB290C94DB29A7
:100050000C94DB290C94DB290C94A39E0C94DD29D1
:100060000C94DB290C94238A0C94CF8A0C94DB2902
:100070000C94DB290C94DB290C94DB290C94DB29F0
:100080000C94DB290C94DB290C94DB290C94DB29E0
:100090000C94DB290C94DB290C94DB290C94DB29D0
:1000A0000C94DB290C94DB290C94DB290C94DB29C0
:1000B0000C94DB290C94DB290C94DB290C94DB29B0
:1000C0000C94DB290C94DB290C94DB290C94DB29A0
:1000D0000C94DB290C94DB290C94DB290C94DB2990
:1000E0000C94DB291A2B1F2B242B2E2B382BB12BF6
:1000F000422B4A2B522B5C2B662B702B7F2B892B90
:10010000B12B932B9D2BA72BD52BD82BC72BCB2BD0
:10011000D12B0F2CDC2BE02BE62BEA2BEE2BF42B38
:10012000F82BFC2B0F2C022C062C0A2CF758DD5830
:10013000DA58E058E358E658F258E9580359EC58B1
:10014000EF58568A5C8A6D8A788A808A958A848A72
:10015000958A888A8C8A958A928A0D970B972F9711
:100160002C972A9761975E975C97BA97889785979F
:100170008397084AD73B3BCE016E84BCBFFDC12F9D
:100180003D6C74319ABD56833DDA3D00C77F11BE88
:10019000D9E4BB4C3E916BAAAABE000000803F058B
:1001A000A84CCDB2D44EB93836A9020C50B99186BC
:1001B00088083CA6AAAA2ABE000000803F000D9431
:1001C0006B260D94C1050D949B214E414E494E491D
:1001D0005459494E46CDCCCC3D0AD7233C17B7D114
:1001E0003877CC2B329595E6241FB14F0A000020BA
:1001F000410000C84200401C4620BCBE4CCA1B0E39
:100200005AAEC59D7400000A0B02090C0D0E0807BA
:1002100003040100000000000000000000000000D6
:1002200000000000000000000000000000000000CE
:10023000001211100000000000000000000000008B
:10024000000000000000000000000001021020205B
:10025000080810204010204080020102010804021A
:100260000101020408102040808040201008040290
:1002700001800402018040201008040201080402E9
:1002800001010204081020408001020408102040EF
:100290008005050505070508080808020202020A8C
:1002A0000A08080404040401010101010101010319
:1002B00003030303030303040707070C0C0C0C0CD4
:1002C0000C0C0C0202020206060606060606060BC7
:1002D0000B0B0B0B0B0B0B0000200023002600293F
:1002E000002C002F0032000001000003010601096C
:1002F0000100002200250028002B002E00310034D0
:100300000002010000050108010B0100002100248A
:100310000027002A002D00300033000101000004F6
:100320000107010A0101060D00FE09016602D6203F
:10033000FFFE0BFE0AFE0D0060221969808080809E
:100340008080800080183363A0A0A00357675050BE
:10035000F850F850500259692078A0A0702828F071
:100360002002596948A85010204050A890025868AF
:1003700040A0A040A0989068281363808080113B23
:100380006B2040408080808080404020113B6B800B
:100390004040202020202040408006556520A87045
:1003A000A8200455652020F8202011336360408088
:1003B000065161F811336340E040025969080810A2
:1003C00010204040808002596920508888888888A1
:1003D00050200259692060A02020202020F80259D6
:1003E000697088880810204080F8025969F8081060
:1003F000207008088870025969101030505090F829
:100400001010025969F88080B0C808088870025935
:100410006970888080F088888870025969F80810AF
:100420001020204040400259697088888870888870
:10043000887002596970888888780808887011382F
:100440006840E040000040E04011386840E0400073
:100450000060408002596908102040804020100848
:10046000045464F80000F802596980402010081014
:1004700020408002596970888808102020002002DE
:10048000596970888898A8A8B08078025969205066
:10049000888888F8888888025969F04848487048F0
:1004A0004848F00259697088808080808088700296
:1004B0005969F048484848484848F0025969F88066
:1004C0008080F0808080F8025969F8808080F08018
:1004D0008080800259697088808080988888700246
:1004E000596988888888F888888888123969E0403E
:1004F000404040404040E002596938101010101050
:10050000109060025969888890A0C0A090888802E5
:1005100059698080808080808080F802596988884D
:10052000D8A8A88888888802596988C8C8A8A898BF
:1005300098888802596970888888888888887002B5
:100540005969F0888888F080808080015A6A7088B4
:100550008888888888A87008025969F0888888F097
:10056000A090888802596970888080700808887017
:10057000025969F820202020202020200259698873
:10058000888888888888887002596988888888500F
:100590005050202002596988888888A8A8A8A850A7
:1005A00002596988885050205050888802596988BB
:1005B0008850502020202020025969F8081010206F
:1005C000404080F8113B6BE080808080808080809C
:1005D00080E0025969808040402010100808113BDB
:1005E0006BE0202020202020202020E008536320E2
:1005F0005088015161F82A226280400256667008D4
:1006000078889868025969808080F088888888F0A6
:1006100002566670888080887002596908080878D8
:1006200088888888780256667088F88088700259B1
:100630006930484040F04040404000586870888829
:100640008878088870025969808080B0C888888856
:10065000881238684000C040404040E0004A6A10BC
:1006600000301010101090906002596980808090C6
:10067000A0C0A09088123969C0404040404040402E
:10068000E0025666D0A8A8A8A888025666B0C88816
:10069000888888025666708888888870005868F054
:1006A000888888F0808080005868788888887808F2
:1006B0000808025666B0C88080808002566670883E
:1006C000601088700258684040F040404048300256
:1006D0005666888888889868025666888888505048
:1006E000200256668888A8A8A8500256668850201E
:1006F0002050880058688888889868088870025652
:1007000066F810204080F8015B6B1820202020C084
:10071000202020201822196980808080808080809D
:1007200080015B6BC0202020201820202020C008E2
:10073000536348A890FFFFFFFFFFFFFFFFFFFFFF8E
:10074000FFFFFFFFFFFFFFFFFFFFFFFFFFFFFFFFB9
:10075000FFFFFFFFFFFF0D0060221969800080800E
:1007600080808080800358682070A8A0A0A8702096
:1007700002596930484040E0404048B0035666881E
:10078000705050708802596988885050F820F820BD
:1007900020221969808080800080808080124A6ACF
:1007A000609080609090601090601A3262A0A00308
:1007B00059697088A8D8C8D8A88870045767700885
:1007C00078887800F80356662850A0A05028045373
:1007D00063F80808163161E00359697088E8D8D8D1
:1007E000E8D888700A5161F81744646090906003FB
:1007F00057672020F8202000F807356540A02040EA
:10080000E007356540A04020C02A226240800058A1
:10081000688888888898E8808002596978E8E8E8DC
:10082000E868282828262161C020226240800735F8
:100830006540C04040E0045767708888887000F8C1
:10084000035666A050282850A0025A6A40C0404073
:10085000E00818283808025A6A40C04040E01028D2
:10086000081038025A6A40A04020A04818283808CA
:10087000025969200020204080888870025A6A400E
:10088000200020508888F88888025A6A10200020AA
:10089000508888F88888025A6A3048002050888832
:1008A000F88888025A6A28500020508888F888887A
:1008B000025A6A50500020508888F88888025A6A84
:1008C00020502020508888F8888802596958A0A0B4
:1008D000A0B0E0A0A0B8005B6B70888080808080B2
:1008E00088702040025A6A402000F88080F08080A2
:1008F000F8025A6A102000F88080F08080F8025ACE
:100900006A304800F88080F08080F8025A6A5050BF
:1009100000F88080F08080F8123A6A804000E04061
:1009200040404040E0123A6A204000E040404040F1
:1009300040E0124A6A609000E04040404040E012CF
:100940003A6AA0A000E04040404040E0025969F00F
:10095000484848E8484848F0025A6A2850008888C1
:10096000C8A8988888025A6A4020007088888888B9
:100970008870025A6A1020007088888888887002FF
:100980005A6A30480070888888888870025A6A28B5
:10099000500070888888888870025A6A50500070A9
:1009A0008888888888700355658850205088015B46
:1009B0006B08709898A8A8A8C8C87080025A6A40A6
:1009C000200088888888888870025A6A10200088E9
:1009D000888888888870025A6A30480088888888A1
:1009E000888870025A6A5050008888888888887081
:1009F000025A6A102000888850202020200259695D
:100A000080F0888888F0808080025969609090A08A
:100A1000A0908888B00259694020007008788898B2
:100A2000680259691020007008788898680259692E
:100A3000304800700878889868025969285000701A
:100A4000087888986802596950500070087888982A
:100A500068025A6A304830007008788898680256F0
:100A600066702870A0A850005868708880808870D0
:100A700020400259694020007088F880887002592F
:100A8000691020007088F880887002596930480029
:100A90007088F88088700259695050007088F8801A
:100AA0008870123969804000C040404040E01239EF
:100AB00069204000C040404040E012496960900019
:100AC000C040404040E0123969A0A000C040404012
:100AD00040E0025A6A50206010708888888870024E
:100AE0005969285000B0C888888888025969402010
:100AF0000070888888887002596910200070888882
:100B00008888700259693048007088888888700227
:100B10005969285000708888888870025969505037
:100B200000708888888870035767202000F80020AC
:100B300020015868087098A8A8C8708002596940B8
:100B40002000888888889868025969102000888861
:100B50008888986802596930480088888888986829
:100B6000025969505000888888889868005B6B102B
:100B700020008888889868088870005A6A8080B049
:100B8000C88888C8B08080005B6B50500088888817
:100B9000986808887001050700FE0500FB01F22037
:100BA000FFFE05FE05FE0200400215258080800044
:100BB00080053242A0A002556550F850F850014619
:100BC000562070C030E02002556590102040480249
:100BD0005565608068906805122280800225354046
:100BE000808080400225358040404080043343A00F
:100BF00040A003334340E0400122324080043141B1
:100C0000E002112180025565081020408002455500
:100C10006090909060022535C040404040024555AC
:100C2000E0106080F0024555E0106010E00245558C
:100C30002060A0F020024555F080E010E00245550C
:100C40006080E09060024555F0102040400245551C
:100C500060906090600245556090701060031323AF
:100C6000800080021424800080800235452040806E
:100C70004020033343E000E00235458040204080BF
:100C8000024555E0106000400255657088B8A870B4
:100C9000024555609090F090024555E090E090E05C
:100CA0000235456080808060024555E0909090E07C
:100CB000023545E080E080E0023545E080E080805C
:100CC0000245557080B090700245559090F090901C
:100CD000023545E0404040E002455530101090603C
:100CE00002455590A0C0A09002354580808080E0EC
:100CF00002556588D8A8888802455590D0B0909054
:100D00000245556090909060024555E09090E080DB
:100D1000014656609090906010024555E09090E03A
:100D20009002455570806010E0023545E04040403B
:100D30004002455590909090600245559090A0A03B
:100D40004002556588A8A8A850024555909060902B
:100D5000900245559090701060023545E02040802B
:100D6000E0022535C0808080C0025565804020109B
:100D700008022535C0404040C005324240A0024133
:100D800051F0052232804002445470909070024528
:100D90005580E09090E002344460808060024555C8
:100DA000107090907002445460B0C06002354520CD
:100DB00040E04040004656709090701060024555EB
:100DC00080E0909090021525800080808000273779
:100DD000400040404040800245558090A0E0900295
:100DE00015258080808080025464F0A8A8A8024461
:100DF00054E090909002445460909060004656E019
:100E00009090E080800046567090907010100234F0
:100E100044A0C0808002445470C030E00235454098
:100E2000E0404020024454909090700244549090CE
:100E3000A040025464A8A85050023444A04040A0EE
:100E4000004656909090701060024454F02040F09C
:100E5000023545604080406002152580808080809A
:100E6000023545C0402040C005425250A0FFFFFF60
:100E7000FFFFFFFFFFFFFFFFFFFFFFFFFFFFFFFF82
:100E8000FFFFFFFFFFFFFFFFFFFFFFFFFFFF02006E
:100E900040FFFFFFFFFFFFFFFFFFFFFFFFFFFFFF21
:100EA000FFFFFFFFFFFFFFFFFFFFFFFFFFFFFFFF52
:100EB000FFFFFFFFFFFFFFFFFFFFFFFFFFFFFFFF42
:100EC000FFFFFFFFFFFFFFFFFFFFFFFFFFFFFFFF32
:100ED000FFFFFFFFFFFFFFFFFFFFFFFFFFFFFFFF22
:100EE000FFFFFFFFFFFFFFFFFFFFFFFFFFFFFFFF12
:100EF00001050800FF060121023520FFFF07FF065C
:100F0000FF090050221656808080800080153353E0
:100F1000A0A0A00257575050F850F8505002575711
:100F20002070A07028702013355580A040A02002AA
:100F3000475740A0A040A0A05025135380808012A6
:100F40002656408080808040122656804040404097
:100F5000800245559060F060900255552020F820A1
:100F600020113353604080044151F011335340E06D
:100F70004002465610102040808012365640A0A0F5
:100F8000A0A04012365640C0404040E002465660A5
:100F900090106080F0024656F0206010906002468B
:100FA000562060A0F02020024656F080E0109060AD
:100FB0000246566080E0909060024656F010202075
:100FC00040400246566090609090600246566090A5
:100FD00090701060122555C0C000C0C01136566018
:100FE00060006040801236562040808040200343DD
:100FF00053F000F0123656804020204080123656C2
:1010000040A020400040015858304898A8A890407F
:1010100030024656609090F09090024656E090E084
:101020009090E0024656609080809060024656E0C4
:1010300090909090E0024656F080E08080F002466A
:1010400056F080E0808080024656609080B09060CC
:101050000246569090F0909090123656E0404040F4
:1010600040E002465670202020A04002465690A044
:10107000C0A0A0900246568080808080F002465634
:1010800090F0F090909002465690D0F0B0B0900260
:101090004656609090909060024656E09090E080B6
:1010A00080014757609090D0B06010024656E090A3
:1010B00090E0909002465660904020906012365624
:1010C000E040404040400246569090909090600230
:1010D0004656909090906060024656909090F0F046
:1010E00090024656909060609090025656888850C4
:1010F000202020024656F010204080F0123656E0A4
:1011000080808080E0024656808040201010123699
:1011100056E020202020E016325240A0014151F03C
:1011200016225280400244547090907002465680BD
:1011300080E09090E0123454608080600246561047
:10114000107090907002445460B0C0600246562007
:101150005040E04040014555609070106002465696
:101160008080E09090901236564000C04040E011E0
:1011700037572000202020A040024656808090E073
:101180009090123656C040404040E0025454D0A8DF
:10119000A8A8024454E0909090024454609090605B
:1011A000014555E090E08080014555709070101029
:1011B000024454A0D0808012345460C020C0024643
:1011C000564040E0405020024454909090701234B9
:1011D00054A0A0A04002545488A8A850024454909F
:1011E0006060900145559090709060024454F020EA
:1011F00040F0024757304020C02040302216568031
:101200008080808080024757C02040304020C00648
:10121000425250A0FFFFFFFFFFFFFFFFFFFFFFFF56
:10122000FFFFFFFFFFFFFFFFFFFFFFFFFFFFFFFFCE
:10123000FFFFFFFFFF0900502216568000808080CC
:10124000800146562070A0A070200246562050E033
:101250004050A002555588705070880256568850EC
:10126000F820F82022175780808000808080024775
:10127000577080E0907010E0173151A00256567000
:10128000A8C8C8A87014355560A06000E003435397
:1012900050A050123353E02020143151E002565632
:1012A00070E8D8E8D870173151E015335340A040AA
:1012B00012355540E04000E014355540A02040E094
:1012C000143555C020C020C016225240800145551B
:1012D000909090E08002565678E8E868282824111B
:1012E0005180112252408014355540C04040E014D6
:1012F000355540A04000E0034353A050A00247579B
:10130000808080A060F0200247578080A0D010200D
:101310007002475780408060A0F02012365640008F
:101320004080A04002475740206090F090900247D4
:101330005720406090F0909002475760906090F086
:10134000909002475750A06090F0909002475790BD
:10135000006090F0909002475760906090F09090FD
:1013600002465670A0A0F0A0B00147576090808060
:101370009060400247574020F080E080F0024757DD
:101380002040F080E080F00247576090F080E080DD
:10139000F00247579000F080E080F012375780400D
:1013A000E0404040E01237572040E0404040E0122B
:1013B000375740A0E0404040E0123757A000E040DF
:1013C0004040E00256567048E8484870024757507F
:1013D000A090D0B0909002475740206090909060CD
:1013E000024757204060909090600247576090609D
:1013F0009090906002475750A06090909060024794
:101400005790006090909060123353A040A0024625
:101410005670B0B0D0D0E0024757402090909090E6
:10142000600247572040909090906002475760902C
:10143000909090906002475790009090909060023A
:1014400057571020885020202002465680E0909068
:10145000E0800246566090A0A090A002475740202E
:10146000007090907002475720400070909070027A
:1014700047572050007090907002475750A000705E
:1014800090907002465650007090907002475760DE
:10149000906070909070025454F068B07811355597
:1014A000608080604002475740200060B0C060020A
:1014B000475720400060B0C060024757609000600E
:1014C000B0C060024656500060B0C060123757800E
:1014D0004000C04040E0123757204000C04040E08C
:1014E00012375740A000C04040E0123656A000C05E
:1014F0004040E0024757A040A0107090600247575C
:1015000050A000E0909090024757402000609090DB
:1015100060024757204000609090600247576090FB
:10152000006090906002475750A000609090600269
:1015300046569000609090601235554000E00040A3
:1015400002445470B0D0E002475740200090909081
:10155000700247572040009090907002475760906B
:1015600000909090700246569000909090700148C4
:101570005820400090907090600147578080E09024
:10158000E08080014757900090907090602020206C
:1015900020002020202020200025753A253032759B
:1015A00000253032753A25303275002575642025C6
:1015B0003032753A25303275003FFFF03800703117
:1015C00086302387102787902F87D02F03D0203095
:1015D000102078102078102030102F03D02F87D0C3
:1015E0002787902387103186303800703FFFF03F07
:1015F000FFF038007030FC3020FC102078102030D4
:10160000102C00D02E31D02F7BD02F7BD02E31D07C
:101610002C00D020301020781020FC1030FC303806
:1016200000703FFFF0041040020820020820041060
:101630004008208010410010410008208004104024
:101640000000001FFFF81FFFF81FFFF81FFFF81F23
:10165000E02010201020101020102020102010302A
:10166000300840048003001FE03FF03FF03FF01FD0
:10167000E01FE03FF03FF03FF00FC0078003004560
:1016800072723A207574663820666F6E74206E6FC1
:101690007420696E697469616C697A65642E0045AD
:1016A00072723A207574663820666F6E74206E6FA1
:1016B0007420696E697469616C697A65642E00458D
:1016C00072723A207574663820666F6E74206E6F81
:1016D0007420696E697469616C697A65642E005062
:1016E0006C65617365207265736574005052494E74
:1016F0005445522048414C544544007F80FFC0FF70
:10170000C0FFC07F807F80FFC0FFC0FFC03F001EC2
:10171000000C00FFFFFF0E000E000E000E000E007A
:101720000E000E000E007FC03F801F000E00040060
:1017300004000E001F003F807FC00E000E000E0050
:101740000E000E000E000E000E0000FE0003FF80D3
:101750000783C00E01C00E00E01C00E07F00E03EE9
:1017600000E01C00E00800E00000E00001C00E0105
:10177000C00F078007FF0001FC0003F8000FFE0008
:101780001E0F00380700380380700380700FE07070
:1017900007C0700380700100700000380000380737
:1017A000001E0F000FFE0003F80000060C00FE07ED
:1017B000022603BC017FFE08FE08FE05080806009D
:1017C0000040F0C88888987810050808060000C016
:1017D000F88888888888F80505050600012030F813
:1017E00030200508080600002070F820202020E0A6
:1017F0000509090600FF2070A8A8B8888870200590
:101800000606060001E08CEA8C8A0A050909060032
:10181000FFF8A88888888888A8F8050A0A0600FEC4
:10182000205050505088A8A8887003030306000376
:1018300040A040FFFFFFFFFFFFFFFFFFFFFFFFFF95
:10184000FFFFFFFFFFFFFFFFFF0000000605FF0196
:101850000707060200808080808000800303030663
:101860000105A0A0A005060606000050F85050F89B
:10187000500509090600FF2070A8A07028A8702054
:10188000050707060000C8C81020409898050707FC
:1018900006000040A0A040A89068010303060205CE
:1018A0008080800309090601FF204040808080403D
:1018B00040200309090601FF8040402020204040CD
:1018C0008005070706000020A8702070A8200505E5
:1018D000050600012020F820200203030601FFC0B6
:1018E0004080050101060003F8020202060100C063
:1018F000C0050707060000081010204040800507BB
:1019000007060000708898A8C888700307070601BA
:101910000040C040404040E00507070600007088D6
:1019200008102040F8050707060000F808103008E6
:10193000887005070706000010305090F810100559
:101940000707060000F880F00808887005070706FA
:101950000000304080F0888870050707060000F816
:1019600008101020202005070706000070888870E6
:10197000888870050707060000708888780810605E
:10198000020505060100C0C000C0C002060606012F
:10199000FFC0C000C0408003050506010120408053
:1019A0004020050303060002F800F80305050601C0
:1019B0000180402040800507070600007088102045
:1019C0002000200507070600007088B8A8B88070BE
:1019D000050707060000708888F8888888050707CB
:1019E000060000F04848704848F005070706000068
:1019F00070888080808870050707060000F04848DE
:101A0000484848F0050707060000F88080F080800D
:101A1000F8050707060000F88080F0808080050741
:101A20000706000070888080988870050707060008
:101A300000888888F8888888030707060100E04046
:101A400040404040E0050707060000381010101025
:101A500090600507070600008890A0C0A090880548
:101A60000707060000808080808080F80507070651
:101A7000000088D8A888888888050707060000889D
:101A800088C8A89888880507070600007088888895
:101A9000888870050707060000F08888F08080803D
:101AA00005070706000070888888A8906805070762
:101AB000060000F08888F0A090880507070600005F
:101AC00070888070088870050707060000F82020DD
:101AD000202020200507070600008888888888883D
:101AE0007005070706000088888888505020050781
:101AF0000706000088888888A8A850050707060000
:101B000000888850205088880507070600008888CC
:101B10005020202020050707060000F8081020406C
:101B200080F80309090601FFE080808080808080C2
:101B3000E005070706000080404020101008030958
:101B4000090601FFE020202020202020E0050303DB
:101B50000600052050880501010600FEF803030376
:101B600006010580402005050506000070087888FC
:101B7000780507070600008080F0888888F0050552
:101B800005060000708080887005070706000008C1
:101B90000878888888780505050600007088F08038
:101BA00070050707060000304840E0404040050748
:101BB000070600FE70888888780870050707060009
:101BC000008080F0888888880307070601004000AD
:101BD000C0404040E00409090601FE10003010102A
:101BE0001010906005070706000080808890E09044
:101BF00088030707060100C04040404040E005055B
:101C000005060000D0A8A8A8A8050505060000B094
:101C1000C8888888050505060000708888887005D2
:101C200007070600FEF0888888F080800507070611
:101C300000FE78888888780808050505060000B049
:101C4000C880808005050506000078807008F005D2
:101C500007070600002020F82020201805050506AB
:101C6000000088888898680505050600008888882F
:101C700050200505050600008888A8A85005050520
:101C800006000088502050880507070600FE888857
:101C90008850204080050505060000F8102040F817
:101CA0000309090601FF20404040804040402001D8
:101CB00009090602FF80808080808080808003097F
:101CC000090601FF8040404020404040800503035A
:101CD00006000248A890FF1FFFFFFFFFFFFF600004
:101CE00000000001FF400000000000FF8000000035
:101CF00000007F83CF00000C303F87FF80000C3056
:101D00001F867980000C000F8C30C7838C30E78CE5
:101D100030CFC7CC31F38C30DCECEC33B98C30D81D
:101D20006C6C33198C30D06C0C33198C30D86C0C33
:101D300033198C30DC6C0E3B198C30CF7C079F192B
:101D40008C30C77C038F1940000000000002600047
:101D500000000000061FFFFFFFFFFFF8000000006B
:101D60000000000000000000000000000000000073
:101D70000000000000000000000000000000000C57
:101D8000000000000000000C000000000000001235
:101D900000000000000000230000000000000021FF
:101DA000000000000000004C800000000000005E09
:101DB000800000000000009240000000000000A130
:101DC0004000000000000121200000000000027F10
:101DD000900000000000020010000000000007FF5B
:101DE000F8000000000004000800000000000800E7
:101DF00004000000000008000600000000001000C1
:101E0000020000000000301E010000000000207FE2
:101E100081000000000041FFE0800000000043FC62
:101E2000F08000000000873B7840000000018EDB5E
:101E3000FC60000000010FEBCC20000000021FED51
:101E4000B610000000021FDEB6100000000439CDFD
:101E50007F080000000436E0FF08000000087EC094
:101E6000BB84000000187F005D86000000107FC06A
:101E7000ED82000000203CC07301000000203B33D5
:101E80007F01000000701BE77E03800000C81DEE8C
:101E9000DE04C00000880FDEDC04400001240FDFF8
:101EA0003C092000012607DBF8192000027203E735
:101EB000F0139000025101FFE02290000489007F9E
:101EC000802448000904801E004824000BFE4000C6
:101ED00000DFF40010004000008002001FFFFFFF41
:101EE000FFFFFE00000000000000000000000000F6
:101EF0000000000000000000000000001022103C64
:101F00003C0E1F00102210042211040010221008A1
:101F100022110400102210083C110400102210109D
:101F20002211040010221020221104001E1C1E3C4D
:101F30003C0E040000000000000000000000000053
:101F40000000000000000000000000000000000091
:101F50000000000000000000000000000000000081
:101F60000000000000000000000000000000000071
:101F70000000000000000000000000000000000061
:101F80000000000000000000000000000000000051
:101F90000000000000000000000000060900FE062E
:101FA000018902FE20FFFE07FE06FE00000006007B
:101FB000070106060602008080808000800303037C
:101FC000060103A0A0A00507070600FF5050F85027
:101FD000F850500509090600FE2070A8A07028A836
:101FE00070200608080600FF40A848102048540842
:101FF0000507070600FF6090906098906801030352
:102000000602038080800207070602FF408080806E
:102010008080400207070602FF8040404040408029
:102020000505050600008850F850880505050600DE
:10203000002020F820200204040602FEC040408058
:10204000050101060002F8020202060200C0C004F7
:1020500006060601001010204080800406060601D6
:102060000060909090906003060606010040C0401A
:102070004040E00406060601006090102040F00495
:102080000606060100F020601010E00506060600B6
:102090000010305090F810040606060100F080E0B1
:1020A0001010E00406060601006080E090906004D5
:1020B0000606060100F01010204040040606060146
:1020C00000609060909060040606060100609090A9
:1020D000701060020505060200C0C000C0C0020703
:1020E000070602FEC0C000C040408005050506008E
:1020F000001860806018050303060001F800F80569
:102100000505060000C0300830C0040707060100BE
:10211000609010604000400506060600007090A820
:10212000B08070050606060000205088F8888805F3
:102130000606060000F088F08888F004060606010E
:1021400000609080809060040606060100E0909098
:102150009090E0040606060100F080E08080F00424
:102160000606060100F080E0808080040606060175
:1021700000609080B090600406060601009090F028
:10218000909090030606060100E040404040E005C4
:1021900006060600003810101090600406060601BE
:1021A0000090A0C0A09090040606060100808080E8
:1021B0008080F005060606000088D8A8A888880454
:1021C000060606010090D0B0909090050606060025
:1021D00000708888888870040606060100E09090E8
:1021E000E080800407070601FF609090D0B0601087
:1021F000040606060100E09090E0909004060606B2
:102200000100609040209060050606060000F8205E
:1022100020202020040606060100909090909060F7
:10222000040606060100909090F060600506060620
:1022300000008888A8A8D8880506060600008850EF
:10224000202050880506060600008888502020209F
:10225000040606060100F010204080F00306060682
:102260000100E080808080E0040606060100808096
:1022700040201010030606060100E020202020E088
:102280000503030600032050880501010600FEF83F
:102290000202020602048040040404060100709059
:1022A00090700406060601008080E09090E004042F
:1022B00004060100708080700406060601001010FC
:1022C0007090907004040406010060B0C0700406B1
:1022D00006060100205040E040400406060601FECC
:1022E0006090907010600406060601008080E09007
:1022F00090900306060601004000C04040E003083D
:10230000080601FE200060202020A04004060606EA
:1023100001008080A0C0A090030606060100C04016
:10232000404040E0050404060000D0A8A88804044A
:1023300004060100E09090900404040601006090FF
:1023400090600406060601FEE09090E0808004069E
:10235000060601FE7090907010100404040601003F
:10236000A0D0808004040406010070C030E00406A0
:10237000060601004040E04050200404040601002D
:102380009090907004040406010090906060050431
:102390000406000088A8A850040404060100906008
:1023A00060900406060601FE909090709060040410
:1023B00004060100F02040F003070706010020405A
:1023C00040804040200107070602FF808080808017
:1023D00080800307070601008040402040408004C1
:1023E000020206010350A0FFFFFFFFFFFFFFFFFFF8
:1023F000FFFFFFFFFFFFFFFFFFFFFFFFFFFFFFFFED
:10240000FFFFFFFFFFFFFFFF0000000600070106C0
:10241000060602008000808080800406060601FF18
:102420002070A0A070200507070600FF304840F08C
:102430004040F8050505060000A8508850A805068C
:10244000060600008850F820F8200107070602FF62
:10245000808080008080800407070601FF70806014
:10246000906010E0030101060105A00607070600C1
:1024700000788494A494847803050506010160A083
:102480006000E00505050600002850A05028040360
:1024900003060100F01010040101060102F0060716
:1024A000070600007884B4A4A4847804010106011E
:1024B00005F00403030601026090600507070600AB
:1024C000FF2020F8202000F803050506010140A0A8
:1024D0002040E0030505060101C0204020C00202A3
:1024E0000206020440800405050601FF9090B0D06A
:1024F0008005060606000078E8E868282801010142
:10250000060202800202020602FE40800305050662
:10251000010140C04040E003050506010140A04024
:1025200000E0050505060000A0502850A005080899
:102530000600FF40C04050703078100508080600C3
:10254000FF40C04050680810380508080600FFC06A
:10255000204030F0307810040707060100200020EA
:1025600060809060050707060000402020507088BA
:10257000880507070600001020205070888805078E
:1025800007060000205020507088880507070600C5
:10259000002850205070888805070706000050006A
:1025A00020507088880507070600002050205070D2
:1025B000888805060606000078A0F0A0A0B80408E8
:1025C000080601FE609080809060204004070706A6
:1025D00001004020F080E080F004070706010020A1
:1025E00040F080E080F00407070601002050F080F2
:1025F000E080F00407070601005000F080E080F062
:102600000307070601008040E0404040E003070761
:102610000601002040E0404040E0030707060100BB
:1026200040A0E0404040E0030707060100A000E0B2
:10263000404040E00506060600007048E848487043
:1026400004070706010050A090D0B090900407073F
:10265000060100402060909090600407070601008A
:1026600020406090909060040707060100205060B1
:102670009090906004070706010050A06090909031
:102680006004070706010050006090909060050507
:102690000506000088502050880408080601FF1035
:1026A00070B0B0D0D0E08004070706010040209051
:1026B0009090906004070706010020409090909051
:1026C0006004070706010020509090909060040776
:1026D00007060100500090909090600507070600E3
:1026E000001020885020202004060606010080E00B
:1026F0009090E0800406060601006090A0A090A0E3
:10270000040707060100402000709090700407073E
:102710000601002040007090907004070706010039
:102720002050007090907004070706010050A00030
:102730007090907004060606010050007090907032
:1027400004070706010020502070909070050404D3
:1027500006000070A8B0780406060601FE708080AE
:1027600070204004070706010040200060B0C070E0
:1027700004070706010020400060B0C0700407078E
:1027800006010020500060B0C0700406060601007B
:10279000500060B0C070030707060100804000C011
:1027A0004040E0030707060100204000C04040E031
:1027B00003070706010040A000C04040E0030606F2
:1027C000060100A000C04040E004070706010030F9
:1027D00060107090906004070706010050A000E0B0
:1027E00090909004070706010040200060909060E0
:1027F000040707060100204000609090600407076E
:102800000601002050006090906004070706010058
:1028100050A0006090906004060606010050006021
:102820009090600505050600002000F800200404D3
:102830000406010070B0D0E0040707060100402044
:1028400000909090700407070601002040009090CF
:1028500090700407070601002050009090907004CB
:1028600006060601005000909090700409090601C8
:10287000FE2040009090907090600408080601FED1
:102880008080E09090E080800408080601FE5000FF
:102890009090907090605072696E742066726F6D47
:1028A000205344005072696E742066726F6D20531D
:1028B0004400022E2E004D61696E0046696C616D08
:1028C000656E740053746570732F6D6D004A657288
:1028D0006B00416363656C65726174696F6E00566D
:1028E000656C6F6369747900436F6E6669677572B2
:1028F0006174696F6E004573746570732F6D6D0040
:102900004573746570732F6D6D005A7374657073C1
:102910002F6D6D005A73746570732F6D6D00597350
:10292000746570732F6D6D005973746570732F6DBE
:102930006D005873746570732F6D6D0058737465F6
:1029400070732F6D6D00416476616E636564205312
:10295000657474696E67730056652D6A65726B00E5
:1029600056652D6A65726B00567A2D6A65726B002A
:10297000567A2D6A65726B0056792D6A65726B0006
:1029800056792D6A65726B0056782D6A65726B00F8
:1029900056782D6A65726B00416476616E6365647A
:1029A0002053657474696E677300416D61782045CA
:1029B00000416D6178204500416D6178205A0041E9
:1029C0006D6178205A00416D6178205900416D6138
:1029D00078205900416D6178205800416D61782060
:1029E0005800412D74726176656C00412D747261DE
:1029F00076656C00412D7265747261637400412DBF
:102A00007265747261637400416363656C00416355
:102A100063656C00416476616E6365642053657420
:102A200074696E6773005654726176206D696E002A
:102A30005654726176206D696E00566D696E00564F
:102A40006D696E00566D6178204500566D61782085
:102A50004500566D6178205A00566D6178205A0005
:102A6000566D6178205900566D6178205900566D79
:102A70006178205800566D61782058004164766175
:102A80006E6365642053657474696E6773004C6F80
:102A90006164206D6D004C6F6164206D6D00556E3A
:102AA0006C6F6164206D6D00556E6C6F6164206D9C
:102AB0006D00416476616E6365204B004164766110
:102AC0006E6365204B00416476616E6365642053DC
:102AD000657474696E67730044697361626C652024
:102AE0007374657070657273004D3834004C657690
:102AF000656C2058204178697300004175746F201F
:102B0000686F6D6500473238004D6F7665206178DB
:102B10006973004D61696E00457874727564657201
:102B200020004D6F7665205A004D6F766520590064
:102B30004D6F76652058004D6F76656D656E74003B
:102B4000457874727564657220004D6F766520302B
:102B50002E316D6D004D6F766520316D6D004D6FBE
:102B600076652031306D6D004D6F76652061786936
:102B70007300486F74656E6420746F6F20636F6CB0
:102B80006400457874727564657220004D6F7665D7
:102B9000205A004D6F76652059004D6F766520589C
:102BA000004D6F7665205A004D6F76652059004DB7
:102BB0006F76652058005761697420666F720066F1
:102BC000696C616D656E7420707572676500005088
:102BD0006C6561736520776169742E00507265734E
:102BE0007320627574746F6E00746F2072657375F4
:102BF0006D65207072696E74005761697420666F2C
:102C0000720066696C616D656E74206C6F61640042
:102C1000496E736572742066696C616D656E7400CF
:102C2000616E6420707265737320627574746F6E68
:102C300000746F20636F6E74696E75650050726505
:102C4000737320627574746F6E00746F20686561B1
:102C500074206E6F7A7A6C65004E6F7A7A6C65209C
:102C600068656174696E6700506C65617365207793
:102C70006169742E2E2E005761697420666F720090
:102C800066696C616D656E7420756E6C6F61640051
:102C90005761697420666F720066696C616D656E5C
:102CA00074206368616E676500746F20737461726D
:102CB00074004368616E67696E672046696C616D78
:102CC000656E7400554E4C4F41442046494C414D71
:102CD000454E54004C4F41442046494C414D454ED1
:102CE000540020204E6F7A7A6C653A20002000450F
:102CF0006E642066696C616D656E74206368616ED8
:102D00006765005075726765206D6F7265000043DE
:102D100068616E67652066696C616D656E740055EB
:102D20006E6C6F61642066696C616D656E74004CD9
:102D30006F61642066696C616D656E74004D36303C
:102D40003020423020542564004D373032203B255E
:102D500064004D37303220542564004D3730312027
:102D600054256400507265686561742043757374FE
:102D70006F6D005072656865617420437573746F80
:102D80006D00507265686561742041425300507255
:102D9000656865617420504C41004261636B004E70
:102DA0006F2053442063617264005072696E742016
:102DB00066726F6D2053440041626F7574205072CB
:102DC000696E746572004368616E67652066696C40
:102DD000616D656E74004368616E67652066696C3D
:102DE000616D656E74004D36303020423000436FA7
:102DF0006E66696775726174696F6E0054656D7097
:102E000065726174757265004D6F76656D656E747F
:102E100000526573756D65207072696E740054752B
:102E20006E650053746F70207072696E740050612B
:102E3000757365207072696E7400496E666F2073D9
:102E4000637265656E0053746F70207072696E7482
:102E5000004D61696E005072696E742061626F721C
:102E6000746564004D3234004D323520500A4D32C5
:102E7000340050726F6265205A204F666673657425
:102E80000042616279737465702059004261627911
:102E900073746570205800466C6F7700466C6F77CE
:102EA0000046616E20737065656420310046616E76
:102EB000207370656564203100426564004265647A
:102EC000004E6F7A7A6C65004E6F7A7A6C650053AB
:102ED00070656564005370656564004D61696E00DE
:102EE000426162797374657020590042616279733E
:102EF000746570205800436F6F6C646F776E004686
:102F0000616E20737065656420320046616E2073C7
:102F10007065656420320046616E2073706565647B
:102F200020310046616E2073706565642031004277
:102F3000656400426564004E6F7A7A6C65004E6F7E
:102F40007A7A6C65004D61696E00526573746F72B8
:102F500065206661696C73616665004C6F61642011
:102F600073657474696E67730053746F7265207350
:102F7000657474696E67730050726F6265205A20C1
:102F80004F666673657400416476616E63656420A4
:102F900053657474696E6773004D61696E00507299
:102FA0006F6265205A204F6666736574004C756CBD
:102FB0007A426F742054415A2036207265616479D8
:102FC0002E005072696E74696E672E2E2E0050723C
:102FD000696E74207061757365640043617264206A
:102FE00072656D6F766564004361726420696E730B
:102FF0006572746564004D33310043616E6E6F74A9
:1030000020656E746572207375626469723A20007F
:103010002E0A006F70656E206661696C65642C20F5
:1030200046696C653A20006175746F25632E6700F0
:103030006572726F722077726974696E6720746F3F
:103040002066696C650A004E6F74205344207072CC
:10305000696E74696E670A005344207072696E74F9
:10306000696E67206279746520002E0A0044656CE1
:103070006574696F6E206661696C65642C204669B1
:103080006C653A200046696C652064656C65746502
:10309000643A0057726974696E6720746F206669BC
:1030A0006C653A20002E0A006F70656E20666169BB
:1030B0006C65642C2046696C653A20002E0A006F0E
:1030C00070656E206661696C65642C2046696C656C
:1030D0003A200046696C652073656C6563746564AD
:1030E0000A002053697A653A200046696C65206FB2
:1030F00070656E65643A20002066696C653A200050
:10310000667265736800646F696E67004E6F772042
:1031100000454E4420535542524F5554494E450A9E
:10312000002220706F73002220706172656E743A05
:103130002200535542524F5554494E452043414C6D
:103140004C207461726765743A2200747279696EFA
:103150006720746F2063616C6C207375622D6763E8
:103160006F64652066696C65732077697468207484
:103170006F6F206D616E79206C6576656C732E20A3
:103180004D4158206C6576656C2069733A310A00B0
:103190004D3234004D323320257300534420636197
:1031A0007264206F6B0A006F70656E526F6F7420CF
:1031B0006661696C65640A00766F6C756D652E6971
:1031C0006E6974206661696C65640A005344206905
:1031D0006E6974206661696C0A00286E6F206669EA
:1031E0006C65290043616E6E6F74206F70656E2090
:1031F00073756264697220007C3C3E5E2B3D3F2FFC
:103200005B5D3B2C2A225C004F4646004F4E00651A
:1032100063686F3A004572726F723A004572726F5E
:10322000722077726974696E6720746F204545500B
:10323000524F4D210A005072657373206275747489
:103240006F6E20286F72204D3130382920746F2026
:1032500068656174206E6F7A7A6C650A00507265D9
:10326000737320627574746F6E20286F72204D31F5
:1032700030382920746F20726573756D650A0049B6
:103280006E736572742066696C616D656E74206121
:103290006E6420707265737320627574746F6E2033
:1032A000286F72204D313038290A004D3630303ABF
:1032B00020546F6F20636F6C6400486F74656E6498
:1032C00020746F6F20636F6C640A00486F74656EC2
:1032D0006420746F6F20636F6C640A00496E7365BD
:1032E00072742066696C616D656E7420616E642015
:1032F000707265737320627574746F6E20286F72BC
:10330000204D313038290A0063616E63656C0072AC
:103310006573756D656400726573756D65007061C8
:103320007573656400706F7765726F6666002F2F26
:10333000616374696F6E3A0020573A0020573A0073
:10334000457874727564657220436F6F6C696E673F
:103350002E2E2E0045787472756465722048656162
:1033600074696E672E2E2E00202F002042403A00F6
:1033700020403A004D383420582059205A2045002A
:10338000546865726D616C2052756E617761790069
:10339000453120544845524D414C2052554E4157DD
:1033A00041590042656400202D20496E76616C69A8
:1033B00064206578747275646572206E756D6265DF
:1033C0007220210A0048656174696E672066616930
:1033D0006C6564004265640048656174696E6720CD
:1033E0006661696C65640045312048656174696E89
:1033F00067206661696C6564004D494E54454D50C7
:103400002074726967676572656400453120457292
:10341000723A204D494E54454D5000426564004D6E
:10342000415854454D5020747269676765726564F0
:10343000004531204572723A204D415854454D5057
:103440000042656400626564002C207379737465C2
:103450006D2073746F7070656421204865617465B8
:10346000725F49443A200023646566696E652044B2
:10347000454641554C545F004B6420004B69200089
:103480004B7020000062656400504944204175740F
:103490006F74756E652066696E6973686564212056
:1034A00050757420746865206C617374204B702CA7
:1034B000204B6920616E64204B6420636F6E7374CF
:1034C000616E74732066726F6D2062656C6F772019
:1034D000696E746F20436F6E666967757261746997
:1034E0006F6E2E680A00504944204175746F7475E0
:1034F0006E65206661696C6564212074696D656F15
:1035000075740A00546865726D616C2052756E6145
:1035100077617900453120544845524D414C205245
:10352000554E4157415900426564004865617469D0
:103530006E67206661696C6564004531204865618D
:1035400074696E67206661696C6564004265640039
:10355000504944204175746F74756E6520666169C9
:103560006C6564212054656D706572617475726557
:1035700020746F6F20686967680A00204B643A20E6
:1035800000204B693A2000204B703A20000A20436B
:103590006C617373696320504944200A002054759C
:1035A0003A2000204B753A2000206D61783A2000C7
:1035B000206D696E3A200020643A20002062696123
:1035C000733A2000504944204175746F74756E65DC
:1035D0002073746172740A00504944204175746FFD
:1035E00074756E65206661696C6564212054656D33
:1035F000706572617475726520746F6F2068696799
:10360000680A001000AD0330016A0150022B0170FE
:10361000030A019004F500B005E500D006D800F0DB
:1036200007CE001009C500300ABE00500BB700706D
:103630000CB100900DAB00B00EA600D00FA200F0B0
:10364000109D0010129900301395005014920070D4
:10365000158E0090168B00B0178700D0188400F0EC
:10366000198100101B7E00301C7B00501D790070FA
:103670001E7600901F7300B0207000D0216E00F005
:10368000226B00102469003025660050266300700C
:1036900027610090285E00B0295C00D02A5900F014
:1036A0002B5600102D5400302E5100502F4E00701C
:1036B000304B0090314800B0324500D0334200F02A
:1036C000343E0010363B003037370050383300703E
:1036D000392E00903A2900B03B2300D03C1B00F06B
:1036E0003D1100103F0100F03F00001000C9021022
:1036F000012C014001220170011801B0010E01F0FE
:103700000104015002FA00B002F0003003E600D0DC
:1037100003DC009004D2007005C800A006BE0000C3
:1037200008B400B009AA00D00BA000600E9600609B
:10373000118C000015820020197800C01D6E00A0B9
:10374000226400B0275A00902C500000314600E05F
:10375000343C0010383200903A2800603C1E00A033
:103760003D1400803E0A00203F00006F70656E002F
:10377000545249474745524544003A20007A5F7009
:10378000726F6265007A5F6D696E00795F6D617856
:1037900000795F6D696E00785F6D617800785F6DAC
:1037A000696E005265706F7274696E6720656E6431
:1037B00073746F70207374617475730A00456E645E
:1037C00073746F7073202563202563202563202583
:1037D000630020503A00205A3A0020593A002058FD
:1037E0003A00656E6473746F7073206869743A2070
:1037F00000486F6D696E67206661696C6564004999
:103800006E76616C69642065787472756465720A9D
:103810000045313A200045303A20005A3A200059FC
:103820003A20004D53312C4D53322C4D5333205000
:10383000696E730A583A20004D6963726F7374653C
:10384000707320756E617661696C61626C650A00E7
:10385000205A3A0020593A0020436F756E74205860
:103860003A00C23100001C260000F4190000D80FF5
:103870000000EB080000C0040000750200004001D9
:10388000000024F4D43050C38E20C2A24017828B93
:103890007011127A910D816CD90AA861E108C7589C
:1038A0006607615143061E4B5D05C145A7041A41D9
:1038B0001104093D9803713931034036DB02653349
:1038C0009102D4305402802E1D02632CEE01752A21
:1038D000C501B028A001102781018F2564012B2488
:1038E0004B01E0223401AC211F018D200D01801F0E
:1038F000FC00841EED00971DDF00B81CD200E61B03
:10390000C600201BBC00641AB200B219A8000A1934
:10391000A0006A189900D117910040178B00B516C6
:10392000840031167E00B31579003A157300C71470
:103930006F0058146A00EE136600881363002513A5
:103940005E00C7125B006C12570015125400C111C3
:10395000510070114F0021114B00D61049008D10FD
:1039600047004610440002104200C00F4000800F84
:103970003E00420F3C00060F3B00CB0E3800930E7A
:1039800037005C0E3500270E3400F30D3200C10DF8
:103990003100900D3000600D2E00320D2D00050D10
:1039A0002C00D90C2B00AE0C2900850C29005C0CD6
:1039B0002700350C27000E0C2600E80B2400C40B52
:1039C0002400A00B23007D0B23005A0B2100390B90
:1039D0002100180B2000F80A1F00D90A1E00BB0A9C
:1039E0001E009D0A1D00800A1D00630A1C00470A74
:1039F0001B002C0A1B00110A1A00F7091A00DD0926
:103A00001900C4091900AB091900920917007B09B4
:103A10001800630917004C09160036091600200922
:103A200016000A091500F5081500E0081400CC0876
:103A30001400B8081400A4081400900813007D08AE
:103A400012006B08130058081200460812003408D0
:103A50001100230811001208110001081100F007DD
:103A60001000E0071000D0071000C0071000B007DA
:103A70000F00A107100091070E0083070F007407C5
:103A80000F0065070E0057070E0049070E003B07A1
:103A90000D002E070E0020070D0013070D0006076E
:103AA0000D00F9060C00ED060D00E0060C00D40632
:103AB0000C00C8060C00BC060C00B0060C00A406E6
:103AC0000B0099060C008D060B0082060B00770692
:103AD0000B006C060B0061060A0057060B004C0633
:103AE0000A0042060A0038060A002E060A002406CA
:103AF0000A001A060A001006090007060A00FD055A
:103B00000900F4050900EB050900E2050900D905E3
:103B10000900D0050900C7050900BE050900B50563
:103B20000800AD050800A50509009C0508009405DE
:103B300008008C050800840508007C050800740551
:103B400008006C050700650508005D0507005605BF
:103B500008004E0507004705070040050800380526
:103B60000700310507002A050700230507001C058B
:103B70000600160507000F050700080506000205E8
:103B80000700FB040600F5040700EE040600E80445
:103B90000600E2040700DB040600D5040600CF049B
:103BA0000600C9040600C3040600BD040600B704ED
:103BB0000600B1040500AC040600A6040600A0043B
:103BC00005009B04060095040500900406008A0485
:103BD000050085040500800406007A0405007504CC
:103BE0000500700405006B0405006604050061040F
:103BF00005005C04050057040500520405004D044F
:103C0000050048040500430405003E0404003A048E
:103C1000050035040500300404002C0405002704C9
:103C20000400230405001E0404001A040400160402
:103C30000500110404000D04040009040500040437
:103C4000040000040400FC030400F8030400F4036F
:103C50000400F0030400EC030400E8030400E403A0
:103C60000400E0030400DC030400D8030400D403D0
:103C70000400D0030400CC030400C8030300C50300
:103C8000030024F404D9201BC40C5C0E9804C4095E
:103C90005F0265077101F405F900FB04B3004804F5
:103CA0008700C10369005803550003034500BE02A5
:103CB0003A008402310053022A002902250004023E
:103CC0002000E4011C00C8011900AF011700980191
:103CD00014008401130071011000610110005101F2
:103CE0000E0043010D0036010B002B010B002001DB
:103CF0000B00150109000C01090003010800FB007D
:103D00000800F3000800EB000700E4000600DE00F6
:103D10000600D8000600D2000600CC000500C7004F
:103D20000500C2000500BD000400B9000400B50094
:103D30000400B1000400AD000400A9000400A500C7
:103D40000300A20003009F0004009B0003009800F2
:103D500003009500020093000300900003008D0013
:103D600002008B000300880002008600020084002D
:103D70000300810002007F0002007D0002007B0042
:103D80000200790002007700010076000200740052
:103D9000020072000100710002006F0002006D005D
:103DA00001006C0002006A00010069000200670067
:103DB000010066000100650001006400020062006D
:103DC000010061000100600001005F0002005D0071
:103DD00001005C0001005B0001005A000100590075
:103DE0000100580001005700010056000100550075
:103DF0000100540001005300000053000100520074
:103E0000010051000100500001004F0001004E0070
:103E100000004E0001004D0001004C0001004B006D
:103E200000004B0001004A00010049000100480069
:103E30000000480001004700010046000000460065
:103E4000010045000000450001004400010043005E
:103E50000000430001004200000042000100410058
:103E6000000041000100400001003F0000003F0051
:103E700001003E0000003E0001003D0000003D004A
:103E800001003C0000003C0000003C0001003B0041
:103E900000003B0001003A0000003A000100390038
:103EA0000000390001003800000038000000380030
:103EB0000100370000003700010036000000360026
:103EC000000036000100350000003500000035001C
:103ED0000100340000003400000034000100330011
:103EE0000000330000003300010032000000320007
:103EF00000003200010031000000310000003100FC
:103F000001003000000030000000300001002F00F0
:103F100000002F0000002F0000002F0001002E00E5
:103F200000002E0000002E0001002D0000002D00DA
:103F300000002D0000002D0001002C0000002C00CE
:103F400000002C0000002C0001002B0000002B00C2
:103F500000002B0000002B0001002A0000002A00B6
:103F600000002A0000002A000100290000002900AA
:103F7000000029000000290000002900010028009D
:103F80000000280000002800000028000000280091
:103F90000100270000002700000027000000270084
:103FA0000000270001002600000026000000260077
:103FB000000026000000260001002500000025006A
:103FC000000025000000250000002500000025005D
:103FD0000100240000002400000024000000240050
:103FE0000000240001002300000023000000230043
:103FF0000000230000002300000023000000230035
:104000000100220000002200000022000000220027
:104010000000220000002200010021000000210019
:10402000000021000000210000002100000021000C
:1040300000002100010020000000200000002000FE
:1040400000002000000020000000200000002000F0
:104050000000200001001F0000001F0000001F00E2
:1040600000001F0000001F0000001F0000001F00D4
:1040700001001E0000001E0000001E0000001E00C7
:10408000000020204D36303320003A0A0020286DF1
:104090006D29002055004C0046696C616D656E7499
:1040A000206C6F61642F756E6C6F6164206C656E3F
:1040B000677468733A0A0020204D393030204B0075
:1040C0004C696E65617220416476616E63653A0A7F
:1040D0000020204D383531205A005A2D50726F6221
:1040E00065204F66667365740020440020490020F7
:1040F000204D33303420500020440020490020203F
:104100004D33303120500050494420736574746938
:104110006E67733A0A0020460020420020480020C3
:10412000204D3134352053004D6174657269616CE6
:104130002068656174757020706172616D65746569
:1041400072733A0A0020204D3432302053004175FA
:10415000746F20426564204C6576656C696E673AC1
:104160000A00204500205A00205900205800205401
:104170000020530020204D32303520420020453CA5
:104180006D61785F655F6A65726B3E0020583C6DBB
:1041900061785F785F6A65726B3E20593C6D61782B
:1041A0005F795F6A65726B3E205A3C6D61785F7A19
:1041B0005F6A65726B3E00416476616E6365643A66
:1041C00020423C6D696E5F7365676D656E745F74E8
:1041D000696D655F75733E20533C6D696E5F666502
:1041E0006564726174653E20543C6D696E5F7472E3
:1041F0006176656C5F66656564726174653E00201A
:10420000540020520020204D3230342050004163B1
:1042100063656C65726174696F6E2028756E697470
:10422000732F7332293A20503C7072696E745F614B
:104230006363656C3E20523C726574726163745FA7
:10424000616363656C3E20543C74726176656C5F9B
:10425000616363656C3E0A00204500205A002059C6
:104260000020204D3230312058004D6178696D7545
:104270006D20416363656C65726174696F6E20289F
:10428000756E6974732F7332293A0A002045002035
:104290005A0020590020204D3230332058004D6103
:1042A00078696D756D2066656564726174657320EB
:1042B00028756E6974732F73293A0A0053746570F8
:1042C000732070657220756E69743A0A0020204D63
:1042D0003134392043203B20556E69747320696E58
:1042E0002043656C736975730A00202047323120C2
:1042F0002020203B20556E69747320696E206D6DFF
:104300000048617264636F6465642044656661752A
:104310006C742053657474696E6773204C6F6164AC
:1043200065640A00282300002823000064000000C0
:104330002823000000009643000096430000404000
:104340000000C8410000C9420000C9420000C84442
:104350000000D243290A002062797465733B206310
:10436000726320002073746F7265642073657474C7
:10437000696E67732072657472696576656420285A
:1043800000202863616C63756C6174656429210A7F
:104390000020213D2000454550524F4D20435243BF
:1043A000206D69736D61746368202D202873746FAC
:1043B0007265642920002053697A653A2000496EAD
:1043C0006465783A2000204D61726C696E3D563606
:1043D00034290A00454550524F4D20766572736965
:1043E0006F6E206D69736D61746368202845455058
:1043F000524F4D3D00290A002062797465733B20BD
:10440000637263200053657474696E67732053741C
:104410006F726564202800454550524F4D206461FD
:10442000746173697A65206572726F722E0A00502A
:10443000726F62696E67206661696C65640A00501C
:10444000726F62696E67206661696C6564005761AE
:10445000726E696E673A20486F6D696E67204275AB
:104460006D702044697669736F72203C20310A00B8
:10447000020204486F6D652025732573257320663D
:1044800069727374002066697273740A005A005965
:10449000005800486F6D65200020746F6F206C6FAE
:1044A0006E6720657874727573696F6E20707265BF
:1044B00076656E7465640A0020636F6C64206578AD
:1044C00074727573696F6E2070726576656E74654F
:1044D000640A0020453A00205A3A0020593A005810
:1044E0003A00000048420000484200004040FF01FE
:1044F000FF0000A0400000A040000000400000A01D
:10450000430080A143000087430000A0C1008097C2
:10451000430000000000009643008097430000879E
:10452000430000A0C10000A0C10000000020746F83
:104530006F206C6F6E6720657874727573696F6E2B
:104540002070726576656E7465640A0020636F6C16
:104550006420657874727573696F6E207072657609
:10456000656E7465640A00627573793A20706175CE
:1045700073656420666F7220696E7075740A0062DC
:104580007573793A2070617573656420666F722067
:10459000757365720A00627573793A2070726F6381
:1045A000657373696E670A004D3131372050726F41
:1045B0006265207375636365737366756C0A0020AA
:1045C000496E76616C696420657874727564657291
:1045D0002000205A3A200020593A200042656420E9
:1045E000583A200050726F6265205A204F666673F9
:1045F00065743A20003F5A206F7574206F662072F0
:10460000616E676520282D3220746F2035290A00DD
:104610004D31343520533C696E6465783E206F75AA
:1046200074206F662072616E67652028302D3129F5
:104630000A00436C69636B20746F20726573756D3B
:10464000652E2E2E00220A00556E6B6E6F776E203F
:10465000636F6D6D616E643A202200454550524F84
:104660004D204F4B0A004E6F206D6F76652E004532
:1046700043484F00494E464F004552524F52530057
:1046800044525952554E00434F4D4D554E494341AA
:1046900054494F4E006F6666006F467446794680F7
:1046A00046874644454255473A004C756C7A426FFE
:1046B000742054415A2036204F46462E00205A007E
:1046C000205900580020204D61783A2000205A00DF
:1046D000205900580020204D696E3A2000536F6623
:1046E0007420656E6473746F70733A20002569736B
:1046F0000025696D20256973002569682025696D8D
:104700002025697300256964202569682025696D65
:104710002025697300256979202569642025696849
:104720002025696D20256973005072696E742074AC
:10473000696D653A20004D3131332053002F2F2011
:10474000004361703A004D4F54494F4E5F4D4F4406
:10475000455300544845524D414C5F50524F5445CB
:104760004354494F4E004155544F5245504F5254B7
:104770005F53445F5354415455530050524F4D5072
:10478000545F535550504F525400454D4552474584
:104790004E43595F50415253455200434153455F88
:1047A0004C494748545F4252494748544E45535339
:1047B00000544F47474C455F4C49474854530053BA
:1047C0004F4654574152455F504F5745520042554E
:1047D000494C445F50455243454E54004C45564564
:1047E0004C494E475F44415441005A5F50524F423A
:1047F00045004155544F4C4556454C005052494E8A
:10480000545F4A4F420050524F4752455353004164
:1048100055544F5245504F52545F54454D500056D9
:104820004F4C554D455452494300454550524F4D0C
:104830000042494E4152595F46494C455F545241EE
:104840004E534645520053455249414C5F584F4ED6
:104850005F584F4646004649524D574152455F4EBC
:10486000414D453A4D61726C696E20204649524D6A
:10487000574152455F56455253494F4E3A322E30BA
:104880002E302E39392045585452554445525F54E4
:104890005950453A53696E676C6545787472756412
:1048A00065724165726F563220534F555243455FD2
:1048B000434F44455F55524C3A68747470733A2FB5
:1048C0002F636F64652E616C6570686F626A6563E3
:1048D00074732E636F6D2F646966667573696F6E8E
:1048E0002F4D41524C494E2050524F544F434F4C44
:1048F0005F56455253494F4E3A312E30204D414379
:1049000048494E455F545950453A4C756C7A426F50
:10491000742054415A20362045585452554445522B
:104920005F434F554E543A3120555549443A383437
:104930003566303033632D616562642D34653533FF
:104940002D613662392D3764303938346664653606
:1049500030390A002020536D6F6F7468696E6720CC
:10496000286D6D293A202020202020202020202082
:10497000202020202020530020204261636B6C61A6
:1049800073682044697374616E636520286D6D29B6
:104990003A20202020202020200020202020202815
:1049A00046312E30203D2066756C6C2C2046302E12
:1049B00030203D206E6F6E65290A002020436F7203
:1049C00072656374696F6E20416D6F756E742F46EA
:1049D0006164652D6F75743A2020202020460061A7
:1049E00063746976653A0A00696E004261636B6CB4
:1049F00061736820636F7272656374696F6E20699A
:104A0000732000486F6D6520585920666972737471
:104A10000A00486F6D6520585920666972737400EA
:104A2000426564204C6576656C696E67200046615E
:104A3000696C656420746F20656E61626C652042EC
:104A40006564204C6576656C696E670A0042656432
:104A5000204C6576656C20436F7272656374696F74
:104A60006E204D61747269783A000A0A42656420CA
:104A70004C6576656C20436F7272656374696F6E06
:104A8000204D61747269783A00202B000A436F72DE
:104A9000726563746564204265642048656967686F
:104AA000742076732E2042656420546F706F6C6F93
:104AB00067793A0A00202B000A426564204865693C
:104AC00067687420546F706F6772617068793A0A12
:104AD0002020202B2D2D2D204241434B202D2D2BEE
:104AE0000A2020207C202020202020202020202080
:104AF0007C0A204C207C20202020282B29202020CC
:104B0000207C20520A2045207C20202020202020AC
:104B1000202020207C20490A2046207C20282D2986
:104B2000204E20282B29207C20470A2054207C203E
:104B3000202020202020202020207C20480A202007
:104B4000207C20202020282D29202020207C20545B
:104B50000A2020207C20202020202020202020200F
:104B60007C0A2020204F2D2D2046524F4E54202DC0
:104B70002D2B0A2028302C30290A0034746820702C
:104B8000726F626520706F696E742C206469737433
:104B9000616E63652066726F6D20706C616E653A40
:104BA0002000202844525952554E290047323920BE
:104BB0004175746F20426564204C6576656C696E42
:104BC00067003F20284C2C522C462C4229206F7520
:104BD00074206F6620626F756E64732E0A003F50FA
:104BE000726F626520706F696E7473202859292076
:104BF000697320696D706C61757369626C652028DA
:104C0000322D32292E0A003F50726F626520706F7C
:104C1000696E74732028582920697320696D706C3F
:104C200061757369626C652028322D32292E0A0065
:104C30003F2856296572626F7365206C6576656CD6
:104C400020697320696D706C61757369626C652091
:104C500028302D34292E0A0043757272656E742037
:104C600066696C653A2000456E642066696C652053
:104C70006C6973740A00426567696E2066696C65C9
:104C8000206C6973740A00416476616E6365204B21
:104C90003D003F4B2076616C7565206F7574206F09
:104CA000662072616E67652028302D3130292E0A0A
:104CB000004D31313720486F7420456E64204865BF
:104CC0006174696E672E2E2E0A4D313034205331B7
:104CD00037302054300A473238204F310A473120CC
:104CE000593235205A31302046353030300A4D3176
:104CF000303920523137302054300A4D313137208D
:104D00005265776970696E67206E6F7A7A6C650A92
:104D100054300A473120582D31362059323520463B
:104D2000353030300A4731205A310A4D3130392080
:104D3000523137300A473120582D3136205932351B
:104D40002046343030300A473120582D3136205932
:104D500039352046343030300A473120582D31362D
:104D6000205932352046343030300A473120582D12
:104D70003136205939352046343030300A47312019
:104D8000582D3136205932352046343030300A47DC
:104D90003120582D313620593935204634303030C5
:104DA0000A473120582D31362059323520463430CB
:104DB00030300A473120582D3136205939352046B8
:104DC000343030300A473120582D313620593235B1
:104DD0002046343030300A473120582D31362059A2
:104DE00039352046343030300A473120582D31369D
:104DF000205932352046343030300A473120582D82
:104E00003136205939352046343030300A47312088
:104E10005A31350A4D3130362053323535200A4764
:104E2000302058302059300A4D3130392052313637
:104E3000302054300A4D3130370A0020466C6F77ED
:104E40003A200020643A0020693A0020703A00209D
:104E50004500205A00205900204D39322058004387
:104E6000290A0061626C656420286D696E20746592
:104E70006D70200064697300656E00436F6C642080
:104E800065787472756465732061726520002054C2
:104E900000205200416363656C65726174696F6ED6
:104EA0003A205000496E76616C69642065787472AE
:104EB000756465720A0020643A0020693A00207027
:104EC0003A00536C6565702E2E2E0047322F473303
:104ED0002062616420706172616D65746572730A2D
:104EE0000050726F6265205A204F66667365743A8F
:104EF0002000446F6E6520736176696E6720666975
:104F00006C652E0A005344207265616420657272DC
:104F10006F720A00446F6E65207072696E74696EFC
:104F2000672066696C650A0053544F505045442E03
:104F300020005072696E7465722073746F707065B2
:104F4000642064756520746F206572726F72732EB1
:104F50002046697820746865206572726F722061DE
:104F60006E6420757365204D39393920746F207255
:104F70006573746172742E202854656D706572615A
:104F8000747572652069732072657365742E205381
:104F9000657420697420616674657220726573742B
:104FA000617274696E67290A004E6F2043686563F9
:104FB0006B73756D2077697468206C696E65206EFF
:104FC000756D6265722C204C617374204C696E653E
:104FD0003A20004E6F20436865636B73756D2077D0
:104FE000697468206C696E65206E756D6265722CDF
:104FF000204C617374204C696E653A2000636865CB
:10500000636B73756D206D69736D617463682C20BB
:105010004C617374204C696E653A20004C696E6572
:10502000204E756D626572206973206E6F74204C1E
:10503000617374204C696E65204E756D6265722BCC
:10504000312C204C617374204C696E653A20004D00
:1050500031313000526573656E643A2000204200A1
:105060002050006F6B00220A00656E7175657565D2
:10507000696E67202200504944204175746F747531
:105080006E65206661696C656421204261642065FB
:1050900078747275646572206E756D6265720A004F
:1050A00042656420636F6F6C696E672E2E2E00421E
:1050B00065642068656174696E672E2E2E006F6BC3
:1050C000004739310A4730205A31352046363030D2
:1050D0000A4739300A4730205831373020593239A1
:1050E000302046333030300A4D313137205072692C
:1050F0006E742061626F727465642E002020506CA3
:10510000616E6E657242756666657242797465732A
:105110003A20002046726565204D656D6F72793AC0
:105120002000436F6D70696C65643A204D61722098
:10513000203820323031390A00207C2041757468D3
:105140006F723A2028416C657068204F626A65630F
:10515000747320496E632E2C204C756C7A426F74E8
:1051600020476974205265706F7369746F72792972
:105170000A0000204C61737420557064617465648A
:105180003A2000322E302E302E39390A004D61720D
:105190006C696E0020536F6674776172652052658A
:1051A0007365740A00205761746368646F672052E6
:1051B000657365740A002042726F776E206F757494
:1051C0002052657365740A002045787465726E61BB
:1051D0006C2052657365740A00506F776572557064
:1051E0000A0073746172740A004B494C4C45442E9A
:1051F00020005072696E7465722068616C74656419
:105200002E206B696C6C28292063616C6C656421AD
:105210000A004B494C4C20636175736564206279C8
:1052200020746F6F206D75636820696E61637469A7
:1052300076652074696D65202D2063757272656EC8
:105240007420636F6D6D616E643A20004730205AA0
:1052500031300A4731320A4D31303920523136303F
:105260000A4D3131372050726F62696E6720626576
:10527000640070726F62655F726577697065005077
:10528000726F62696E67206661696C6564004D319A
:10529000313720426564206C6576656C696E6720E5
:1052A0006661696C65642E0A4730205A31300A47BE
:1052B000302045300A4D33303020503235205338BD
:1052C00038300A4D333030205035302053300A4DBD
:1052D0003330302050323520533838300A4D333097
:1052E00030205035302053300A4D3330302050328A
:1052F0003520533838300A47342053310070726FEC
:1053000062655F6661696C65640050726F746563A5
:105310007465642050696E0A0025301D0C18282918
:1053200024311C0B174527232F1B0A444316222B1D
:105330001A4142033809FF36030806020200010041
:105340008640B96B7D75B58D1CA965E6E100E3006B
:10535000DF009D7511241FBECFEFD1E2DEBFCDBFB0
:1053600000E00CBF13E0A0E0B2E0E2E8F5E602E006
:105370000BBF02C007900D92AE3FB107D9F726E1EF
:10538000AEEFB3E001C01D92A230B207E1F719E21F
:10539000C9EAD9E200E006C021970109802FFE0189
:1053A0000F94D12AC03AD10780E00807A9F70E94DC
:1053B00015350D94B0320C9400001F920F920FB669
:1053C0000F9211242F933F938F939F93AF93BF938B
:1053D0008091FF0390910004A0910104B091020418
:1053E0003091FE0323E0230F2D3720F40196A11DF9
:1053F000B11D05C026E8230F0296A11DB11D209303
:10540000FE038093FF0390930004A0930104B093E4
:1054100002048091030490910404A0910504B091CA
:1054200006040196A11DB11D80930304909304040A
:10543000A0930504B0930604BF91AF919F918F9103
:105440003F912F910F900FBE0F901F9018952FB77F
:10545000F8946091FF037091000480910104909191
:1054600002042FBF08953FB7F894809103049091F0
:105470000404A0910504B091060426B5A89B05C0BC
:105480002F3F19F00196A11DB11D3FBFBA2FA92FC3
:10549000982F8827820F911DA11DB11DBC01CD0140
:1054A00042E0660F771F881F991F4A95D1F708952C
:1054B0008F929F92AF92BF92CF92DF92EF92FF9224
:1054C0006B017C01D0DF4B015C01C114D104E1040C
:1054D000F104F1F091D3C7DFDC01CB018819990900
:1054E000AA09BB09883E9340A105B10570F321E0EC
:1054F000C21AD108E108F10888EE880E83E0981EF0
:10550000A11CB11CC114D104E104F10421F7DDCFC9
:10551000FF90EF90DF90CF90BF90AF909F908F90D3
:105520000895789484B5826084BD84B5816084BD1B
:1055300085B5826085BD85B5816085BDEEE6F0E00C
:10554000808181608083E1E8F0E010828081826068
:105550008083808181608083E0E8F0E080818160E9
:105560008083E1EBF0E0808184608083E0EBF0E019
:10557000808181608083E1E9F0E0808182608083C6
:10558000808181608083E0E9F0E0808181608083B8
:10559000E1EAF0E0808182608083808181608083A5
:1055A000E0EAF0E0808181608083E1E2F1E08081E7
:1055B00082608083808181608083E0E2F1E080818D
:1055C00081608083EAE7F0E080818460808380816D
:1055D0008260808380818160808380818068808315
:1055E0001092C10008951F93CF93DF93182FEB0102
:1055F00061E016D1209711F460E004C0CF3FD105DF
:1056000031F461E0812FDF91CF911F9145C1E12FEE
:10561000F0E0EB5FFD4FE4914E2F50E0FA0131973F
:10562000E231F10508F09DC08827EE58FF4F8F4FFB
:105630000D94D12A84B5806884BDC7BD97C084B558
:10564000806284BDC8BD92C08091800080688093D4
:105650008000D0938900C093880088C0809180002A
:10566000806280938000D0938B00C0938A007EC0BC
:1056700080918000886080938000D0938D00C093DB
:105680008C0074C08091B00080688093B000C0939B
:10569000B3006CC08091B00080628093B000C09372
:1056A000B40064C080919000806880939000D09393
:1056B0009900C09398005AC08091900080628093B6
:1056C0009000D0939B00C0939A0050C080919000AE
:1056D000886080939000D0939D00C0939C0046C04A
:1056E0008091A00080688093A0008091A0008F7BB3
:1056F0008093A000D093A900C093A80037C08091E8
:10570000A00080628093A000D093AB00C093AA0059
:105710002DC08091A00088608093A000D093AD0040
:10572000C093AC0023C08091200180688093200149
:10573000D0932901C093280119C080912001806273
:1057400080932001D0932B01C0932A010FC0809138
:105750002001886080932001D0932D01C0932C01FB
:1057600005C0C038D1050CF04CCF46CFDF91CF91AA
:105770001F91089590E0FC013197E231F10508F0A6
:105780004EC08827EC57FF4F8F4F0D94D12A809140
:1057900080008F7703C0809180008F7D8093800090
:1057A000089580918000877FF9CF84B58F7702C0FC
:1057B00084B58F7D84BD08958091B0008F7703C03C
:1057C0008091B0008F7D8093B0000895809190000B
:1057D0008F7707C0809190008F7D03C080919000EB
:1057E000877F8093900008958091A0008F7707C0F5
:1057F0008091A0008F7D03C08091A000877F80935F
:10580000A0000895809120018F7707C0809120012A
:105810008F7D03C080912001877F809320010895B0
:10582000CF93DF9390E0FC01E55BFD4F2491FC01F9
:10583000EF56FD4F8491882361F190E0880F991F06
:10584000FC01E55FFC4FC591D491FC01EF50FD4F89
:10585000A591B491611109C09FB7F89488812095F2
:1058600082238883EC912E230BC0623061F49FB7B2
:10587000F8943881822F809583238883EC912E2B96
:105880002C939FBF06C08FB7F894E8812E2B2883F6
:105890008FBFDF91CF9108951F93CF93DF93282F70
:1058A00030E0F901EB5FFD4F8491F901E55BFD4FBD
:1058B000D491F901EF56FD4FC491CC23C1F0162FBE
:1058C000811158DFEC2FF0E0EE0FFF1FEF50FD4F7E
:1058D000A591B4918FB7F894111105C09C91ED2F4B
:1058E000E095E92302C0EC91ED2BEC938FBFDF91A3
:1058F000CF911F910895CF93DF93282F30E0F901C6
:10590000EB5FFD4F8491F901E55BFD4FD491F90107
:10591000EF56FD4FC491CC2389F081112BDFEC2F82
:10592000F0E0EE0FFF1FE952FD4FA591B491EC910D
:10593000ED2381E090E021F480E002C080E090E07F
:10594000DF91CF91089508951F920F920FB60F9295
:1059500011240BB60F922F933F934F935F936F9346
:105960007F938F939F93AF93BF93EF93FF93E091B8
:105970000402F09105021995FF91EF91BF91AF914B
:105980009F918F917F916F915F914F913F912F9157
:105990000F900BBE0F900FBE0F901F9018951F9287
:1059A0000F920FB60F9211240BB60F922F933F93C5
:1059B0004F935F936F937F938F939F93AF93BF9317
:1059C000EF93FF93E0910602F09107021995FF9182
:1059D000EF91BF91AF919F918F917F916F915F9167
:1059E0004F913F912F910F900BBE0F900FBE0F90D4
:1059F0001F9018951F920F920FB60F9211240BB69D
:105A00000F922F933F934F935F936F937F938F9357
:105A10009F93AF93BF93EF93FF93E0910802F091B0
:105A200009021995FF91EF91BF91AF919F918F91CD
:105A30007F916F915F914F913F912F910F900BBE8E
:105A40000F900FBE0F901F9018951F920F920FB6D8
:105A50000F9211240BB60F922F933F934F935F93A6
:105A60006F937F938F939F93AF93BF93EF93FF9326
:105A7000E0910A02F0910B021995FF91EF91BF910D
:105A8000AF919F918F917F916F915F914F913F91D6
:105A90002F910F900BBE0F900FBE0F901F90189577
:105AA0001F920F920FB60F9211240BB60F922F93E5
:105AB0003F934F935F936F937F938F939F93AF9396
:105AC000BF93EF93FF93E0910002F09101021995CB
:105AD000FF91EF91BF91AF919F918F917F916F91C6
:105AE0005F914F913F912F910F900BBE0F900FBE82
:105AF0000F901F9018951F920F920FB60F921124BE
:105B00000BB60F922F933F934F935F936F937F93B7
:105B10008F939F93AF93BF93EF93FF93E091020214
:105B2000F09103021995FF91EF91BF91AF919F9171
:105B30008F917F916F915F914F913F912F910F9036
:105B40000BBE0F900FBE0F901F9018951F920F92D3
:105B50000FB60F9211240BB60F922F933F934F93D2
:105B60005F936F937F938F939F93AF93BF93EF93C5
:105B7000FF93E0910C02F0910D021995FF91EF91C6
:105B8000BF91AF919F918F917F916F915F914F9155
:105B90003F912F910F900BBE0F900FBE0F901F9053
:105BA00018951F920F920FB60F9211240BB60F92F9
:105BB0002F933F934F935F936F937F938F939F9315
:105BC000AF93BF93EF93FF93E0910E02F0910F021A
:105BD0001995FF91EF91BF91AF919F918F917F9117
:105BE0006F915F914F913F912F910F900BBE0F904E
:105BF0000FBE0F901F90189508951F93CF93DF93BA
:105C0000EC011D821C821F821E82198681E088871A
:105C100082E28A871F861E86FE01B396CE01C19658
:105C20002FEF2193E817F907E1F711E018A3CE0150
:105C3000E1D51F8B188E198E80E48A8F1B8E8BEC1A
:105C400091E39AAB89ABDF91CF911F910895DB016E
:105C5000ED91FC911994EF92FF921F93CF93DF93F4
:105C60001F921F92CDB7DEB77C01DC01D196ED917A
:105C7000FC91D29782E069837A83199520E030E025
:105C80004AE069817A81C701E2DF182FD701D196F6
:105C9000ED91FC91D29783E01995D701D196ED91C2
:105CA000FC91D29780E01995812F0F900F90DF9192
:105CB000CF911F91FF90EF9008950F931F93CF9373
:105CC000DF93EC018B01E9A9FAA982E01995E9A912
:105CD000FAA981E0199520E030E044E1B801CE0155
:105CE000B6DF9E012D5C3F4F47E1B801CE01AFDF2B
:105CF000E9A9FAA980E0DF91CF911F910F91199442
:105D0000EF92FF921F93CF93DF93EC017B01E9A900
:105D1000FAA982E01995E9A9FAA981E0199520E08C
:105D200030E045E1B701CE0192DF182F882339F02A
:105D30009E012D5C3F4F47E1B701CE0188DFE9A905
:105D4000FAA980E01995812FDF91CF911F91FF90E3
:105D5000EF900895FC01448F258F9C01245E3F4FF6
:105D600042E375CFCF93DF931F92CDB7DEB79E018D
:105D70002F5F3F4F46E46BDF89810F90DF91CF911A
:105D80000895CF93DF931F92CDB7DEB79E012F5FAB
:105D90003F4F47E45CDF89810F90DF91CF910895F9
:105DA00020E030E048E453CFCF93DF93EC016A81E9
:105DB0007B81D8DF88836A817B81CE01E2DF8983A2
:105DC0006A817B81CE01ECDF8B879E012D5C3F4F8A
:105DD0006A817B8147E1CE01DF91CF9138CFCF93AC
:105DE000DF93EC016A817B8136DF882319F0CE01D5
:105DF000DBDF81E0DF91CF9108958F929F92AF9288
:105E0000BF92CF92EF920F93CF93DF931F921F9287
:105E1000CDB7DEB74C015B012A834983EEDEF40186
:105E2000B382A282498147A32A8120A705A3E4A2C5
:105E3000C3A2C4010F900F90DF91CF910F91EF900B
:105E4000CF90BF90AF909F908F90C9CFFC0162819F
:105E5000738133CFCF93DF93EC01EE85FF853097CD
:105E600009F019956A817B81CE01DF91CF9148CFEE
:105E7000362F242FFC0162817381432F6BCF0F9348
:105E8000FC0182819381648F458F278F068F9F014C
:105E9000245E3F4F4BE3BC01CF010F91D8CEFC01F4
:105EA00060A30895BF92CF92DF92EF92FF920F937B
:105EB0001F93CF93DF936C01D62FB42EC22F78019E
:105EC000CC2369F0F701049120E04B2D6D2FC60122
:105ED000D6DFFFEFEF1AFF0AC150D85FF1CFDF9195
:105EE000CF911F910F91FF90EF90DF90CF90BF90D7
:105EF00008958F929F92AF92BF92CF92DF92EF92CE
:105F0000FF920F931F93CF93DF935C01C62EC42F94
:105F1000D22ED02F220F220F220F1ED0882379F0ED
:105F2000DC0F8D2C912CCD1751F087012D2D4C2F8E
:105F30006C2DC501B7DFE80CF91CCF5FF4CFDF9102
:105F4000CF911F910F91FF90EF90DF90CF90BF9076
:105F5000AF909F908F9008950F93FC010150040F14
:105F600084A996A9941718F0081728F402C00817F6
:105F700050F0041740F42150260F83A995A99617D5
:105F800020F4281720F480E007C0281720F481E0CF
:105F9000261710F0F8CF81E00F91089581E0089561
:105FA0002EE93FE0009729F0F9013197F1F70197C9
:105FB000F9CF0895FC01128280818150838314827D
:105FC0000895FC0180819281980F9283218192171C
:105FD00060F494819F5F94839381890F821710F0FE
:105FE0008FEF820F838381E0089580E00895FC01A4
:105FF00091E08381861708F490E031E0461708F0BD
:1060000030E0832F892B21E05281451708F420E0EE
:106010002823832F8923822B0895DC01FB01108222
:1060200012968C911297818315968C9115978150B9
:10603000828313968C9183830895FB014181238190
:10604000213029F0233031F468EF640F04C0642F4D
:10605000485F01C0642FCBCFDC0115962C911597BA
:106060001696ED91FC911797CF01820F911D820F2B
:10607000911D1192E817F907E1F70895FC01A68137
:10608000B7818281481B8581483018F0A80FB11D67
:106090004770382F369536953695562F577080E8CD
:1060A00090E002C0959587955A95E2F7439F402D61
:1060B0001124669566956695E62FF0E0E40FF11DD4
:1060C000EA0FFB1F3081222311F0832B02C0809541
:1060D000832380830895FB014181DC0112962C917A
:1060E0001297421760F013962C911397241738F0EB
:1060F000608115962C91621710F42481BFCF08950A
:10610000CF92DF92FF920F931F93CF93DF936C0197
:10611000EB01FA809B81913051F030F0923049F0E0
:10612000933051F41FEF09C010E001E007C011E007
:1061300004C010E00FEF02C010E000E0F7FE03C063
:10614000BE01C601C8DF9881900F98839981910F95
:106150009983FF0C99F7DF91CF911F910F91FF90D9
:10616000DF90CF9008950F931F93CF93DF93890112
:10617000FB01C281D3814233D9F058F44531E1F0BB
:10618000473109F1443141F5CE0166DFCE0112DF1E
:1061900023C04634E1F04734E1F04B33E9F4B90170
:1061A000CE014BDF8823C1F0B801CE01A9DF14C0B6
:1061B000B901CE0190DF10C0CE0103DF882369F062
:1061C000CE014ADF09C0B901CE0127DF05C08D81AC
:1061D00001C08981F801808381E0DF91CF911F9117
:1061E0000F910895CF92DF92EF92FF920F931F933A
:1061F000CF93DF937C01D62FD42EC22F122FC62E21
:10620000C20E6C2D611B183038F00FEF20E04D2DC1
:10621000C70135DE1850F5CF6C2F687F6D0F2C2F1E
:10622000277071F097E029272F5F27700FEF10E09C
:1062300001C0000F2A95EAF720E04D2DC7011FDEAF
:10624000DF91CF911F910F91FF90EF90DF90CF9052
:106250000895CF92DF92EF92FF920F931F93CF9307
:10626000DF937C01D62ED42FC22F122FC42EC20E44
:106270004C2D411B183038F00FEF21E06D2DC70178
:10628000FEDD1850F5CF4C2F487F4D0F2C2F277077
:1062900071F097E029272F5F27700FEF10E001C002
:1062A000000F2A95EAF721E06D2DC701E8DDDF91A7
:1062B000CF911F910F91FF90EF90DF90CF900895B5
:1062C000DF92EF92FF920F931F93CF93DF937C01A6
:1062D000162FC42FD22ED02F3FDE8823F9F02D2D7C
:1062E0004C2F612FC7017EDF2D2F4C2F612FC7014F
:1062F000B0DF6FEF6D0D610F2D2F4C2FC701A9DFA0
:106300004FEF4D0F4C0F2D2D612FC701DF91CF9116
:106310001F910F91FF90EF90DF9064CFDF91CF91AD
:106320001F910F91FF90EF90DF900895EF92FF92F1
:106330000F931F93CF93DF937C01D62F122FC42F7F
:10634000040F212F4C2F6D2FC7014CDFCF5F0C1393
:10635000F8CFDF91CF911F910F91FF90EF900895AB
:10636000DF92EF92FF920F931F93CF93DF93EC0195
:10637000162FF42EE22EF0DD882329F02E2D4F2D3E
:10638000612FCE01D3DFDF91CF911F910F91FF904D
:10639000EF90DF9008950895FC01E60FF11D8491C0
:1063A00090E0982F88273196E4918E0F911D0895E3
:1063B000FC0184910895FCDF882321F0823011F0E4
:1063C00083E0089586E0089580E00895FC018081CF
:1063D000089566E0E1CF68E0DFCF0A96FC01849182
:1063E00008950B96FC0184910895DC011496ED91BB
:1063F000FC911597319684910895BF92CF92DF92C8
:10640000EF92FF920F931F93CF93DF938C01E62EB1
:10641000DC011496CD91DC911597CE01C9DFF82EE1
:10642000F80184819581C7DFC82EF1E0FF1203C017
:106430002FE0B22E02C0BB24BA94D80114968D91DD
:106440009C911597CADFF82EF80184819581C9DFE8
:10645000D82ED80114968D919C911597BCDFB0E68B
:10646000BE1538F4009729F0C80FD91F91E6F92E10
:106470000FC0F80184819581ACDFF0E4FE1538F49B
:10648000009729F0C80FD91F81E4F82E01C061964A
:10649000DE1490F4D80150961C92509753961C929B
:1064A000539754961C92549751961C92519752961A
:1064B0001C9280E090E066C0DF1460F38C2D90E0C9
:1064C000FE0124912F3F11F4219657C0FE104CC0BD
:1064D000D80114968D919C9115976ADF9E012F5FCC
:1064E0003F4FFE01882311F08230E1F48491D801FE
:1064F00053968C935397F901249154962C93549767
:10650000FE013396E4915096EC935097FE01349639
:10651000E4915196EC935197FE013596E491529691
:10652000EC9320C08491982F9F709250D80152967E
:106530009C93529782958F7051968C935197F90145
:106540002491822F8F7054968C93549722952F709C
:1065500053962C935397FE013296E491E295EF7097
:106560005096EC93CE010EC0FE013296E491EB21E1
:106570009C012E0F311DC20FD31FFD1409F48ACFC9
:10658000F3949ECFDF91CF911F910F91FF90EF90E9
:10659000DF90CF90BF9008954F925F926F927F925D
:1065A0009F92AF92BF92CF92DF92EF92FF920F93A2
:1065B0001F93CF93DF931F92CDB7DEB72C01C62E6A
:1065C000942E622F1ADF7C01892B09F43AC0F20164
:1065D00084819581F0DEB82EF201138904898189C6
:1065E000C80E8289981AD92CD01A212F4D2D6C2DC6
:1065F000C201B2DC882311F1EB0CF11C195F169576
:1066000016951695612E712CD914C1F03C2D5701A9
:106610008A2D8E19811770F4F501049120E04D2D1B
:10662000632FC20139832BDCFFEFAF1ABF0A398118
:10663000385FEECFE60CF71CD394E6CFF2018089E9
:1066400001C080E00F90DF91CF911F910F91FF90DB
:10665000EF90DF90CF90BF90AF909F907F906F9022
:106660005F904F9008950F931F93CF93DF9300D0C7
:10667000CDB7DEB78C01DC015596ED91FC915697B4
:106680002B834A83698319954A81480F2B8169813D
:10669000C8010F900F900F90DF91CF911F910F9134
:1066A0007BCFAF92BF92DF92EF92FF920F931F9337
:1066B000CF93DF931F921F92CDB7DEB77C01D62E0A
:1066C000042FDC015596ED91FC91569729833A836E
:1066D0001995080F2981A22E3A81B32E10E0F501F9
:1066E00021915F01222339F0402F6D2DC70154DF26
:1066F000D80E180FF4CF812F0F900F90DF91CF910C
:106700001F910F91FF90EF90DF90BF90AF90089591
:10671000DF92EF92FF920F931F93CF93DF937C0151
:10672000D62FD42E8901DC015596ED91FC91569718
:106730001995D80EC0E0F8012491222349F04D2D7F
:106740006D2FC70129DFD80FC80F0F5F1F4FF3CF81
:106750008C2FDF91CF911F910F91FF90EF90DF90E1
:106760000895DC0114962D913C9115972115310562
:1067700009F43FC057968C915797F901811108C0D1
:106780003596E4915896EC935897F9013C9611C0D0
:10679000813041F43F96E4915896EC935897F90173
:1067A000709607C03D96E4915896EC935897F9017E
:1067B0003E96E4915996EC93599758968C91589738
:1067C000082E000C990B59962C915997821B910910
:1067D00027FD93955A962C915A97203441F0829F29
:1067E000C001112426E0969587952A95E1F75B96DE
:1067F0008C93089524EE31E3FC01368B258B0895AC
:10680000CF92DF92EF92FF920F931F93CF93DF937C
:106810008C017B016A01CB01FA011995D82F8823DD
:1068200011F1682FC801E9DDF801C189C195FFEFB9
:10683000EF1AFF0AC701F6011995F801882351F0F4
:106840008089C80FC701F6011995D82F682FC80194
:10685000D4DDEDCFD03221F091898389890F01C039
:1068600080898C0F01C080E0DF91CF911F910F9143
:10687000FF90EF90DF90CF90089546EE51E3C0CFA8
:10688000CF93DF93FC01248135812617370741F030
:10689000EC017583648365DF84EE91E39E8B8D8BC1
:1068A000DF91CF9108954F925F926F927F92AF9256
:1068B000BF92CF92DF92EF92FF920F931F93CF93ED
:1068C000DF93CDB7DEB729013A019B01AC01241952
:1068D0003509460957098A899B89AC89BD89BC015C
:1068E000CD016A197B098C099D090F94512AA801D1
:1068F000970124193509460957090F94B52ACA0189
:10690000B9016A0D7B1D8C1D9D1DDF91CF911F91DB
:106910000F91FF90EF90DF90CF90BF90AF907F905E
:106920006F905F904F90089580E090E008950895F3
:10693000CF92DF92EF92FF920F931F93CF93DF934B
:106940006C017A018B01C0E0D0E0CE15DF0589F043
:10695000D8016D918D01D601ED91FC910190F081EE
:10696000E02DC6011995892B11F47E0102C02196F4
:10697000ECCFC701DF91CF911F910F91FF90EF9066
:10698000DF90CF900895DC01ED91FC910190F081B2
:10699000E02D1994CF93CFB7F8948091070481111B
:1069A00027C0E6ECF2E08491E0E8F2E09491E82F71
:1069B000F0E0EE0FFF1FE55FFC4FA591B491EC9165
:1069C000E92321F461E085E30E944C2C61E085E33A
:1069D0000E94102C8CB580618CBD8CB580648CBD00
:1069E00061E084E30E94102C61E083E30E94102C9C
:1069F000809107048F5F80930704CFBFCF910895E4
:106A0000CF92EF920F93FC0113AE14AE15AE049625
:106A1000F4D90F91EF90CF9008958EBD00000DB482
:106A200007FEFDCF8EB5089508950E94912AFCDFE0
:106A30000F94BC25C0E0D0E00F9440262097E1F3EE
:106A40000E940000F9CFE8E2F4E083AF64AF08955C
:106A5000EF92FF920F931F93CF93DF937A016F3FD3
:106A600071058105910509F048F488E294E08BDF17
:106A70008CE294E0BADC282F30E014C0C0916304AB
:106A8000D09164044D2F50E0EC2FF0E08B019C017D
:106A9000BF018CE294E000D6C80FC0936304D0938A
:106AA00064049C01C901DF91CF911F910F91FF9068
:106AB000EF900895EF92FF920F931F93CF93DF9380
:106AC0008B01C8E2D4E0FBACECAC4E2D50E06F2D56
:106AD00070E09C018CE294E035D6F80EFBAEECAE93
:106AE000DF91CF911F910F91FF90EF900895EF925A
:106AF000FF920F931F93CF93DF938B01C8E2D4E0F3
:106B0000FBACECAC4E2D50E06F2D70E09C018CE2A4
:106B100094E063D6F80EFBAEECAEDF91CF911F91FF
:106B20000F91FF90EF9008956FEF7FEFC3CF4FEF7E
:106B30005FEF8ECFCF9389EE95E00E94FA65C82F64
:106B400060E870E089EE95E0B5DFC63138F460E2C8
:106B500070E080E090E0EBDFCF5FF7CFCF9108955A
:106B60004F925F926F927F928F929F92AF92BF925D
:106B7000CF92DF92EF92FF920F931F93CF93DF9309
:106B8000CDB7DEB72D970FB6F894DEBF0FBECDBFE1
:106B90008091DF05882309F48AC06091BE0B709153
:106BA000BF0B072E000C880B990B0F94EB2711E0FD
:106BB0002091BA0B3091BB0B4091BC0B5091BD0B97
:106BC0000F944C2918160CF010E06091980B7091FE
:106BD000990B072E000C880B990B0F94EB27209133
:106BE000940B3091950B4091960B5091970B0F940D
:106BF0004C2918160CF4106810931A04C09058020F
:106C0000D0905902E0905A02F0905B0220E030E010
:106C1000A901C701B6010F94492787FD05C020E0EF
:106C200030E040E05FE304C020E030E040E05FEBB4
:106C3000C701B6010F9470260F94B827CB010E94AC
:106C4000E783BC0185E194E00F94672FC0905C025C
:106C5000D0905D02E0905E02F0905F0220E030E0B4
:106C6000A901C701B6010F94492787FD05C020E09F
:106C700030E040E05FE304C020E030E040E05FEB64
:106C8000C701B6010F9470260F94B827CB010E945C
:106C9000E783BC0180E194E00F94672F80E692E0E7
:106CA0000E941888BC0188E094E00F94672F0E942E
:106CB0001F67182F81E051D620911A0427FF03C0C7
:106CC00048E00CE002C042E102E08091600490E004
:106CD000449774F480916204841750F027FD34C106
:106CE00089E496E17C0123E060E58CE294E001D93F
:106CF000809160048431B0F480916204823090F01D
:106D0000112309F424C18091B40B882309F41FC115
:106D100089EB95E17C0102E123E042E068E68CE248
:106D200094E0E7D8809160048C31D0F590911A04FA
:106D30008090BA0B9090BB0BA090BC0BB090BD0B99
:106D4000C090BE0BD090BF0B843128F480916204B8
:106D5000883008F033C280916004883008F40EC295
:106D6000809160048C3108F410C28090940B909054
:106D7000950BA090960BB090970B8091980B9091EB
:106D8000990B20916004283008F405C280916004BA
:106D90008C3108F407C2809160048C3108F408C279
:106DA00080914F0883FF26C080917F06882311F1D0
:106DB000809160048433F0F4809162048A32D0F0D0
:106DC00007E028E04AE26AE28CE294E0C9DA05E0F2
:106DD00022E04CE262E38CE294E0C2DA04E02AE0D2
:106DE00041E36AE28CE294E06BDA4BE262E38CE22C
:106DF00094E03ED880916004853328F48091620449
:106E0000813308F0A7C00E949D66823048F09091BF
:106E10006004943328F490916204923308F0A2C085
:106E2000809160048F3208F05EC0809162048832E5
:106E300008F459C00F94F2212B013C018CE3C82EB9
:106E4000D12CE12CF12CC301B201A70196010F94C2
:106E5000932ACA01B901A70196010F94932ACA0186
:106E6000062FD72E5901AE014F5F5F4F7A0150E8D0
:106E7000451651E5550651E06506710408F48CC0CD
:106E8000B90128E130E040E050E00F94932A290155
:106E90003A01DF920F93C50168E170E00F946C2A0C
:106EA0009F938F935F924F928BEA95E19F938F937D
:106EB000FF92EF920F94962F0FB6F894DEBF0FBE9D
:106EC000CDBF5AE0451651046104710408F08EC02C
:106ED00098E0892F880F980F892F81956FE2855A46
:106EE000B2DDC70121DE809160048632A0F480917A
:106EF00062048E3180F008E020E84EE160E08CE230
:106F000094E02EDA80916004863228F48091620445
:106F10008F3108F06DC080916004823328F4809135
:106F200062048B3208F00EC180916004813408F055
:106F30003AC280916204873308F435C26EE380E080
:106F400082DD812FF7DD2FC285E296E1CBCE8FEE79
:106F500095E1E0CE04E02AE441E366E38CE294E0CC
:106F6000AFD951CFF8E48F9FB0011124072E000C48
:106F7000880B990B0F94EB272AE037ED43E25CE393
:106F80000F9487290F94BD27262F02E042E367E381
:106F90008CE294E0E5D944CF84E6A816B10498F4D5
:106FA000DF920F933F932F9381EA95E19F938F9305
:106FB000FF92EF920F94962F0FB6F894DEBF0FBE9C
:106FC000CDBF95E086CFDF920F933F932F9389E952
:106FD00095E19F938F93FF92EF920F94962F0FB6A8
:106FE000F894DEBF0FBECDBF96E073CF99E071CFAE
:106FF00060E08CE294E00E944F2F65E283E023DDA5
:1070000068E570E080E090E092DD65E28BE01BDDFA
:10701000112321F085E194E087DD24C080917F0C6D
:1070200080FD17C035E1E32E34E0F32EF7016191C6
:107030007F016623B9F06F3234F4062E000C770B13
:10704000880B990B04C06FE370E080E090E06FDD87
:10705000EDCF80917E0C80FDDDCF6FEF7FEF8DE86F
:1070600095E145DD65E288E2EEDC69E570E080E00F
:1070700090E05DDD65E280E3E6DC112321F080E154
:1070800094E052DD24C080917F0C81FD17C020E187
:10709000E22E24E0F22EF70161917F016623B9F020
:1070A0006F3234F4062E000C770B880B990B04C05A
:1070B0006FE370E080E090E03ADDEDCF80917E0CF0
:1070C00081FDDDCF6FEF7FEF8DE895E110DD65E2AB
:1070D0008DE4B9DC6AE570E080E090E028DD65E2EF
:1070E00085E5B1DC112321F088E094E01DDD24C0AA
:1070F00080917F0C82FD17C098E0E92E94E0F92E74
:10710000F70161917F016623B9F06F3234F4062EE6
:10711000000C770B880B990B04C06FE370E080E0E4
:1071200090E005DDEDCF80917E0C82FDDDCF6FEF2D
:107130007FEF82E995E1DBDC61E08CE294E00E9484
:107140004F2FE9CE83E009D462E383E07CDC66E084
:1071500070E080E090E0EBDC81E0FFD362E38CE064
:1071600072DC80915202909153020E94B183DCDC68
:1071700065E270E080E090E0DADCD6CE8091AB0B87
:1071800011112DC08111ECCD2AC08091620485318E
:1071900008F059C0EACD2091870B111184C021114C
:1071A000F5CD81C080916204853108F0B0C0F3CD87
:1071B00080916204853108F0DAC0F2CD90FD03C001
:1071C0008FE496E102C087E696E17C010CE022E0C4
:1071D00048E068E08CE294E00E94792FBCCDB601D3
:1071E000DD0C880B990B0F94EB2720E030E040E09A
:1071F0005FE30F9470260F94B827CB010E94B183F0
:107200007C01FC0180818032E1F4F70181818032D0
:1072100011F401E001C002E0902F990F900F892F27
:10722000819567E0815F0FDC83E090E0801B91092E
:107230008E0D9F1D79DC69E070E080E090E077DCE6
:107240008FCD03E0E9CF20E030E040E05FE3C5010F
:10725000B4010F9470260F94B827CB010E94B1831C
:107260007C01FC0180818032E1F4F7018181803270
:1072700011F401E001C002E0902F990F900F892FC7
:1072800081956CE1815FDFDB83E090E0801B9109F9
:107290008E0D9F1D49DC69E070E080E090E047DCE6
:1072A00064CD03E0E9CFBC01990F880B990B0F94D3
:1072B000EB2720E030E040E05FE30F9470260F946E
:1072C000B827CB010E94B1837C01FC018081803210
:1072D000E1F4F7018181803211F401E001C002E0A4
:1072E000902F990F900F892F819567E0845AABDB1F
:1072F00083E090E0801B91098E0D9F1D15DC69E0F5
:1073000070E080E090E013DC41CD03E0E9CF20E0C5
:1073100030E040E05FE3C501B4010F9470260F94A4
:10732000B827CB010E94B1837C01FC0180818032AF
:10733000E1F4F7018181803211F401E001C002E043
:10734000902F990F900F892F81956CE1845A7BDBE8
:1073500083E090E0801B91098E0D9F1DE5DB69E0C5
:1073600070E080E090E0E3DB16CD03E0E9CF009130
:10737000B40B002309F414CD6CE187E664DBF4E67A
:107380000F9FC001112481589F4F6FEF70E00F9441
:10739000802ACB010E94B183C7DB65E270E080E008
:1073A00090E0C5DBFDCC2D960FB6F894DEBF0FBE86
:1073B000CDBFDF91CF911F910F91FF90EF90DF90A4
:1073C000CF90BF90AF909F908F907F906F905F9085
:1073D0004F9008950F931F93CF93DF93CDB7DEB7F0
:1073E00028970FB6F894DEBF0FBECDBF8A0123E009
:1073F000660F771F2A95E1F7680F791F48E050E084
:10740000CE0101960F94CA2E29813A81F80180811C
:1074100091812817390790F08217930760F09C81BB
:107420008281981758F081E090E03B8123812317F7
:1074300038F080E005C081E090E002C08FEF9FEF60
:1074400028960FB6F894DEBF0FBECDBFDF91CF9167
:107450001F910F910895EF92FF920F931F93CF9377
:10746000DF93EC018B017A018A859B85861797074C
:1074700029F08881998104DA1B870A878885998594
:10748000019681F00E811F81B70188819981F5D91C
:10749000080F111D888599858017910718F481E0E0
:1074A00090E010C06E818A81680F97014C818881BD
:1074B0009981F7D82E813F81280F311D3F832E837C
:1074C00080E090E0DF91CF911F910F91FF90EF90BE
:1074D00008954F925F926F927F928F929F92AF9298
:1074E000BF92CF92DF92EF92FF920F931F93CF93B1
:1074F000DF93CDB7DEB72D970FB6F894DEBF0FBE82
:10750000CDBF6C012A013B01490158011B861C8635
:10751000CE0101967C0188E0F70111928A95E9F786
:10752000DB01CA0127E0B695A795979587952A951F
:10753000D1F79A838983F42FFF77FD878F2F8058A7
:107540008B838C831A8619864F3F5105610571051F
:1075500009F018F460E070E026C060911D0470919D
:107560001E048E01075F1F4F97014AEE59E3809179
:107570001B0490911C040E944B6497FDEBCF69851E
:107580007A8583E0660F771F8A95E1F780911B0467
:1075900090911C04680F791F48E050E0C7010F94D8
:1075A000CA2E6F8178856115710519F44B86B60175
:1075B00006C0C616D70619F08D8580688B87AE0188
:1075C000455F5F4FC401F50119952D960FB6F894EC
:1075D000DEBF0FBECDBFDF91CF911F910F91FF9006
:1075E000EF90DF90CF90BF90AF909F908F907F9063
:1075F0006F905F904F9008956F927F928F929F92BD
:10760000AF92BF92CF92DF92EF92FF920F931F93B0
:10761000CF93DF9300D01F92CDB7DEB76C017B0113
:107620003A015901480119821A821B821C82AE015B
:107630004F5F5F4FB301C7010E94AB647C0149817A
:107640005A816B817C81411551056105710529F0D5
:1076500084019501C6013DDFE6CF0F900F900F909A
:107660000F90DF91CF911F910F91FF90EF90DF90DE
:10767000CF90BF90AF909F908F907F906F90089524
:1076800021E020931F04EBE1F4E091838083738376
:10769000628380E090E008957F92AF92BF92CF9294
:1076A000DF92EF92FF920F931F93CF93DF93CDB7AB
:1076B000DEB72C970FB6F894DEBF0FBECDBF6C01BE
:1076C000762EF72F842FE52FB901A801D601149645
:1076D000AD90BC90159790911F04911109C02FEBAC
:1076E00036E1482F672DC60113D880E090E018C01E
:1076F000DA82C9827B82FC838D83EE8318861F82A7
:10770000FA86E9861C861B860BE21AE39E012F5F30
:107710003F4FC501DEDEB501C601B2D88F81988525
:107720002C960FB6F894DEBF0FBECDBFDF91CF9180
:107730001F910F91FF90EF90DF90CF90BF90AF908F
:107740007F900895CF92DF92EF92FF920F931F9355
:10775000CF93DF93CDB7DEB72C970FB6F894DEBF8B
:107760000FBECDBF7C01C901F701C480D580209137
:107770001F04211108C02FE936E1C7010E94883398
:1077800080E090E01BC0FA82E9826B837C834D83AA
:107790005E8318861F821A8709871C861B860BE268
:1077A0001AE39E012F5F3F4F45E454E6BC01C6013A
:1077B00023DFB601C70164D88F8198852C960FB658
:1077C000F894DEBF0FBECDBFDF91CF911F910F9117
:1077D000FF90EF90DF90CF900895CF92DF92EF92DD
:1077E000FF920F931F93CF93DF93CDB7DEB72C9704
:1077F0000FB6F894DEBF0FBECDBF7C01C901F70103
:10780000C480D58020911F04211108C02FE736E1E4
:10781000C7010E94883380E090E01BC0FA82E982B1
:107820006B837C834D835E8318861F821A8709874A
:107830001C861B860BE21AE39E012F5F3F4F48E434
:1078400054E6BC01C601D8DEB601C70119D88F8144
:1078500098852C960FB6F894DEBF0FBECDBFDF9192
:10786000CF911F910F91FF90EF90DF90CF900895EF
:10787000CF93DF93EC01262F4CAD6BAD04960E94A5
:1078800033332BAD082E000C990B820F911D8BAF5B
:1078900081E090E0DF91CF9108950F939CE0899F64
:1078A000802D112421E0280F20932704845F8093EA
:1078B000260490E002964091600450E084179507FA
:1078C00014F480E033C0822F90E02091620430E015
:1078D00082179307B4F76623A9F061E08CE294E085
:1078E0000E944F2F409127044E5F0BE020E860E09C
:1078F0008CE294E00E94B03160E08CE294E00E945F
:107900004F2F05C061E08CE294E00E944F2F609100
:107910002604809160046817A0F29091270480915A
:107920006204891770F280E08ED881E00F9108958B
:10793000CF93DF93FC0185ADEF012496811105C043
:1079400081E085AFCE010E94EF2ECE01DF91CF9175
:107950000C94262F6FEF7FEFCAC8482F50E020917C
:107960002504022E000C330B4217530781F080933D
:107970002504813031F46AE97FE18CE294E00C94D3
:1079800040346AEA77E18CE294E00C944034089544
:10799000EF92FF920F9388E294E0CADF8CE5E82E25
:1079A0008DE1F82E00E428E040E060E08CE294E015
:1079B0000E94792F65E273E08CE294E00E944034EB
:1079C00022E133E041E169E38CE294E00E9451332B
:1079D00065E97BE08CE294E00E94403428E133E0EA
:1079E0004CE16AE38CE294E00E94513360EF7EE068
:1079F0008CE294E00E94403428E233E049E26BE3F9
:107A00008CE294E00E94513360EF7EE08CE294E0DF
:107A10000E94403424E333E04EE36DE38CE294E0D3
:107A20000E94513326E333E04EE362E48CE294E0BB
:107A30000E9451338CE294E00E942A2F8111AECF34
:107A400064EC79E080E090E00E9447836AEA77E1A5
:107A50008CE294E00F91FF90EF900C94403461E041
:107A60008CE59DE195DF64EC79E080E090E00C949A
:107A70004783CF92DF92EF92FF920F931F93CF93A2
:107A8000DF93EDDFC0912C0400912D04D0E0BE0106
:107A90006853710977FF02C06F5F7F4F75956795D7
:107AA000D62E88E294E044DFCE01C0979695879564
:107AB000182FC257D109D695C7954EEEC42EC00EC9
:107AC000DAEFD00F87EDE82E8CE1F82E03E127E006
:107AD0004CE06D2D8CE294E00E94792F83E03DDF35
:107AE00026E333E04C2D612F8CE294E00E94513369
:107AF0002FE333E04D2F6C2F8CE294E00E94513342
:107B00008CE294E00E942A2F8111DCCF64EC79E0B2
:107B100080E090E0DF91CF911F910F91FF90EF9067
:107B2000DF90CF900C94478360E070E08AE99FE19A
:107B3000A7CD1F93CF93DF93C0912D04C695C69513
:107B400088E294E0F5DEDC2FDD0F1D2F1C0F83E0B3
:107B500004DF6C2F80E00E94233589EE95E00E94BF
:107B600094356D2F80E00E9423358CEE96E1F2DE95
:107B7000612F80E00E9423358FED96E1EBDE8CE2F1
:107B800094E00E942A2F8111E2CFDF91CF911F91C3
:107B900008950895CF93E62F6CE0869F602D112401
:107BA00081E0860F80932704645F60932604462F4C
:107BB00050E04E5F5F4F2091600430E04217530762
:107BC0000CF44CC090E02091620430E082179307DF
:107BD0000CF044C0CE2F8EE30E94233565E470E0A4
:107BE00080E090E00E94973561E36C0F062E000C58
:107BF000770B880B990B0E94973560E270E080E06C
:107C000090E00E9497356091BA0B7091BB0B809108
:107C1000BC0B9091BD0B0F94B827CB010E94B18390
:107C20000E9494356FE270E080E090E00E9497350A
:107C30000E941F67811109C085E0C89FF0011124CF
:107C4000E955F44F8481811109C08091BE0B909158
:107C5000BF0B0E94B183CF910C949435CF910895BE
:107C6000CF92DF92EF92FF920F931F93CF93DF9308
:107C70001F921F92CDB7DEB77B01622F49830DDEC5
:107C80004981882309F444C0442311F101151105E9
:107C9000F9F4C7010E941B6626E130E0281B310978
:107CA00037FF02C02F5F3F4F3595279530E82158A9
:107CB000822F830F87FD0DC060E270E080E090E0CE
:107CC0002A8339830E949735398131502A81F0CF38
:107CD00030E8C32ED12CB601C7010E94773576015A
:107CE000E81AF90A0115110511F41E2D07C0FF2429
:107CF000B701C8010E945A351E2D181B173040F0DD
:107D000060E270E080E090E00E949735181BF6CFAB
:107D10000F900F90DF91CF911F910F91FF90EF90F7
:107D2000DF90CF9008950F93CF93DF93982F862FF6
:107D3000EA01692FB2DD882331F168E770E0CE01F6
:107D40000E947735C8E7C81BC73040F060E270E09A
:107D500080E090E00E949735C81BF6CF6091260422
:107D60008AE70E942335602F000F770B880B990B51
:107D70000E94973560E270E080E090E0DF91CF9163
:107D80000F910C949735DF91CF910F910895CF9279
:107D9000DF92EF92FF920F931F93CF93DF93982F71
:107DA000862F6A017901692F78DD882309F447C09D
:107DB000C701002321F00E941B66182F03C00E94F8
:107DC000FA65182FC4E1D0E0C11BD1098C2F880FB0
:107DD000C80FCC0FD0E0BE01C6010E947735C81B8A
:107DE0006AE370E080E090E00E949735C73040F091
:107DF00060E270E080E090E00E949735C81BF6CF0B
:107E00008AEF189F802D11246091260480580E94CB
:107E10002335C701002349F0DF91CF911F910F91C6
:107E2000FF90EF90DF90CF9095CDDF91CF911F9194
:107E30000F91FF90EF90DF90CF900C949435DF91ED
:107E4000CF911F910F91FF90EF90DF90CF90089509
:107E5000BF92CF92DF92EF92FF920F931F93CF9337
:107E6000DF936C017B010E941B66C82FC7010E9433
:107E7000FA6504E110E0081B11098C2F90E0BB2487
:107E8000B394081719071CF0B12CC5E201C0CFE16B
:107E90002C2F30E0A9014E5F5F4F8091600490E08D
:107EA0004817590744F0295031098091620490E045
:107EB00082179307BCF5D0E0E114F104D9F16AE32D
:107EC00070E080E090E00E949735BB2081F0C45FB5
:107ED00080916004C81770F12C2F30E029503109CF
:107EE0008091620490E0821793071CF423C0DD2385
:107EF00009F1802F880F800F6C2F880F0E94233587
:107F000060E270E080E090E00E949735C701DF9169
:107F1000CF911F910F91FF90EF90DF90CF90BF9086
:107F20000C9494356C2F80E00E942335C60112DD3D
:107F3000D1E0C2CFDF91CF911F910F91FF90EF90D1
:107F4000DF90CF90BF900895EF92FF920F93CF9361
:107F5000DF93D82FC62F7901682F8C2F9EDC8823C2
:107F6000F1F0002331F062E070E080E090E00E94E8
:107F700097352D2F4C2F65E1C7010E94D0666EE723
:107F800070E00E945A35CEE7C81BC73040F060E26F
:107F900070E080E090E00E949735C81BF6CFDF913B
:107FA000CF910F91FF90EF9008958F929F92AF9293
:107FB000BF92CF92DF92EF92FF920F936B017C0101
:107FC0008090210490902204A0902304B090240477
:107FD000A50194010F944927882301F120E030E0A6
:107FE000A901C701B6010F944927882351F0A501C3
:107FF0009401C701B6010F94492787FD04C081E0B1
:1080000003C080E001C08FEF80932004C092210460
:10801000D0922204E0922304F09224048091600420
:10802000813128F480916204833008F048C0809147
:108030006004853128F480916204843108F04FC0D7
:10804000809160048F3308F057C0809162048F32B2
:1080500008F452C08AE4E82E87E1F82E00E123E01C
:108060004FE265E08CE294E00E94792F9AE7E92ED6
:1080700097E1F92E23E04FE26AE58CE294E00E945A
:10808000792F8091200440E3481B20E3E22E27E172
:10809000F22E0DE022E06EE68CE294E00E94792F51
:1080A0008091200441E3481B36E1E32E37E1F32EB3
:1080B00022E069E18CE294E00E94792F1DC080915A
:1080C000200444E0481B5BEFE52E56E1F52E0CE062
:1080D00022E062E48CE294E00E94792FA8CF43E191
:1080E000E42E47E1F42E01E023E044E16CE38CE26E
:1080F00094E00E94792FA4CF0F91FF90EF90DF9032
:10810000CF90BF90AF909F908F900895CF92EF92B5
:108110000F93CF93DF93C8E2D4E01B821A8287E5E6
:1081200093E099838883CC24CA94EE24EA9406E4ED
:1081300027E448E460E172E0CE010E94003583E666
:1081400093E099838883DF91CF910F91EF90CF9047
:1081500008959091050194709093030187FD76C076
:10816000A39890910501909594709093030190913C
:108170000501947090930301982F990F86FD72C0AA
:10818000A39880910501809584708093030180916C
:108190000501847080930301292F220F96FD60C092
:1081A000A39880910501809584708093030180914C
:1081B0000501847080930301922F990F26FD4EC014
:1081C000A39880910501809584708093030180912C
:1081D0000501847080930301292F220F96FD3CC076
:1081E000A39880910501809584708093030180910C
:1081F0000501847080930301922F990F26FD2AC0F8
:10820000A3988091050180958470809303018091EB
:108210000501847080930301292F220F96FD18C059
:10822000A3988091050180958470809303018091CB
:10823000050184708093030126FD16C0A3988091E8
:10824000050180958470809303010895A39A89CFD6
:10825000A39AE7CFA39AD5CFA39AC3CFA39AB1CFBE
:10826000A39A9FCFA39A8DCFA39A80910501809561
:1082700084708093030108952F923F925F927F92C2
:108280009F92AF92BF92CF92DF92EF92FF920F93A5
:108290001F93CF93DF937C011B01942E69018AE029
:1082A000481709F47BC0A5E14A134EC0DB011296C2
:1082B000ED91FC9113971281C681D781A49A88E22F
:1082C0008A950000E9F700EE010F80E1582E510E6B
:1082D00098E2792E88EF3DDF872D8A950000E9F737
:1082E000103208F046C0812F8077806832DF812FFE
:1082F0008295807F2EDF872D8A950000E9F780E840
:1083000028DF80E026DF872D8A950000E9F78AEFD5
:1083100020DF872D8A950000E9F75E01B0E1AB0E02
:10832000B11C8881807F15DF89918295807F11DF64
:10833000CA15DB05B1F7872D8A950000E9F71F5FA5
:108340000F5F1511C7CFA4989601492DB101C70140
:10835000DF91CF911F910F91FF90EF90DF90CF9021
:10836000BF90AF909F907F905F903F902F900C9424
:10837000B330802F80778068ECDE802F8295807FFD
:10838000E8DE872D8A950000E9F780E8E2DE80E8E4
:10839000E0DE872D8A950000E9F7B9CF9C9AA49872
:1083A0009B9AA3988091040184608093040180913A
:1083B00005018095847080930301A49AC8E28C2FF4
:1083C0008A950000E9F788E790E00E94D02F88EFB7
:1083D000C0DE8C2F8A950000E9F780E2BADE80E0EB
:1083E000B8DE8C2F8A950000E9F780E0B2DE80E8E5
:1083F000B0DE8C2F8A950000E9F780E0AADE80E1EC
:10840000A8DE8C2F8A950000E9F78FE090E00E94AB
:10841000D02F80E29EDE80E49CDE8C2F8A950000C7
:10842000E9F780E296DE80E694DECA950000E9F77F
:1084300010E0D8E208E2812F807780688ADE812F01
:108440008295807F86DE8D2F8A950000E9F780E88F
:1084500080DE80E07EDE8D2F8A950000E9F78AEFCE
:1084600078DE8D2F8A950000E9F7C0E280E071DEAA
:1084700080E06FDE9D2F9A950000E9F7C150B1F7BB
:1084800088EF67DE802F8A950000E9F71F5F1032C2
:1084900009F0D1CF80E05DDE80EC5BDE88E28A957A
:1084A0000000E9F7A49850CF0E943C7441E050E0EE
:1084B00060E070E0811103C040E050E0BA014093F9
:1084C000DB055093DC056093DD057093DE051092AB
:1084D000B50581E080938F0583E080931F020895A6
:1084E000CF92DF92EF92FF920F931F93CF93DF9380
:1084F0000E9439756C0161E081E00E942A63C0919D
:10850000B505D0E081E0C81AD108C11117C080912B
:108510007E05811104C00E941A6781119BC0809161
:108520001F02882359F081E090917E05911180E02F
:1085300004E024E046EB58E26D2FF5DB62E478E0DE
:1085400089EC97E00E94227B809142088F3201F1F2
:1085500080914F0883FF1CC0C130C1F480917E051B
:10856000813021F40E941A6781117CC080911F0222
:10857000882361F081E090917E05913009F080E0E0
:1085800000E22EE342EB58E26D2FCDDB92E001C01A
:1085900091E080911F02882309F454C0760111E014
:1085A0001C0F8FEFE816F80609F44CC0C91345C03C
:1085B00060E070E0C7010E94587190914F0880916F
:1085C0007E0594FF22C08C1354C00E941A67882332
:1085D00009F44FC082E498E00E94E6731092B5055A
:1085E00082E090E0A0E0B0E08093DB059093DC05B2
:1085F000A093DD05B093DE0581E080938F05109296
:10860000E00583E080931F0250C08C1304C00E94D9
:108610001A6781113DC080911F02882361F081E0BB
:1086200090917E059C1380E000E02BEF35E146E958
:1086300058E26D2F89DC912F01C09F5F81E0E81A1D
:10864000F108AFCFDF5FCF5FD53009F05ECF9093F9
:108650007D052BC00E947A6280918F05882309F4E2
:108660005ECF23C021DF80918F05882309F47ECF60
:108670001CC080911F028823F1F281E090917E0559
:108680009C1380E001E02BEF35E144EA58E2D1CFC2
:1086900082E498E00E94E36F0E9474620E94996BEA
:1086A00080918F05882309F4B6CFDF91CF911F9178
:1086B0000F91FF90EF90DF90CF900895CF93DF93CD
:1086C000EC01CB01BA010F94EB272AE037ED43E22E
:1086D0005CE30F948729688379838A839B83DF9186
:1086E000CF910895CF93DF93EC01CB01BA010F94A2
:1086F000EB27688379838A839B83DF91CF910895E9
:10870000CF93DF93EC01CB01BA010F94EB2720E06C
:1087100030E048EC52E40F948729688379838A8398
:108720009B83DF91CF910895CF93DF93EC01CB0131
:10873000BA010F94EB2720E030E048EC52E40F94AC
:1087400087290F94BD27688379838A839B83DF9170
:10875000CF910895CF93DF93EC01CB01BA010F9431
:10876000EB272AE037ED43E25CE30F948729688327
:1087700079838A839B83DF91CF910895CF93DF9391
:10878000EC01CB01BA010F94EB272AE037ED43E26D
:108790005CE30F948729688379838A839B83DF91C5
:1087A000CF9108956EE573E487E194E40C948E62B2
:1087B00062E773E481E994E40C948E6260E873E408
:1087C00084E394E40C948E6264E973E48DEA94E4A7
:1087D0000C948E626AEA73E481E594E40C948E62F0
:1087E0006EEB73E48AEF93E40C948E620C94F4E5E0
:1087F0000C943BE6CF93DF9300D01F92CDB7DEB74A
:108800000F94EB272AE037ED43E25CE30F948729CE
:1088100069837A838B839C83CE0101960E9457875C
:108820000F900F900F900F90DF91CF910895CF93FD
:10883000DF9300D01F92CDB7DEB70F94EB272AE06D
:1088400037ED43E25CE30F94872969837A838B8356
:108850009C83CE0101960E9450840F900F900F9040
:108860000F90DF91CF910895CF93DF9300D01F92A7
:10887000CDB7DEB70F94EB2720E030E048EC52E4B0
:108880000F94872969837A838B839C83CE01019619
:108890000E94FE850F900F900F900F90DF91CF9167
:1088A0000895CF93DF9300D01F92CDB7DEB70F941A
:1088B000EB272AE037ED43E25CE30F9487296983D5
:1088C0007A838B839C83CE0101960E94B6860F909B
:1088D0000F900F900F90DF91CF910895CF92DF927C
:1088E000EF92FF926B017C0120E030E0A9010F9430
:1088F000492787FD05C020E030E040E05FE304C089
:1089000020E030E040E05FEBC701B6010F94702635
:108910000F94B827CB01FF90EF90DF90CF900C948D
:10892000B1830F94EB27DACFCF93DF9300D01F9260
:10893000CDB7DEB70F94BD270F94E92769837A83FB
:108940008B839C83CE0101960E94FE850F900F9031
:108950000F900F90DF91CF9108950F94EB2720E0B7
:1089600030E048EC52E40F948729DECFCF93DF93B9
:108970001F921F92CDB7DEB789839A830E94A961A7
:1089800040E050E0BA0189819A810F900F90DF9109
:10899000CF910C944F620F93CF93DF9361E081E00E
:1089A0000E942A63C091B505D0E0C11119C0809121
:1089B0007E05811104C00E941A678111AAC08091AE
:1089C0001F02882309F45DC081E090917E0591111A
:1089D00080E004E024E048EE58E26D2FA4D951C0B5
:1089E000C130D1F480917E05813021F40E941A6754
:1089F000811197C080911F02882309F442C081E051
:108A000090917E05913009F080E003E02EE34FED78
:108A100058E26D2F88D935C0C230C9F480917E05E7
:108A2000823021F40E941A67811184C080911F0254
:108A3000882339F181E090917E05923009F080E041
:108A400003E02EE342ED58E26D2F6DD91AC0C3301A
:108A5000C1F480917E05833021F40E941A67811150
:108A600072C080911F02882361F081E090917E05A1
:108A7000933009F080E003E02EE34DEC58E26D2FD7
:108A800052D90E94386281111CC0C430E1F4809137
:108A90007E05843021F40E941A6781115DC08091A7
:108AA0001F02882309F461C081E090917E05943013
:108AB00009F080E003E02EE344EC58E26D2F33D957
:108AC00054C084E001C085E0C8131AC080917E05BF
:108AD0008C1304C00E941A67811149C080911F0243
:108AE000882369F081E090917E059C1380E003E08B
:108AF0002EE34BEB58E26D2F16D98C2F01C08C2F33
:108B0000DF5FCF5FD53009F050CF8F5F80937D0559
:108B100036C00E947A6280918F05882309F44FCF76
:108B20002EC089E697E422DF80918F05882309F41F
:108B300061CF25C089EB9BE419DF80918F058823E5
:108B400009F474CF1CC081E399E410DF80918F0594
:108B5000882309F486CF13C083E89EE407DF809161
:108B60008F05882309F49BCF0AC085E0C9CF86E32F
:108B700096E4FCDE80918F05882309F4AFCFDF9166
:108B8000CF910F9108952F923F924F925F926F92E3
:108B90007F928F929F92AF92BF92CF92DF92EF928D
:108BA000FF920F931F93CF93DF93CDB7DEB7279735
:108BB0000FB6F894DEBF0FBECDBF1C017F836E835E
:108BC0009C2C8D2CA982CA01B9010F94B8279B0156
:108BD000AC01EE81FF8160817181828193812A8362
:108BE0003B834C835D830F94B8272A813B814C8162
:108BF0005D815B016C01A21AB30AC40AD50AC801DF
:108C0000B7010F94B8272A813B814C815D817B019C
:108C10008C01E21AF30A040B150BF981FF938F9272
:108C20009F9288ED882E83E4982E6E817F81C1010A
:108C30000E94CB610F900F900F9027960FB6F8947B
:108C4000DEBF0FBECDBFDF91CF911F910F91FF907F
:108C5000EF90DF90CF90BF90AF909F908F907F90DC
:108C60006F905F904F903F902F9008956F927F92FA
:108C70008F929F92AF92BF92CF92DF92EF92FF922C
:108C80000F931F93CF93DF9300D01F92CDB7DEB722
:108C900061E081E00E942A636090B505712C61104B
:108CA00019C080917E05811104C00E941A6781114C
:108CB00095C080911F02882309F487C081E09091BC
:108CC0007E05911180E004E024E046EC5AE2672D35
:108CD0002AD87BC081E068122BC080917E0581304C
:108CE00021F40E941A67811181C080911F0288239C
:108CF00009F46BC011E080917E05813009F010E02D
:108D00008091AD0C9091AE0CA091AF0CB091B00CD5
:108D100089839A83AB83BC83CE0101960E945084E1
:108D200000E09C0142EB5AE2672D812F30D84DC004
:108D300082E0681224C080917E05823021F40E9476
:108D40001A67811184C080911F02882309F43DC0F5
:108D500011E080917E05823009F010E060911D0BDA
:108D600070911E0B80911F0B9091200BB7DD00E0DE
:108D70009C014EE95AE2672D812F09D826C083E075
:108D8000681223C080917E05833021F40E941A6707
:108D9000811175C080911F028823B9F011E0809184
:108DA0007E05833009F010E06091210B7091220B59
:108DB0008091230B9091240B91DD00E09C014EE803
:108DC0005AE2672D812F0E94C73E7394639485E019
:108DD000781265CF84E080937D0568C00E947A6236
:108DE00080918F05882309F464CF60C020E030E0D3
:108DF00048EC52E46091AD0C7091AE0C8091AF0CD8
:108E00009091B00C0F9487290F94B8271F921F924E
:108E10001F9222ED822E23E4922E5B016C011CE353
:108E2000E12E16E8F12E01E010E020E030E0A9018B
:108E30006DEA7CE08CEB9AE20E94CB610F900F9080
:108E40000F9080918F05882309F44FCF2FC081E0C8
:108E50000E940F67A12CC12CD12CE12CF12C08E42D
:108E600013E420E030E0A9016DE17BE088EA9AE2BA
:108E70008ADE80918F05882309F465CF17C081E0D1
:108E80000E940F67A12CC12CD12CE12CF12C08E4FD
:108E900013E420E030E0A90161E27BE086E99AE298
:108EA00072DE80918F05882309F474CF0F900F90A4
:108EB0000F900F90DF91CF911F910F91FF90EF9046
:108EC000DF90CF90BF90AF909F908F907F906F90EA
:108ED0000895AF92CF92DF92EF92FF920F931F937C
:108EE000CF93DF9361E081E00E942A63D091B505C2
:108EF000C0E0D1111AC080917E05811104C00E948A
:108F00001A67811103C180911F02882309F4F5C0FB
:108F100081E090917E05911180E004E024E04CE72F
:108F20005AE26C2F0E94933EE8C0D13029F580911F
:108F30007E05813021F40E941A678111EFC0809173
:108F40001F02882309F4D9C011E080917E05813089
:108F500009F010E060915F0D7091600D8091610DDE
:108F60009091620DBBDC00E09C014EE65AE26C2F52
:108F7000812F0E94C73EC1C0D23029F580917E0565
:108F8000823021F40E941A678111E2C080911F0291
:108F9000882309F4B2C011E080917E05823009F087
:108FA00010E06091630D7091640D8091650D90915A
:108FB000660D94DC00E09C0140E65AE26C2F812FA4
:108FC0000E94C73E9AC0D33029F580917E05833038
:108FD00021F40E941A678111D5C080911F02882355
:108FE00009F48BC011E080917E05833009F010E018
:108FF0006091670D7091680D8091690D90916A0D77
:109000006DDC00E09C0142E55AE26C2F812F0E944A
:10901000C73E73C0D43029F580917E05843021F499
:109020000E941A678111C8C080911F02882309F429
:1090300064C011E080917E05843009F010E06091F9
:109040006B0D70916C0D80916D0D90916E0D46DCE5
:1090500000E09C0144E45AE26C2F812F0E94C73E3D
:109060004CC0D53029F580917E05853021F40E94D1
:109070001A678111BBC080911F02882309F43DC08B
:1090800011E080917E05853009F010E060917B0D44
:1090900070917C0D80917D0D90917E0D1FDC00E024
:1090A0009C014AE35AE26C2F812F0E94C73E25C0E3
:1090B000D63019F580917E05863021F40E941A671A
:1090C0008111ADC080911F028823B9F011E0809119
:1090D0007E05863009F010E060917F0D7091800D63
:1090E0008091810D9091820DF9DB00E09C0146E2B8
:1090F0005AE26C2F812F0E94C73ECF5FDF5FC530E1
:1091000009F0F7CE87E080937D05A1C00E947A62C6
:1091100080918F05882309F4F6CE99C081E00E94E2
:109120000F67A12CC12CD12CE12C10ECF12E09E7FA
:1091300014E420E030E040E85FE36FE57DE085E7A0
:109140009AE221DD80918F05882309F4F8CE7FC053
:1091500081E00E940F67A12CC12CD12CE12C10ECD6
:10916000F12E09E714E420E030E040E85FE363E635
:109170007DE087E69AE207DD80918F05882309F478
:1091800005CF65C081E00E940F67A12CC12CD12CB6
:10919000E12C10ECF12E09E714E420E030E040E887
:1091A0005FE367E67DE089E59AE2EDDC80918F057B
:1091B000882309F412CF4BC081E00E940F67A12CD5
:1091C000C12CD12CE12C10ECF12E09E714E420E0A5
:1091D00030E040E85FE36BE67DE08BE49AE2D3DCCD
:1091E00080918F05882309F41FCF31C081E00E9450
:1091F0000F67A12CC12CD12CE12C10ECF12E09E72A
:1092000014E420E030E0A9016BE77DE08FE39AE20F
:10921000BADC80918F05882309F42DCF18C081E036
:109220000E940F67A12CC12CD12CE12C10ECF12E47
:1092300009E714E420E030E0A9016FE77DE080E376
:109240009AE2A1DC80918F05882309F43BCFDF915E
:10925000CF911F910F91FF90EF90DF90CF90AF9043
:1092600008956F927F928F929F92AF92BF92CF920A
:10927000DF92EF92FF920F931F93CF93DF9300D073
:109280001F92CDB7DEB761E081E00E942A63609053
:10929000B505712C61101AC080917E05811104C042
:1092A0000E941A678111BFC080911F02882309F4B0
:1092B000B2C081E090917E05911180E004E024E04D
:1092C00048E959E2672D0E94933EA5C021E0621251
:1092D00025C080917E05813021F40E941A6781119A
:1092E000AAC080911F02882309F495C011E08091E3
:1092F0007E05813009F010E060910B0D70910C0D2E
:1093000080910D0D90910E0DE9DA00E09C0148E886
:1093100059E2672D812F0E94C73E7DC082E068120E
:1093200025C080917E05823021F40E941A67811148
:109330009CC080911F02882309F46DC011E08091C8
:109340007E05823009F010E060910F0D7091100DD4
:109350008091110D9091120DC1DA00E09C0148E757
:1093600059E2672D812F0E94C73E55C023E062124B
:109370002CC080917E05833021F40E941A678111F0
:109380008EC080911F02882309F445C011E08091AE
:109390007E05833009F010E08091130D9091140D3B
:1093A000A091150DB091160D89839A83AB83BC8370
:1093B000CE0101960E94B68600E09C0148E659E283
:1093C000672D812F0E94C73E26C084E0681223C00B
:1093D00080917E05843021F40E941A67811199C022
:1093E00080911F028823B9F011E080917E058430BE
:1093F00009F010E06091170D7091180D8091190D12
:1094000090911A0D6BDA00E09C0148E559E2672D56
:10941000812F0E94C73E7394639425E072123ACF65
:1094200070927D058FC00E947A6280918F0588239B
:1094300009F43ACF87C081E00E940F67A12CC12CAC
:10944000D12CE12C10E8F12E07E714E420E030E005
:1094500040E85FE36BE07DE080E999E294DB809196
:109460008F05882309F43DCF6DC081E00E940F670E
:10947000A12CC12CD12CE12C10E8F12E07E714E42B
:1094800020E030E040E85FE36FE07DE080E899E2D3
:109490007ADB80918F05882309F44BCF53C081E09C
:1094A0000E940F6720E030E048EC52E46091130D19
:1094B0007091140D8091150D9091160D0F948729C0
:1094C0000F94B8275B016C012AE0A21AB108C10809
:1094D000D1081F921F921F929AEE892E93E4992E23
:1094E0001EEAE12E12E8F12E01E010E02AE030E061
:1094F00040E050E063E17DE080E799E20E94CB61CB
:109500000F900F900F9080918F05882309F439CF29
:1095100019C081E00E940F67A12CC12CD12CE12C35
:1095200010E8F12E07E714E420E030E040E85FE3C4
:1095300067E17DE080E699E226DB80918F05882354
:1095400009F44ECF0F900F900F900F90DF91CF91B5
:109550001F910F91FF90EF90DF90CF90BF90AF9051
:109560009F908F907F906F9008952F923F924F928F
:109570005F926F927F928F929F92AF92BF92CF92A3
:10958000DF92EF92FF920F931F93CF93DF93CDB7AC
:10959000DEB727970FB6F894DEBF0FBECDBF1C0114
:1095A0007F836E83CA01B901E982FA820B831C832F
:1095B0009C2C8D2CAD822AE037ED43E25CE30F94C6
:1095C00087290F94B8272B013C012AE037ED43E2AD
:1095D0005CE3EE81FF8160817181828193810F94D0
:1095E00087290F94B8275B016C01A418B508C60839
:1095F000D7082AE037ED43E25CE3C801B7010F94D6
:1096000087290F94B8277B018C01E418F508060917
:109610001709FD81FF938F929F928EED882E83E430
:10962000982EA30192016E817F81C1010E94CB61BE
:109630000F900F900F9027960FB6F894DEBF0FBED5
:10964000CDBFDF91CF911F910F91FF90EF90DF90F1
:10965000CF90BF90AF909F908F907F906F905F90D2
:109660004F903F902F9008952F923F924F925F928C
:109670006F927F928F929F92AF92BF92CF92DF9222
:10968000EF92FF920F931F93CF93DF93CDB7DEB787
:1096900027970FB6F894DEBF0FBECDBF1C017F83A6
:1096A0006E83E982FA820B831C839C2C8D2CAD8205
:1096B000CA01B9010F94E9272AE037ED43E25CE3E0
:1096C0000F9487290F94B8272B013C01EE81FF816D
:1096D00060817181828193810F94E9272AE037EDBF
:1096E00043E25CE30F9487290F94B8275B016C0178
:1096F000A418B508C608D708C801B7010F94E92710
:109700002AE037ED43E25CE30F9487290F94B827F2
:109710007B018C01E418F50806091709FD81FF9308
:109720008F929F9284EE882E83E4982EA30192015B
:109730006E817F81C1010E94CB610F900F900F90CD
:1097400027960FB6F894DEBF0FBECDBFDF91CF9145
:109750001F910F91FF90EF90DF90CF90BF90AF904F
:109760009F908F907F906F905F904F903F902F9041
:1097700008959F92AF92BF92CF92DF92EF92FF92A5
:109780000F931F93CF93DF9300D01F92CDB7DEB717
:1097900061E081E00E942A639090B505B12C9110A0
:1097A0001AC080917E05811104C00E941A67811140
:1097B00052C180911F02882309F444C181E0909135
:1097C0007E05911180E004E024E044E15AE26B2D33
:1097D0000E94933E37C181E098122CC080917E0593
:1097E000813021F40E941A6781113DC180911F02CE
:1097F000882309F427C111E080917E05813009F0AA
:1098000010E080916F0D9091700DA091710DB0914D
:10981000720D89839A83AB83BC83CE0101960E942B
:10982000FE8500E09C0148E05AE26B2D812F0E94EA
:10983000C73E08C182E098122CC080917E0582301C
:1098400021F40E941A67811128C180911F02882388
:1098500009F4F8C011E080917E05823009F010E033
:109860008091730D9091740DA091750DB091760D4E
:1098700089839A83AB83BC83CE0101960E94FE85C7
:1098800000E09C0144EF59E26B2D812F0E94C73EFE
:10989000D9C083E098122CC080917E05833021F4DA
:1098A0000E941A67811113C180911F02882309F455
:1098B000C9C011E080917E05833009F010E08091ED
:1098C000770D9091780DA091790DB0917A0D8983E3
:1098D0009A83AB83BC83CE0101960E94FE8500E093
:1098E0009C0142EE59E26B2D812F0E94C73EAAC017
:1098F00084E0981228C080917E05843021F40E9473
:109900001A678111FEC080911F02882309F49AC052
:1099100011E080917E05843009F010E060913B0DEC
:1099200070913C0D80913D0D90913E0D0F94E92773
:109930000E94944400E09C0144ED59E26B2D812F7C
:109940000E94C73E7FC085E0981228C080917E05A6
:10995000853021F40E941A678111F0C080911F02A6
:10996000882309F46FC011E080917E05853009F0ED
:1099700010E060913F0D7091400D8091410D9091EC
:10998000420D0F94E9270E94944400E09C0146ECAC
:1099900059E26B2D812F0E94C73E54C086E0981279
:1099A00028C080917E05863021F40E941A678111BB
:1099B000E2C080911F02882309F444C011E0809125
:1099C0007E05863009F010E06091430D7091440DE2
:1099D0008091450D9091460D0F94E9270E94944483
:1099E00000E09C0148EB59E26B2D812F0E94C73E9D
:1099F00029C087E0981226C080917E05873021F427
:109A00000E941A678111D4C080911F028823D1F06F
:109A100011E080917E05873009F010E06091470DDC
:109A20007091480D8091490D90914A0D0F94E9274E
:109A30000E94944400E09C014AEA59E26B2D812F78
:109A40000E94C73EB394939485E0B812A8CE88E0F4
:109A500080937D05C9C00E947A6280918F0588231A
:109A600009F4A7CEC1C081E00E940F67A12CC12CD0
:109A7000D12CE12C1CE5F12E01EC17E420E030E0C4
:109A800040E251E46FE67DE08EE09AE26EDD809187
:109A90008F05882309F4AACEA7C081E00E940F6732
:109AA000A12CC12CD12CE12C1CE5F12E01EC17E4EA
:109AB00020E030E048EC52E463E77DE08EEF99E28D
:109AC00054DD80918F05882309F4BFCE8DC081E0DD
:109AD0000E940F67A12CC12CD12CE12C1CE5F12E8A
:109AE00001EC17E420E030E048EC52E467E77DE069
:109AF0008BEE99E23ADD80918F05882309F4D4CE6C
:109B000073C081E00E940F67A12C66EFC62E63E44C
:109B1000D62E18EBE12E12E8F12E01E010E024E63B
:109B200030E040E050E06BE37DE08BED99E29CDDBE
:109B300080918F05882309F4E6CE56C081E00E940B
:109B40000F67A12C46EFC42E43E4D42E18EBE12E70
:109B500012E8F12E01E010E024E630E040E050E0B1
:109B60006FE37DE08DEC99E27FDD80918F058823A6
:109B700009F4F4CE39C081E00E940F67A12C26EFD2
:109B8000C22E23E4D22E18EBE12E12E8F12E01E0D2
:109B900010E02AE030E040E050E063E47DE08FEB4D
:109BA00099E262DD80918F05882309F402CF1CC001
:109BB00081E00E940F67A12C86EFC82E83E4D82E87
:109BC00018EBE12E12E8F12E01E010E024E630E07F
:109BD00040E050E067E47DE081EB99E245DD809173
:109BE0008F05882309F410CF0F900F900F900F90DE
:109BF000DF91CF911F910F91FF90EF90DF90CF9069
:109C0000BF90AF909F9008952F923F924F925F9296
:109C10006F927F928F929F92AF92BF92CF92DF927C
:109C2000EF92FF920F931F93CF93DF93CDB7DEB7E1
:109C300027970FB6F894DEBF0FBECDBF1C017F8300
:109C40006E83CA01B901E982FA820B831C839C2CC2
:109C50008D2CAD8220E030E048EC52E40F9487294F
:109C60000F94B8272B013C0120E030E048EC52E48F
:109C7000EE81FF8160817181828193810F948729B8
:109C80000F94B8275B016C01A418B508C608D70863
:109C900020E030E048EC52E4C801B7010F94872976
:109CA0000F94B8277B018C01E418F5080609170901
:109CB000FD81FF938F929F9280EF882E83E4982EF0
:109CC000A30192016E817F81C1010E94CB610F903F
:109CD0000F900F9027960FB6F894DEBF0FBECDBF42
:109CE000DF91CF911F910F91FF90EF90DF90CF9078
:109CF000BF90AF909F908F907F906F905F904F90AC
:109D00003F902F9008959F92AF92BF92CF92DF9293
:109D1000EF92FF920F931F93CF93DF9300D01F9288
:109D2000CDB7DEB761E081E00E942A639090B5056F
:109D3000B12C91101AC080917E05811104C00E943F
:109D40001A678111D4C080911F02882309F4C7C00B
:109D500081E090917E05911180E004E024E046E4EA
:109D600059E26B2D0E94933EBAC081E098122CC03C
:109D700080917E05813021F40E941A678111BFC055
:109D800080911F02882309F4AAC011E080917E050A
:109D9000813009F010E080914F0D9091500DA0910D
:109DA000510DB091520D89839A83AB83BC83CE0150
:109DB00001960E94578700E09C0142E359E26B2D17
:109DC000812F0E94C73E8BC082E098122CC08091E8
:109DD0007E05823021F40E941A678111ACC0809107
:109DE0001F02882309F47BC011E080917E05823038
:109DF00009F010E08091530D9091540DA091550DF4
:109E0000B091560D89839A83AB83BC83CE010196B2
:109E10000E94578700E09C014EE159E26B2D812F93
:109E20000E94C73E5CC083E098122CC080917E05E2
:109E3000833021F40E941A67811199C080911F021A
:109E4000882309F44CC011E080917E05833009F02D
:109E500010E08091570D9091580DA091590DB0913F
:109E60005A0D89839A83AB83BC83CE0101960E94ED
:109E7000578700E09C014AE059E26B2D812F0E9438
:109E8000C73E2DC084E098122AC080917E058430A0
:109E900021F40E941A67811186C080911F028823D5
:109EA000F1F011E080917E05843009F010E080919E
:109EB0005B0D90915C0DA0915D0DB0915E0D89835D
:109EC0009A83AB83BC83CE0101960E94578700E042
:109ED0009C0146EF58E26B2D812F0E94C73EB39440
:109EE000939485E0B81225CFB0927D0577C00E948B
:109EF0007A6280918F05882309F425CF6FC081E0B5
:109F00000E940F67A12C68EFC62E63E4D62EE12CC9
:109F10001CE3F12E0CE116E420E030E040EA50E4CE
:109F20006FE47DE08CE399E26FDE80918F058823FA
:109F300009F426CF53C081E00E940F67A12C48EF9F
:109F4000C42E43E4D42EE12C1CE3F12E0CE116E4E4
:109F500020E030E040EA50E463E57DE088E299E209
:109F600053DE80918F05882309F439CF37C081E013
:109F70000E940F67A12C28EFC22E23E4D22EE12CE1
:109F80001CE3F12E0CE116E420E030E040EA50E45E
:109F900067E57DE084E199E237DE80918F058823D3
:109FA00009F44CCF1BC081E00E940F67A12C88EF01
:109FB000C82E83E4D82EE12C1CE3F12E0CE116E42C
:109FC00020E030E040EA50E46BE57DE080E099E29B
:109FD0001BDE80918F05882309F45FCF0F900F90CF
:109FE0000F900F90DF91CF911F910F91FF90EF9005
:109FF000DF90CF90BF90AF909F9008950F93CF9335
:10A00000DF9361E081E00E942A63D091B505C0E052
:10A01000D1111AC080917E05811104C00E941A6777
:10A0200081118BC080911F02882309F47EC081E0DA
:10A0300090917E05911180E004E024E047E35BE22B
:10A040006C2F0E94933E71C0D130D9F480917E056F
:10A05000813021F40E941A67811177C080911F021C
:10A06000882309F462C081E090917E05913009F067
:10A0700080E003E02EE340E35BE26C2F0E94933E1E
:10A0800054C0D230D9F480917E05823021F40E94F0
:10A090001A67811164C080911F02882309F445C0AA
:10A0A00081E090917E05923009F080E003E02EE39C
:10A0B00049E25BE26C2F0E94933E37C0D330D1F46B
:10A0C00080917E05833021F40E941A67811151C06E
:10A0D00080911F02882349F181E090917E059330A1
:10A0E00009F080E003E02EE342E25BE26C2F0E9485
:10A0F000933E1BC0D430C9F480917E05843021F496
:10A100000E941A6781113FC080911F02882369F065
:10A1100081E090917E05943009F080E003E02EE329
:10A1200048E15BE26C2F0E94933ECF5FDF5FC5305A
:10A1300009F06ECFC0937D052FC00E947A62809196
:10A140008F05882309F46ECF27C08AE894E50E9422
:10A15000B64480918F05882309F480CF1DC08FE815
:10A1600094E50E94B64480918F05882309F493CF2B
:10A1700013C084E994E50E94B64480918F0588233A
:10A1800009F4A6CF09C089E994E50E94B6448091FC
:10A190008F05882309F4B8CFDF91CF910F910895EF
:10A1A000CF92DF92EF92FF92CF93C82F0E94272A7F
:10A1B0006B017C0124EA30E74DE75FE36091CC0559
:10A1C0007091CD058091CE059091CF050F944927D0
:10A1D00087FD05C04AEF50E060E070E003C040E05A
:10A1E00050E0BA01C40ED51EE61EF71EC092C80587
:10A1F000D092C905E092CA05F092CB05C093200227
:10A20000CF91FF90EF90DF90CF9008952F923F92E3
:10A210004F925F926F927F928F929F92AF92BF9276
:10A22000CF92DF92EF92FF921F93CF93DF93CDB740
:10A23000DEB72A970FB6F894DEBF0FBECDBF1C0164
:10A24000162F0E941A67882329F01092E5050E94B4
:10A250007A62DAC08091DB059091DC05A091DD0582
:10A26000B091DE058F839887A987BA87892B8A2BBF
:10A270008B2B09F491C0E4E01E9FD0011124BE8312
:10A28000AD83FD01E85AFD4F4080518062807380AC
:10A2900020E030E04AE754E4C301B2010F94702695
:10A2A0006B017C0180914D028823F9F01130A9F0F7
:10A2B00058F01230D1F4C0904902D0904A02E09098
:10A2C0004B02F0904C0211C0C0904102D09042026B
:10A2D000E0904302F090440208C0C0904502D09044
:10A2E0004602E0904702F09048026F8178858985A8
:10A2F0009A850F94EB272091CC053091CD054091A4
:10A30000CE055091CF050F9487299B01AC01C30165
:10A31000B2010F9470264B015C018D819E81885A99
:10A320009D4F9E838D83DC018D929D92AD92BC9258
:10A3300013978F819885A985BA85B7FF1AC020E049
:10A3400030E04AE754E4C301B2010F946F266B0179
:10A350007C019B01AC01C501B4010F94492787FF23
:10A3600016C0AD81BE81CD92DD92ED92FC92139725
:10A370000EC0A7019601C501B4010F944C2918160F
:10A3800034F4ED81FE81C082D182E282F382812F9A
:10A3900007DF81E080931F021092DB051092DC053D
:10A3A0001092DD051092DE0580911F02882361F175
:10A3B00024E0129FF0011124E85AFD4F8081918121
:10A3C000A281B38189839A83AB83BC832DEC3CEC5F
:10A3D0004CEC5DE36091CC057091CD058091CE058C
:10A3E0009091CF050F944C2987FD05C0CE010196B1
:10A3F0000E94EE8405C060E2CE0101960E9466854F
:10A40000BC01C1010E94283F2A960FB6F894DEBF16
:10A410000FBECDBFDF91CF911F91FF90EF90DF90E6
:10A42000CF90BF90AF909F908F907F906F905F90F4
:10A430004F903F902F90089560E08FEA9BE2E6CE28
:10A4400061E088EA9BE2E2CE62E081EA9BE2DECE56
:10A45000CF93DF9300D01F92CDB7DEB70E941A676B
:10A46000882329F01092E5050E947A625DC0609110
:10A47000DB057091DC058091DD059091DE056115AD
:10A4800071058105910569F10F94EB272091CC05A9
:10A490003091CD054091CE055091CF050F9487297D
:10A4A0009B01AC016091640270916502809166022B
:10A4B000909167020F947026609364027093650216
:10A4C000809366029093670283E06ADE81E0809366
:10A4D0001F021092DB051092DC051092DD05109230
:10A4E000DE0580911F028823F9F0209168053091E4
:10A4F000690540916A0550916B0560916402709105
:10A50000650280916602909167020F946F266983BD
:10A510007A838B839C83CE0101960E94EE84BC01DA
:10A5200080E49BE20E94283F0F900F900F900F90C5
:10A53000DF91CF91089521E02093E5056093CC054C
:10A540007093CD058093CE059093CF0540E050E009
:10A55000BA0180916605909167050C944F6260E0A6
:10A5600070E080E291E4E7CF60E070E080E89FE394
:10A57000E2CF6DEC7CEC8CEC9DE3DDCFFF920F9392
:10A580001F93CF93DF93F82E709367056093660552
:10A5900061E081E00E942A63D091B505C0E091E0BE
:10A5A00081E0F816A9F1F81628F082E0F81609F40F
:10A5B0005DC08AC0D111FBC09923D9F080917E057E
:10A5C0001816BCF04091DB055091DC056091DD056B
:10A5D0007091DE054F5F5F4F6F4F7F4F4093DB05FC
:10A5E0005093DC056093DD057093DE058F5F8093EB
:10A5F0007E0580911F02882309F44AC100E010E023
:10A6000021E041E06AE97BE28C2F0E94303E40C1AC
:10A61000D111CDC09923D9F080917E051816BCF0D8
:10A620004091DB055091DC056091DD057091DE0500
:10A630004F5F5F4F6F4F7F4F4093DB055093DC05BB
:10A640006093DD057093DE058F5F80937E058091BA
:10A650001F02882309F41CC100E010E021E041E062
:10A6600063E97BE28C2F0E94303E12C1D1119FC062
:10A670009923D9F080917E051816BCF04091DB0536
:10A680005091DC056091DD057091DE054F5F5F4FF5
:10A690006F4F7F4F4093DB055093DC056093DD05E2
:10A6A0007093DE058F5F80937E0580911F02882363
:10A6B00009F4EEC000E010E021E041E06CE87BE24C
:10A6C0008C2F0E94303EE4C040916402509165029C
:10A6D0006091660270916702409368055093690526
:10A6E00060936A0570936B05D1112CC09923D9F042
:10A6F00080917E051816BCF04091DB055091DC0579
:10A700006091DD057091DE054F5F5F4F6F4F7F4FAA
:10A710004093DB055093DC056093DD057093DE0507
:10A720008F5F80937E0580911F02882309F4E8C023
:10A7300000E010E021E041E062E87BE28C2F0E9423
:10A74000303EDEC083E0F81232C06091BA0B7091E7
:10A75000BB0B8091BC0B9091BD0B20917C0B211108
:10A7600026C00F94B82720912F0230913002621733
:10A770007307ECF4D130C9F480917E05813021F467
:10A780000E941A6781118EC080911F02882369F090
:10A7900081E090917E05913009F080E004E024E0B2
:10A7A00042E75BE26C2F0E94933E82E072C0D130A0
:10A7B000D9F480917E05813021F40E941A678111BD
:10A7C00079C080911F02882309F462C081E09091D2
:10A7D0007E05913009F080E004E024E048E65BE289
:10A7E0006C2F0E94933E54C0D230D9F480917E05E4
:10A7F000823021F40E941A67811164C080911F0287
:10A80000882309F445C081E090917E05923009F0DB
:10A8100080E003E02EE34EE55BE26C2F0E94933E66
:10A8200037C0D330D1F480917E05833021F40E946B
:10A830001A67811151C080911F02882349F181E07C
:10A8400090917E05933009F080E003E02EE345E52A
:10A850005BE26C2F0E94933E1BC0D430C9F4809100
:10A860007E05843021F40E941A6781113FC08091D7
:10A870001F02882369F081E090917E05943009F0F1
:10A8800080E003E02EE34AE45BE26C2F0E94933EFB
:10A8900085E0CF5FDF5F90E0C53009F081CE809327
:10A8A0007D0532C00E947A6280918F05882309F469
:10A8B0006BCF2AC00E947A6280918F05882309F4A9
:10A8C00080CF22C08FEA92E50E94B64480918F0526
:10A8D000882309F493CF18C084EB92E50E94B64414
:10A8E00080918F05882309F4A6CF0EC089EB92E5ED
:10A8F0000E94B64480918F05882309F4B8CF04C024
:10A9000083E0F812C5CF21CFDF91CF911F910F9136
:10A91000FF9008954FEF6CE172E580E02FCE4FEF8E
:10A9200060E272E581E02ACE4FEF64E272E582E0F8
:10A9300025CE4FEF68E272E583E020CE0F93CF93F0
:10A94000DF9361E081E00E942A63D091B505C0E009
:10A95000D1111AC080917E05811104C00E941A672E
:10A9600081118BC080911F02882309F47EC081E091
:10A9700090917E05911180E004E024E043E15BE2E8
:10A980006C2F0E94933E71C0D130D9F480917E0526
:10A99000813021F40E941A67811177C080911F02D3
:10A9A000882309F462C081E090917E05913009F01E
:10A9B00080E003E02EE349E05BE26C2F0E94933ECF
:10A9C00054C0D230D9F480917E05823021F40E94A7
:10A9D0001A67811164C080911F02882309F445C061
:10A9E00081E090917E05923009F080E000E22EE354
:10A9F0004BEF5AE26C2F0E94933E37C0D330D1F414
:10AA000080917E05833021F40E941A67811151C024
:10AA100080911F02882349F181E090917E05933057
:10AA200009F080E000E22EE34DEE5AE26C2F0E9426
:10AA3000933E1BC0D430C9F480917E05843021F44C
:10AA40000E941A6781113FC080911F02882369F01C
:10AA500081E090917E05943009F080E000E22EE3E1
:10AA600048ED5AE26C2F0E94933ECF5FDF5FC53006
:10AA700009F06ECFC0937D052FC00E947A6280914D
:10AA80008F05882309F46ECF27C08EEF9FE40E94C4
:10AA9000B64480918F05882309F480CF1DC085E0DE
:10AAA0009BE20E94C96180918F05882309F493CFAE
:10AAB00013C08AEF9AE20E94C96180918F058823B2
:10AAC00009F4A6CF09C089EE9AE20E94C96180917B
:10AAD0008F05882309F4B8CFDF91CF910F910895A6
:10AAE000CF93DF93EC01CB01BA010F94EB270F94C6
:10AAF000B82779836883DF91CF91089560E775E582
:10AB000081E196E50C948E620F931F93CF93DF93B0
:10AB100061E081E00E942A63C091B505D0E081E048
:10AB2000C1112CC08823D9F080917E051816BCF085
:10AB30004091DB055091DC056091DD057091DE05EB
:10AB40004F5F5F4F6F4F7F4F4093DB055093DC05A6
:10AB50006093DD057093DE058F5F80937E058091A5
:10AB60001F02882309F441C000E010E020E041E02A
:10AB70006EE07DE28D2F0E94303E37C0C130D1F4AF
:10AB800080917E05813021F40E941A67811137C0BF
:10AB900080911F02882349F181E090917E059130D8
:10ABA00009F080E000E22EE343E05DE26D2F0E94B9
:10ABB000933E1BC0C230C9F480917E05823021F4DF
:10ABC0000E941A67811122C080911F02882369F0B8
:10ABD00081E090917E05923009F080E000E22EE362
:10ABE0004FEE5CE26D2F0E94933EDF5FCF5F80E00F
:10ABF000D53009F095CF83E080937D050DC0C093DB
:10AC0000250B80918F05882319F206C0C093250B70
:10AC100080918F058823C1F2DF91CF911F910F9111
:10AC200008950F94EB270F94B827CB010C94B183B0
:10AC3000EF92FF920F931F93CF93DF93CDB7DEB7C1
:10AC40002B970FB6F894DEBF0FBECDBF7C014091AD
:10AC50006D05842F042E000C990B20916E05223077
:10AC600051F0233019F02DE33DE20AC047FF06C042
:10AC700029E43DE205C02BE53DE202C022E53DE2CC
:10AC80009F934F933F932F938E010F5F1F4F1F93FF
:10AC90000F930F94962F40912D0250912E024F50FA
:10ACA000510997010F900F900F900F900F900F90F8
:10ACB0004E155F050CF49A013093BF0B2093BE0B29
:10ACC00080E00E949E9AC8010E9437642B960FB6BE
:10ACD000F894DEBF0FBECDBFDF91CF911F910F91D2
:10ACE000FF90EF900895E0916D0587E1E802F00193
:10ACF0001124EA54F44F808591859ACF5F926F9228
:10AD00007F928F929F92AF92BF92CF92DF92EF92FB
:10AD1000FF920F931F93CF93DF93582E80936E056E
:10AD200060936D0561E081E00E942A63D091B505D2
:10AD3000C0E081E023E7622E26E5722ED11138C0F3
:10AD40008823D9F080917E051816BCF04091DB0570
:10AD50005091DC056091DD057091DE054F5F5F4F1E
:10AD60006F4F7F4F4093DB055093DC056093DD050B
:10AD70007093DE058F5F80937E0580911F0288238C
:10AD800009F494C022E0521649F033E0531203C094
:10AD90006FE17DE205C06FE07DE202C06FE27DE21F
:10ADA00000E010E021E041E08C2F0E94303E7EC0A8
:10ADB000D130D9F480917E05813021F40E941A6748
:10ADC00081117DC080911F02882309F46FC081E04A
:10ADD00090917E05913009F080E004E024E04AE99A
:10ADE0005DE26C2F0E94933E61C0D230D9F4809115
:10ADF0007E05823021F40E941A67811168C080911B
:10AE00001F02882309F452C081E090917E059230A0
:10AE100009F080E000E22EE34EE85DE26C2F0E9434
:10AE2000933E44C0D330D1F480917E05833021F429
:10AE30000E941A67811156C080911F028823B1F1C8
:10AE400081E090917E05933009F080E000E22EE3EE
:10AE500042E85DE26C2F0E94933E28C0D43031F569
:10AE600080917E05843021F40E941A67811145C0CB
:10AE700080911F028823D1F011E080917E058430FB
:10AE800009F010E020916D0537E12303F001112452
:10AE9000EA54F44F808591850E94B18300E09C01C3
:10AEA00044E65DE26C2F812F0E94C73ECF5FDF5FDB
:10AEB00080E0C53009F042CFC0937D0555C00E94A7
:10AEC0007A6280918F05882309F47CCF4DC08091F0
:10AED000790590917A05ACDE80918F05882309F47D
:10AEE0008ECF42C080917B0590917C05A1DE809140
:10AEF0008F05882309F4A0CF37C081E00E940F6737
:10AF000060916D0527E16203B0011124FB01EA5451
:10AF1000F44FA084B184C501BB0CAA0BBB0B5C0130
:10AF20006D0138E7A31AB108C108D1086254744F03
:10AF30001F927F926F928EE7882E85E5982E1AEAEF
:10AF4000E12EF12C00E010E028E730E040E050E096
:10AF500083E79DE20E94CB610F900F900F9080914C
:10AF60008F05882309F484CFDF91CF911F910F9132
:10AF7000FF90EF90DF90CF90BF90AF909F908F9019
:10AF80007F906F905F90089560E081E0B7CE8F92E0
:10AF90009F92AF92BF92CF92DF92EF92FF920F9368
:10AFA0001F93CF93DF934C015B016A0160E085E062
:10AFB0000E942A63D091B505F12C82E0E82ED111D0
:10AFC0001AC080911F02882321F180911E028230D5
:10AFD00041F0833019F464EC7CE205C062EB7CE262
:10AFE00002C064ED7CE200E010E021E041E08F2D42
:10AFF0000E94303E0EC0D13061F480911F02882340
:10B0000041F000E010E020E041E0B4018F2D0E940B
:10B01000303EA114B10481F0D23081F480911F023E
:10B02000882309F46EC000E010E020E041E0B501A3
:10B030008F2D0E94303E65C0C2E001C0C3E0C11444
:10B04000D10491F0DC130FC080911F02882351F0CE
:10B0500000E010E020E041E0B6018F2D0E94303E7C
:10B06000CD2F01C0CD2FCF5F21E030E0A114B1047E
:10B0700011F420E030E081E090E0C114D10411F43B
:10B0800080E090E0820F931F029781F0DC130DC0E7
:10B0900080911F02882349F000E010E020E041E0A9
:10B0A0006DEE7CE28F2D0E94303ECF5FDC1314C02A
:10B0B00080911F02882371F000E010E021E040E061
:10B0C00062EE7CE28F2D0E94303E60916C058F2DE8
:10B0D0000E94CA3DE0921F02F394DF5F85E0F81200
:10B0E0006ECFCF5FC0937D05DF91CF911F910F9100
:10B0F000FF90EF90DF90CF90BF90AF909F908F9098
:10B100000895C3E0C114D10409F0ADCFADCF49EA31
:10B110005CE269E97CE280E99CE239CF40E050E002
:10B1200060E87CE287E79CE232CF40E050E068E6EE
:10B130007CE289E59CE22BCF40E050E06AE47CE2CF
:10B140008DE39CE224CF41E35CE260E27CE280E1BB
:10B150009CE21DCF40E050E062E07CE289EF9BE2A0
:10B1600016CF40E050E069EE7BE28CED9BE20FCF22
:10B1700040E050E06FEC7BE28EEC9BE208CF40E0D9
:10B1800050E06FEB7BE286EB9BE201CF61116093B5
:10B190001E0240936C05082E000C990BAA0BBB0BEA
:10B1A0008B30910580F5FC018827EA56FF4F8F4FC1
:10B1B0000D94D12A8EE898E51CC081EB98E519C062
:10B1C00083EA98E516C08AEA98E513C08FEB98E504
:10B1D00010C088EB98E50DC08CE998E50AC085E9B8
:10B1E00098E507C01092250B84E895E502C087E832
:10B1F00098E5009741F021E02093E50540E050E01C
:10B20000BA010C944F620C9474628091D00588232B
:10B2100021F01092E5050E947A620C942F3D9091E6
:10B220004F0893FB882780F993FF06C081E0909137
:10B230007F06911101C080E00895F1DF882339F085
:10B2400080914F0882FB882780F991E08927089533
:10B2500040E061E080E09ADF88E69EE20F94741699
:10B260000C9443D5EADF882321F084E69EE20F9414
:10B2700074160C9459921092FA15109277028091DC
:10B280004F08806280934F080E9461926FEF86E5BD
:10B290009EE20E94AE680C9474620F93CF93DF938A
:10B2A00061E081E00E942A63D091B505C0E08C2F57
:10B2B0008D0FC9F480917E05811104C00E941A6728
:10B2C000811133C080911F02882341F181E0909168
:10B2D0007E05911180E004E024E041E55EE26C2F00
:10B2E0000E94933E1BC08130C9F480917E0581305D
:10B2F00021F40E941A6781111FC080911F028823C8
:10B3000069F081E090917E05913009F080E000E2E3
:10B310002EE346E45EE26C2F0E94933ECF5FC53081
:10B3200031F682E080937D050CC00E947A628091A4
:10B330008F05882339F205C09EDF80918F05882311
:10B34000E1F2DF91CF910F910895EF92FF920F9369
:10B350001F93CF93DF9361E081E00E942A63C09145
:10B36000B50510E0C11118C080917E05811104C09F
:10B370000E941A67811183C180911F02882361F0A6
:10B3800081E090917E05911180E004E024E04AE3A1
:10B390005EE2612F0E94933E0E943862D82F909106
:10B3A0004F0893FBEE24E0F893FF03C038DFF82E3C
:10B3B00001C0F12CDD2309F458C0C130D9F48091CB
:10B3C0007E05813021F40E941A6781115FC180914E
:10B3D0001F02882309F46BC181E090917E059130B2
:10B3E00009F080E000E22EE34EE25EE2612F0E946F
:10B3F000933E5DC1C230D9F480917E05823021F444
:10B400000E941A67811149C180911F02882309F4A3
:10B410004EC181E090917E05923009F080E003E01A
:10B420002EE343E25EE2612F0E94933E40C1C330AF
:10B4300009F047C080917E05833021F40E941A678D
:10B44000811137C180911F02882309F430C181E046
:10B4500090917E05933009F080E003E02EE34EE109
:10B460005EE2612F0E94933E22C18091EF158230EF
:10B4700029F0E3DE811102C0D1E004C0C13009F43B
:10B4800022C1D2E0CD131BC080917E058C1304C075
:10B490000E941A67811139C180911F02882371F0BF
:10B4A00081E090917E059C1380E003E02EE348E06C
:10B4B0005EE2612F0E94933EDC2F01C0DC2FDF5F34
:10B4C00001C0D4E0CD131BC080917E058C1304C055
:10B4D0000E941A67811123C180911F02882371F095
:10B4E00081E090917E059C1380E003E02EE34CEF19
:10B4F0005DE2612F0E94933EDC2F01C0DC2F81E0D2
:10B500008D0FC81318C080917E058C1304C00E9453
:10B510001A6781110EC180911F02882361F081E0BA
:10B5200090917E059C1380E003E02EE34EEE5DE2F9
:10B53000612F0E94933E82E08D0F4091BE0B50918F
:10B54000BF0B90917C0B911107C020912F0230917D
:10B55000300242175307DCF0C81333C080917E05D8
:10B560008C1304C00E941A678111EDC080911F02E4
:10B57000882339F181E090917E059C1380E000E200
:10B580002EE346ED5DE2612F0E94933E1AC0C81380
:10B5900018C080917E058C1304C00E941A67811127
:10B5A000DBC080911F02882361F081E090917E05CD
:10B5B0009C1380E003E02EE346EC5DE2612F0E94E5
:10B5C000933EDD5FCD1318C080917E058C1304C0BF
:10B5D0000E941A678111CAC080911F02882361F0FE
:10B5E00081E090917E059C1380E003E02EE348EB20
:10B5F0005DE2612F0E94933E91E09D0FEE20E9F005
:10B60000F11035C0C91331C080917E058C1304C080
:10B610000E941A678111B4C080911F02882329F10A
:10B6200081E090917E059C1380E003E02EE34AEADE
:10B630005DE2612F0E94933E18C0C91316C080912D
:10B640007E058C1302C00E941A6780911F02882316
:10B6500061F081E090917E059C1380E000E22EE392
:10B660004FE95DE2612F0E94933E92E09D0F1F5FC4
:10B67000CF5F153009F076CE90937D058AC03AD71A
:10B6800080918F05882309F477CE83C0E1DD809116
:10B690008F05882309F49BCE7CC08DE499E50E9438
:10B6A000B64480918F05882309F4AECE72C0D4E0F1
:10B6B00026CF86E09DE50E94B64480918F058823C1
:10B6C00009F4C0CE66C080917E05813021F40E94CD
:10B6D0001A67811112C080911F028823A1F081E0B6
:10B6E00090917E05913009F080E000E22EE341E187
:10B6F0005EE2612F0E94933E06C0B4DD80918F050B
:10B70000882349F346C0D2E0DACE8EE994E50E9460
:10B71000B64480918F05882309F4BECE3AC08AE0F2
:10B720009FE50E94B64480918F05882309F4D4CE0A
:10B7300030C086EB90E60E94B64480918F05882346
:10B7400009F4E9CE26C086EE9DE223D680918F05CE
:10B75000882309F40BCF1DC084EC97E50E94B64402
:10B7600080918F05882309F41CCF13C085E099E5EB
:10B770000E94B64480918F05882309F42DCF09C01B
:10B7800080E792E40E94B64480918F05882309F4F3
:10B7900043CFDF91CF911F910F91FF90EF900895CC
:10B7A0006091B20B70E080E00C94D89260916C02D2
:10B7B00070916D02072E000C880B990B0F94EB27EC
:10B7C0002AE037ED43E25CE30F9487296093680237
:10B7D0007093690280936A0290936B020895CF93ED
:10B7E000DF93EC01CB01BA010F94EB270F94BD2737
:10B7F0006883DF91CF91089540E050E0BA0184EB77
:10B800009CE54DD610926F0510927005109271054F
:10B810001092720581E08093E505089540E050E0C4
:10B82000BA0188EB9CE53BD610926F05109270052B
:10B83000109271051092720581E08093E5050895DC
:10B8400080E00C949E9A6FEE7BE588E29CE566C6EC
:10B850000F94EB270F94BD27862F0C948B83BF92F8
:10B86000CF92DF92EF92FF920F931F93CF93DF93CC
:10B8700000D01F92CDB7DEB7B82E8B010E941A6799
:10B88000882321F01092E50535D660C0C090DB0515
:10B89000D090DC05E090DD05F090DE05C114D10408
:10B8A000E104F10439F11092DB051092DC051092ED
:10B8B000DD051092DE0581E080931F02B6018B2D1D
:10B8C0000E94C49F0D2C000CEE08FF0880916F05AC
:10B8D00090917005A0917105B0917205C80ED91EA6
:10B8E000EA1EFB1EC0926F05D0927005E0927105B2
:10B8F000F092720580911F02882341F124E0B29EEC
:10B90000C0011124FC01E55EF24F7F0160916F05DB
:10B910007091700580917105909172050F94EB27DD
:10B920009B01AC01F70160817181828193810F9449
:10B93000872969837A838B839C8360E2CE01019699
:10B940000E946685BC01C8010E94283F0F900F909D
:10B950000F900F90DF91CF911F910F91FF90EF907B
:10B96000DF90CF90BF9008956BEE7EE280E077CFBE
:10B9700060EE7EE281E073CF4F925F926F927F9292
:10B980008F929F92AF92BF92CF92DF92EF92FF92EF
:10B990000F931F93CF93DF93F901D8019E2C9A0147
:10B9A000550F440B550BEB01A880B9806501BB0C0A
:10B9B000EE08FF0856016701A21AB30AC40AD50AA5
:10B9C0002F01FF0F6608770883017201E21AF30A5C
:10B9D000040B150B9F92BF93AF93EEE78E2EE5E518
:10B9E0009E2ED9D40F900F900F90DF91CF911F9181
:10B9F0000F91FF90EF90DF90CF90BF90AF909F900E
:10BA00008F907F906F905F904F9008956F927F928C
:10BA10008F929F92AF92BF92CF92DF92EF92FF925E
:10BA20000F931F93CF93DF9361E081E013D6D09102
:10BA3000B505C0E020ED622E2BE5722ED1111AC0A3
:10BA400080917E05811104C00E941A67811121C175
:10BA500080911F02882309F413C181E090917E0533
:10BA6000911180E004E024E04BED5EE26C2F0E9437
:10BA7000933E06C1D13011F580917E05813021F4CD
:10BA80000E941A6781110CC180911F02882309F45A
:10BA9000F7C011E080917E05813009F010E08091BF
:10BAA0005202909153020E94B18300E09C014FEC3E
:10BAB0005EE26C2F812F0E94C73EE2C0D23011F5AA
:10BAC00080917E05823021F40E941A678111FAC0AC
:10BAD00080911F02882309F4D3C011E080917E0574
:10BAE000823009F010E08091BE0B9091BF0B0E9454
:10BAF000B18300E09C0141EC5EE26C2F812F0E943B
:10BB0000C73EBEC0D33011F580917E05833021F44D
:10BB10000E941A678111EBC080911F02882309F4EB
:10BB2000AFC011E080917E05833009F010E0809174
:10BB3000980B9091990B0E94B18300E09C0149EB16
:10BB40005EE26C2F812F0E94C73E9AC0D43001F56F
:10BB500080917E05843021F40E941A678111DCC037
:10BB600080911F02882309F48BC011E080917E052B
:10BB7000843009F010E08091B20B0E948B8300E0CA
:10BB80009C0141EA5EE26C2F812F0E94C73E78C083
:10BB9000D53011F580917E05853021F40E941A6719
:10BBA0008111DEC080911F02882309F469C011E071
:10BBB00080917E05853009F010E080916C029091B3
:10BBC0006D020E94B18300E09C0147E95EE26C2FA8
:10BBD000812F0E94C73E54C0D630D9F480917E0593
:10BBE000863021F40E941A678111CCC080911F0217
:10BBF000882309F445C081E090917E05963009F0D4
:10BC000080E003E02EE34CE85EE26C2F0E94933E5E
:10BC100037C0D730D1F480917E05873021F40E945F
:10BC20001A678111BCC080911F02882349F181E00D
:10BC300090917E05973009F080E003E02EE341E823
:10BC40005EE26C2F0E94933E1BC0D830C9F48091F5
:10BC50007E05883021F40E941A678111ADC0809161
:10BC60001F02882369F081E090917E05983009F0E9
:10BC700080E003E02EE342E75EE26C2F0E94933EF9
:10BC8000CF5FDF5FC53009F0D9CE89E080937D05B5
:10BC90009FC030D480918F05882309F4D9CE98C0F5
:10BCA000E12C00E010E027EE33E04AE050E062E5EE
:10BCB00072E085ED9EE260DE80918F05882309F4B5
:10BCC000E3CE86C081E00E940F67E12C00E21CE514
:10BCD00022E231E040E050E06EEB7BE088EC9EE257
:10BCE0004BDE80918F05882309F4F2CE71C081E08C
:10BCF0000E940F67E12C0BEE1AE927E830E040E0E4
:10BD000050E068E97BE08DEB9EE236DE80918F05A6
:10BD1000882309F401CF5CC081E00E940F67A090E6
:10BD2000B20BB12CC12CD12C1F927F926F9283E267
:10BD3000882E8CE5982EE12CF12C8701EA9420E0E6
:10BD400030E0A90162EB7BE08DEA9EE224D30F9004
:10BD50000F900F9080918F05882309F401CF38C090
:10BD6000E12C06ED1BE527EE33E04AE050E06CE6FF
:10BD700072E08CE99EE200DE80918F05882309F451
:10BD800011CF26C0E6D240E050E0BA018CEF9BE52F
:10BD900086D380918F05882309F428CF19C0D9D282
:10BDA00040E050E0BA018EE09CE579D380918F05A8
:10BDB000882309F438CF0CC0CCD240E050E0BA015F
:10BDC00082EA93E66CD380918F05882309F447CFEC
:10BDD000DF91CF911F910F91FF90EF90DF90CF9067
:10BDE000BF90AF909F908F907F906F9008956091DB
:10BDF000B30B70E081E00C94D89260E070E080E0DA
:10BE00000E94D89260E070E081E00E94D8920E9487
:10BE1000389B6AC32F923F924F925F926F927F92AC
:10BE20008F929F92AF92BF92CF92DF92EF92FF924A
:10BE30000F931F93CF93DF9361E081E00BD4C09108
:10BE4000B505D0E0E7EF2E2EEEE53E2EF0ED4F2EBD
:10BE5000FBE55F2EA0E26A2EACE57A2EC11119C077
:10BE600080917E05811103C0E5D78111C8C0809102
:10BE70001F02882309F492C081E090917E05911100
:10BE800080E004E024E045E45FE26D2F0E94933EF1
:10BE900085C0C13009F580917E05813019F4CAD77B
:10BEA0008111B4C080911F02882309F477C011E08A
:10BEB00080917E05813009F010E08091BE0B909159
:10BEC000BF0B0E94B18300E09C0147E35FE26D2F4E
:10BED000812F0E94C73E62C0C23009F580917E0565
:10BEE000823019F4A7D78111B9C080911F0288232D
:10BEF00009F454C011E080917E05823009F010E011
:10BF00008091980B9091990B0E94B18300E09C0165
:10BF10004FE25FE26D2F812F0E94C73E3FC0C330CA
:10BF2000F1F480917E05833019F484D78111BFC06C
:10BF300080911F02882391F111E080917E0583306A
:10BF400009F010E08091B20B0E948B8300E09C010D
:10BF500047E15FE26D2F812F0E94C73E1FC0C430B2
:10BF6000E9F480917E05843019F464D78111C2C050
:10BF700080911F02882391F011E080917E0584302A
:10BF800009F010E08091B30B0E948B8300E09C01CC
:10BF90004FEF5EE26D2F812F0E94C73E8091BE0B56
:10BFA0009091BF0B2091980B3091990B232B11F49A
:10BFB000892BE1F0C530C1F480917E05853019F4FC
:10BFC00039D78111BAC080911F02882369F081E0BE
:10BFD00090917E05953009F080E000E22EE346EF77
:10BFE0005EE26D2F0E94933E86E001C085E0DF5F38
:10BFF000CF5FD53009F032CF80937D05A4C07AD2CF
:10C0000080918F05882309F432CF9DC081E007D746
:10C01000A090BE0BB090BF0B0B2C000CCC08DD0821
:10C020001F927F926F926EE7862E65E5962E12E242
:10C03000E12EFF24F39400E010E020E030E0A901BD
:10C040006EEB7BE08EE39FE2A6D10F900F900F90F6
:10C0500080918F05882309F425CF75C081E0DFD654
:10C06000A090980BB090990B0B2C000CCC08DD081D
:10C070001F92ABEEBAE9BF93AF934EE7842E45E52E
:10C08000942E11E9E12EF12C00E010E020E030E0E8
:10C09000A90168E97BE083E39FE27DD10F900F90D7
:10C0A0000F9080918F05882309F41FCF4CC081E049
:10C0B000B6D6A090B20BB12CC12CD12C1F925F929E
:10C0C0004F9223E2822E2CE5922EE12CF12C870157
:10C0D000EA9420E030E0A90162EB7BE083E29FE29A
:10C0E0005AD10F900F900F9080918F05882309F4FB
:10C0F0001FCF29C081E093D6A090B30BB12CC12CE7
:10C10000D12C1F923F922F9283E2882E8CE5982E9D
:10C11000E12CF12C8701EA9420E030E0A90163EBE7
:10C120007BE08BE09FE237D10F900F900F908091D2
:10C130008F05882309F41CCF06C05FDE80918F0530
:10C14000882309F440CFDF91CF911F910F91FF9089
:10C15000EF90DF90CF90BF90AF909F908F907F90A7
:10C160006F905F904F903F902F9008950F931F9383
:10C17000CF93DF9361E081E06DD2D091B505C0E04F
:10C18000D11116C080917E05811103C053D6811153
:10C190009AC080911F02882309F43CC081E09091ED
:10C1A0007E05911180E004E024E049E95FE22FC0C0
:10C1B000D130B1F480917E05813019F43BD68111E4
:10C1C00089C080911F02882329F181E090917E052A
:10C1D000913009F080E003E02EE347E85FE217C00A
:10C1E000D230C1F480917E05823019F423D68111BA
:10C1F0007EC080911F02882369F081E090917E05C6
:10C20000923009F080E003E02EE348E75FE26C2F14
:10C210000E94933E2DD1182FD330D1F480917E050A
:10C22000833019F407D681116FC080911F028823D3
:10C2300009F47CC081E090917E05933009F080E0A4
:10C2400000E22EE349E65FE26C2F0E94933E6EC04F
:10C2500081116FC0D430B1F480917E05843019F41F
:10C26000E9D5811158C080911F02882319F181E01E
:10C2700090917E05943009F080E000E22EE34BE5DA
:10C280005FE215C0D530B1F480917E05853009F4A8
:10C2900049C080911F02882369F081E090917E055A
:10C2A000953009F080E000E22EE34AE45FE26C2F73
:10C2B0000E94933E86E0CF5FDF5FC53009F060CF1C
:10C2C00080937D0541C016D180918F05882309F4A4
:10C2D00060CF3AC03ED040E050E0BA018BEC94E42D
:10C2E000DED080918F05882309F46BCF2DC031D02B
:10C2F00040E050E0BA0182EA93E6D1D080918F0508
:10C30000882309F476CF20C0BAD280918F05882384
:10C3100009F48BCF19C0B6D280918F05882309F418
:10C32000A2CF12C087D5811106C0B3CF112309F463
:10C33000C1CF84E0C0CF0E9481BB81E0EFD180916A
:10C340008F05882309F4A5CFDF91CF911F910F911D
:10C350000895809190058630D8F496E0899FF00189
:10C360001124EF56FA4F2091D6053091D70531832D
:10C3700020834091DB055091DC056091DD057091D3
:10C38000DE0542835383648375838F5F80939005BA
:10C3900008950D9474162F923F924F925F926F9270
:10C3A0007F928F929F92AF92BF92CF92DF92EF9245
:10C3B000FF920F931F93CF93DF9300D000D0CDB7A0
:10C3C000DEB71C012B833C834D835E8369837A83B4
:10C3D000C0DF83E080931F0230928E0520928D058E
:10C3E00069817A8170938C0560938B052B813C81E8
:10C3F0004D815E81209387053093880540938905A0
:10C4000050938A05E0928305F09284050093850598
:10C4100010938605A092DB05B092DC05C092DD0585
:10C42000D092DE059092D7058092D6058C8D9D8D99
:10C4300090938205809381058E8D8093800526964A
:10C440000FB6F894DEBF0FBECDBFDF91CF911F9125
:10C450000F91FF90EF90DF90CF90BF90AF909F90A3
:10C460008F907F906F905F904F903F902F900895A6
:10C470008091890D9091860D891B8F7071F4909138
:10C480004F0892FB882780F992FD08C081E09091C7
:10C49000EF15913019F080E0089581E00895209122
:10C4A000D6053091D70528173907E9F09093D705BD
:10C4B0008093D6054093DB055093DC056093DD0542
:10C4C0007093DE058C53964621F41092E505109288
:10C4D00090050E94C93D82E080931F0281E0809315
:10C4E0008F051092E005089540E050E0BA018CE31A
:10C4F00096E6D5CFE0919005EE2379F0E150E093F8
:10C50000900586E0E89FF0011124EF56FA4F40E0D5
:10C5100050E0BA0180819181C2CFE6CF0F931F9383
:10C52000CF93DF93FC01EB018091DB059091DC055B
:10C53000A091DD05B091DE05B7FF08C01092DB05C4
:10C540001092DC051092DD051092DE0580918305C6
:10C5500090918405A0918505B09186054091DB05F9
:10C560005091DC056091DD057091DE05841795071B
:10C57000A607B70744F48093DB059093DC05A093EE
:10C58000DD05B093DE0580911F02882301F18091C3
:10C59000870590918805A0918905B0918A05409101
:10C5A000DB055091DC056091DD057091DE058C01A5
:10C5B0009D01040F151F261F371FC901B8011995CA
:10C5C000BC0180918D0590918E050E94283F80913D
:10C5D000D005811108C0809180058823B1F1809138
:10C5E0001F02882391F180918B0590918C05009713
:10C5F000B1F000918705109188052091890530914F
:10C600008A054091DB055091DC056091DD05709154
:10C61000DE05400F511F621F731FFE011995E09147
:10C620008105F0918205309741F08091800581115C
:10C6300003C08091D00581111995FCD3882329F07E
:10C64000DF91CF911F910F9155CFDF91CF911F9126
:10C650000F910895282F1092D5058091DB059091B8
:10C66000DC05A091DD05B091DE0581309048A10583
:10C67000B10540F01092DB051092DC051092DD054B
:10C680001092DE058091DF05882331F08091DB0573
:10C6900080937E0510928F0580917D051816FCF41D
:10C6A000082E000C990B821B910920917E05022E09
:10C6B000000C330B2817390794F097FF02C080E075
:10C6C00090E080937E05092E000CAA0BBB0B809393
:10C6D000DB059093DC05A093DD05B093DE0580912A
:10C6E0007E056623C1F09091B505891714F48093F7
:10C6F000B5052091B505022E000C330B2C5F3F4F82
:10C70000482F082E000C550B2417350734F484509D
:10C710008093B50508958093B5050895882361F049
:10C7200063E972E084E690E00F946E216AEB72E0B8
:10C7300084E690E00D946E2168EB71E084E190E076
:10C740000D946E218F929F92AF92BF92CF92DF9203
:10C75000EF92FF926FD3882359F01092E505FF9076
:10C76000EF90DF90CF90BF90AF909F908F90C2CE10
:10C7700081E08093E5058090DB059090DC05A0903A
:10C78000DD05B090DE0581149104A104B10409F423
:10C7900046C01092DB051092DC051092DD05109268
:10C7A000DE05B401092C000C880B990B0F94EB27C4
:10C7B0002091230D3091240D4091250D5091260D8F
:10C7C0000F94872920914B0C30914C0C40914D0CCB
:10C7D00050914E0C0F9470266B017C0120E030E0EC
:10C7E00040E050EC0F944C2987FD19C020E030E068
:10C7F00040EA50E4C701B6010F94492718167CF0AF
:10C80000B40182E00E94C49FC0924B0CD0924C0CA9
:10C81000E0924D0CF0924E0C82E080931F028091CA
:10C820001F028823D9F08BE49CE00E945084BC0155
:10C830008EE99FE20E94283F60914B0C70914C0C56
:10C8400080914D0C90914E0CFF90EF90DF90CF9027
:10C85000BF90AF909F908F900C94D53FFF90EF903A
:10C86000DF90CF90BF90AF909F908F90089521E080
:10C8700020937F050F94791610927F0508950E94EA
:10C8800012B84CCF0E9479C549CFFC018081089530
:10C89000FC01849108954F925F926F927F928F92E4
:10C8A0009F92AF92BF92CF92DF92EF92FF920F933F
:10C8B0001F93CF93DF936C017B015A012901672BF2
:10C8C00031F088248394912CC0E0D0E019C0F801A5
:10C8D0001182108227C03701680C791C7694679406
:10C8E000E3012197A201BE01C601F50119951816B1
:10C8F000190654F0892BC9F04301FFEF8F1A9F0AE4
:10C90000E814F90440F702C07E01FACFCE15DF0526
:10C9100030F4CE0102968816990620F02196F8018F
:10C92000D183C0838FEF9FEF05C0F801D183C0830F
:10C9300080E090E0DF91CF911F910F91FF90EF90F9
:10C94000DF90CF90BF90AF909F908F907F906F902F
:10C950005F904F9008958F929F92AF92BF92CF9227
:10C96000DF92EF92FF920F931F93CF93DF93EC012F
:10C970006B017A01FB01199587FD06C0082F10E0B5
:10C9800020E030E0219620C1982F907E903CC1F4A9
:10C99000082F0F7110E020E030E04801590186E0D7
:10C9A000880C991CAA1CBB1C8A95D1F7CE01019654
:10C9B000F60119958F7395018401082B229604C105
:10C9C000982F907F903E19F58F70882E912CA12C76
:10C9D000B12C16E0880C991CAA1CBB1C1A95D1F727
:10C9E000CE010196F60119958F73882A06E0880C0E
:10C9F000991CAA1CBB1C0A95D1F7CE010296F60120
:10CA000019958F7395018401082B2396DDC0982F0B
:10CA1000987F903F81F58770882E912CA12CB12CA6
:10CA2000F6E0880C991CAA1CBB1CFA95D1F7CE0124
:10CA30000196F60119958F73882AA6E0880C991C37
:10CA4000AA1CBB1CAA95D1F7CE010296F601199536
:10CA50008F73882AB6E0880C991CAA1CBB1CBA9557
:10CA6000D1F7CE010396F60119958F7395018401D4
:10CA7000082B2496A9C0982F9C7F983FE9F58370D6
:10CA8000882E912CA12CB12C56E0880C991CAA1C44
:10CA9000BB1C5A95D1F7CE010196F60119958F73FB
:10CAA000882A66E0880C991CAA1CBB1C6A95D1F7E1
:10CAB000CE010296F60119958F73882A76E0880CCC
:10CAC000991CAA1CBB1C7A95D1F7CE010396F601DE
:10CAD00019958F73882AE6E0880C991CAA1CBB1C48
:10CAE000EA95D1F7CE010496F60119958F73950159
:10CAF0008401082B259668C0982F9E7F9C3F09F0E3
:10CB00004AC08170882E912CA12CB12C86E0880C13
:10CB1000991CAA1CBB1C8A95D1F7CE010196F6017F
:10CB200019958F73882A96E0880C991CAA1CBB1C47
:10CB30009A95D1F7CE010296F60119958F73882A3E
:10CB400026E0880C991CAA1CBB1C2A95D1F7CE01A3
:10CB50000396F60119958F73882A36E0880C991C84
:10CB6000AA1CBB1C3A95D1F7CE010496F601199583
:10CB70008F73882A46E0880C991CAA1CBB1C4A9516
:10CB8000D1F7CE010596F60119958F7395018401B1
:10CB9000082B269619C0982F907C903849F4082FBE
:10CBA000007C003871F42196CE01F6011995F7CF7B
:10CBB000082F0E7F0D3F28F02196CE01F601199522
:10CBC000F7CF00E010E09801E114F10429F0F7013B
:10CBD0000083118322833383CE01DF91CF911F9194
:10CBE0000F91FF90EF90DF90CF90BF90AF909F900C
:10CBF0008F9008951F93CF93DF9300D01F92CDB7EE
:10CC0000DEB710E0AE014F5F5F4F65E474E6A3DE70
:10CC100049815A816B817C81452B462B472B11F032
:10CC20001F5FF0CF812F0F900F900F900F90DF912B
:10CC3000CF911F9108951F93CF93DF9300D01F9240
:10CC4000CDB7DEB710E0AE014F5F5F4F68E474E62A
:10CC500082DE49815A816B817C81452B462B472B93
:10CC600011F01F5FF0CF812F0F900F900F900F905A
:10CC7000DF91CF911F9108951092D5058091D00535
:10CC80001092D005882341F040E050E0BA0185EAD7
:10CC900099E505DC0C94943D2091520230915302A9
:10CCA0004091DB055091DC056091DD057091DE055A
:10CCB000C901840F951F2436310571F447305105A1
:10CCC0006105710514F0069732C04A3F5F4F6F4F00
:10CCD0007F4F54F506962BC02436310524F4853653
:10CCE000910514F504C08436910524F41DC08A30E2
:10CCF00091053CF0883E43E094072CF087EE93E0EA
:10CD000002C08AE090E02817390761F0909353023F
:10CD1000809352021092DB051092DC051092DD0523
:10CD20001092DE050C94B03584E690E0E3CF8A30B3
:10CD3000910504F78AE090E0E9CF80914F0882FFE7
:10CD400009C083FF04C080917F06811106C020E0E6
:10CD50002093E8058091E805089580910A06909156
:10CD60000B06A0910C06B0910D060097A105B10528
:10CD700071F3BC01CD016D597F4F8F4F9F4F24E65A
:10CD800030E040E050E00F94932A609106067091E5
:10CD9000070680910806909109060F94932AD8CF30
:10CDA000CF93DF931F92CDB7DEB78091000881113A
:10CDB00003C082E498E02FC0211103C080E098E016
:10CDC0002AC08DE0815048F0440F411DE82FF0E06B
:10CDD000EE5BF74F90814927F5CF8091C705841707
:10CDE000A9F04093C70580E098E0698303DF90E0F5
:10CDF0006981861B910997FF02C080E090E08093D3
:10CE0000D8051092D90588E0809321028091D90538
:10CE100090E08050984F0F90DF91CF9108958093CC
:10CE2000D5051092D1051092D2051092D30510921B
:10CE3000D40508958091D0051092D0050895CF9221
:10CE4000DF92EF92FF920F931F930E94272A009187
:10CE5000C3051091C4052091C5053091C6056B012D
:10CE60007C01C01AD10AE20AF30AF7FC13C0209130
:10CE7000C20520952093C205DC01CB018A549C4F4A
:10CE8000AF4FBF4F8093C3059093C405A093C505D2
:10CE9000B093C60581E09091C205911101C080E078
:10CEA0001F910F91FF90EF90DF90CF900895CF9357
:10CEB00093E090931F0281111092E7050E94272AA8
:10CEC000DC01CB018C509E4FAF4FBF4F8093E105EB
:10CED0009093E205A093E305B093E40568E873E15D
:10CEE00082E090E00F946E21C6E0C15049F00F94AB
:10CEF0000D2162E070E080E090E00E94582AF5CFBA
:10CF0000CF910895AF92BF92CF92DF92EF920F939D
:10CF10001F93CF93DF9300D01F92CDB7DEB78091E0
:10CF200020028F3F09F444C00E94272A0091C805BF
:10CF30001091C9052091CA053091CB05DC01CB01C8
:10CF4000801B910BA20BB30BB7FD32C09091860DE5
:10CF50008091890D8F5F8F70981751F1E0912002B9
:10CF600084E0E802F0011124E559FC4F20E030E0B4
:10CF700040E752E460817181828193810F94502750
:10CF800069837A838B839C83A12CB12C6501E12C6E
:10CF90008E010F5F1F4F24E632E040E652E06CE561
:10CFA00072E088E592E00E940FE48FEF8093200208
:10CFB0000F900F900F900F90DF91CF911F910F91D5
:10CFC000EF90DF90CF90BF90AF9008950F931F9395
:10CFD0000E94272A0091E1051091E2052091E305C6
:10CFE0003091E405DC01CB01801B910BA20BB30B4C
:10CFF000B7FD0FC08091030185FB992790F981E06F
:10D0000089279091030196FF8260629B84608093E0
:10D01000E7058091E70581709091E70591FD8260B9
:10D020009091B605891741F18130A9F028F082303E
:10D0300041F0833059F01EC0913089F09230A9F050
:10D0400019C0992361F0933081F014C0913069F0D8
:10D05000923081F404C0992341F0933059F49091B7
:10D06000DA059F5F9093DA0505C09091DA0591503B
:10D070009093DA058093B6051F910F910895CF9391
:10D08000DF930E94943DE4E0F1E080818F7D808316
:10D09000C5E0D1E0888180958072A3E0B1E08C93F7
:10D0A00080818F7B80838881809580748C936A983F
:10D0B000729A54985C9A82E08093E60587DF10921A
:10D0C000DA05DF91CF91089581E09091E905911102
:10D0D00001C080E00895CF93DF93209100062111D5
:10D0E0001EC0FC0101900020E9F73197EF01C81B39
:10D0F000D90BC731D10534F031972081207C2038FD
:10D10000D9F3F4CFBC01DD27AE0189EE95E00F9491
:10D110007C2FC751DA4F188283E080931F02DF9182
:10D12000CF910895CF93DF93CDB7DEB78E819091E5
:10D130000006891780F0809300069E01275F3F4F0D
:10D140004F81588566E170E089EE95E00F94C52F18
:10D1500083E080931F02DF91CF9108950F931F9377
:10D16000CF93DF938C0167FF03C01092000660E04D
:10D170008091000690E0262F062E000C330B281716
:10D1800039070CF160930006C8010F94DE2EF801F8
:10D19000E80FF91FEF01C01BD10BC731D10534F0E7
:10D1A00031978491807C8038D9F3F4CFDD27AE01AC
:10D1B000B80189EE95E00F94FF2EC751DA4F18821F
:10D1C00083E080931F02DF91CF911F910F9108950B
:10D1D0004F925F926F927F928F929F92AF92BF9287
:10D1E000CF92DF92EF92FF920F931F938BDEEEDED2
:10D1F0008091E70582FF15C08091C105811113C0A0
:10D2000091E09093C1052091FA15211103C08091FE
:10D210007F0589278093D0051092FA1581E047DEBB
:10D2200002C01092C10589B184FB992790F981E071
:10D2300089271091E6058117B9F08093E6058823C8
:10D2400009F4A6C164EF71E080E090E00E9447839A
:10D250000E946674123009F096C10E94367583E010
:10D2600080931F020E94943D0E94272A6B017C013B
:10D270008091BD059091BE05A091BF05B091C005FC
:10D28000A7019601281B390B4A0B5B0B57FF05C002
:10D290008091E005882309F427C2D701C6018C5983
:10D2A0009F4FAF4FBF4F8093BD059093BE05A09396
:10D2B000BF05B093C0056091DA05062E000C770B10
:10D2C00077FF03C0719561957109062E000C770BED
:10D2D000880B990B0F94EB272B013C0120E030E0E9
:10D2E00040E050E40F944C2987FF05C08091D005A1
:10D2F000811183C093C08091D505882309F456C05D
:10D300008090D1059090D205A090D305B090D4051F
:10D3100081149104A104B104E1F120E030E040E087
:10D320005FE3C301B2010F9487292B013C01C701C0
:10D33000B601681979098A099B090F94E9279B01AD
:10D34000AC01C301B2010F94502720E030E04AE75E
:10D3500054E40F9487294B015C0120E030E040EA5F
:10D3600052E40F944C2987FF0FC020E030E040EFDB
:10D3700051E4C501B4010F944C2987FD0AC02AE08D
:10D3800030E040E050E009C024E630E040E050E00A
:10D3900004C021E030E040E050E0C092D105D092DE
:10D3A000D205E092D305F092D40504C021E030E02C
:10D3B00040E050E0A091DA050A2E000CBB0B0F9460
:10D3C000F22A22E030E040E050E00F94B52A80914C
:10D3D000DB059091DC05A091DD05B091DE05820FA3
:10D3E000931FA41FB51F8093DB059093DC05A093CA
:10D3F000DD05B093DE051092DA05D701C601885627
:10D40000954CAF4FBF4F8093B9059093BA05A09349
:10D41000BB05B093BC0581E080931F022091D60527
:10D420003091D70546E62C33340741F48091210230
:10D43000882309F4C0C081508093210220573244D0
:10D4400071F48091D9059091D805891740F4909195
:10D450002102992309F4BFC0915090932102809139
:10D460006F0081FB222720F981FF05C080916F00AA
:10D470008D7F80936F008091990C90919A0CA09170
:10D480009B0CB0919C0C222329F020916F0022600C
:10D4900020936F003AE0B695A795979587953A95B2
:10D4A000D1F7009721E0A207B10520F08FEF9FEFA1
:10D4B000A0E0B0E09695879520911F02211105C04C
:10D4C0003091E00531110CC151C0009741F04091FD
:10D4D000B7055091B8054817590708F047C0809123
:10D4E000E005811117C0223008F08DC080916504DD
:10D4F000811107C081E0809365048CE294E00E9472
:10D50000EF2E8CE294E00E94262F81E08093DF05CD
:10D510008093E00583E00E94AD3C61E08CE294E002
:10D520000E944F2FE091D605F091D70519951092E2
:10D53000DF058091E005811172C01092D0050E9434
:10D54000272ADC01CB018C199D09AE09BF09009186
:10D55000B7051091B80520E030E0081719072A0731
:10D560003B0720F49093B8058093B7058091D605CA
:10D570009091D7058C53964609F4A3C08091E50598
:10D5800081119FC072C060E088EE9FE2E7DD67CE48
:10D590008BD5123009F463CE60E08BED9FE2DEDDC7
:10D5A0008091D6059091D7058C53964609F457CEB5
:10D5B0000E94746254CE8CE0809321028091B70562
:10D5C0009091B80501979093B8058093B70581E0D5
:10D5D00080931F0233CF96E09093210291E09093C5
:10D5E0001F028F5F8093D905D701C6018856954CDD
:10D5F000AF4FBF4F8093B9059093BA05A093BB0579
:10D60000B093BC052CCF243030F0243009F06ECF1D
:10D6100010921F026BCF81E080931F0267CF8CE2D4
:10D6200094E00E942A2F91E0811101C090E0909334
:10D63000E005992309F481CF0E94272ADC01CB0160
:10D640008C199D09AE09BF09C090B705D090B805E7
:10D65000E12CF12CC816D906EA06FB0608F044C0F6
:10D660009093B8058093B7053FC08091B90590911C
:10D67000BA05A091BB05B091BC05C81AD90AEA0A3F
:10D68000FB0AF7FE0E9474628091E00581112CC0B4
:10D6900080911F02813091F0833031F51F910F91FD
:10D6A000FF90EF90DF90CF90BF90AF909F908F90C2
:10D6B0007F906F905F904F900C94C93D10921F0225
:10D6C00013C048E9C40E4AE3D41EE11CF11CC09209
:10D6D000B905D092BA05E092BB05F092BC05D4CF53
:10D6E000009709F417CFF3CE1F910F91FF90EF90A1
:10D6F000DF90CF90BF90AF909F908F907F906F9072
:10D700005F904F90089561E029DD0C947462CF938F
:10D71000DF931F921F92CDB7DEB789839A83AFDC68
:10D7200089819A81F0DF0F900F90DF91CF910C9457
:10D73000993D80914F0882FD05C08091EF158230A0
:10D7400061F410C080910008811103C082E498E068
:10D7500002C080E098E061E0BECC813031F08DEA1B
:10D760009FE205C08EEC9FE202C082EC9FE26FEF69
:10D77000F5CC8CE396E69093D7058093D605089573
:10D7800061E0FC0180810E944C2C8FEF0C94238D72
:10D79000CF93DF93EC018A810E94E48C60E0888162
:10D7A000DF91CF910C944C2C8F929F92AF92BF92AD
:10D7B000EF92FF920F931F93CF93DF93EC018B01B6
:10D7C0007A010E94272A4B015C012CE2820E21E0A3
:10D7D000921EA11CB11C0E94FD8C8B838F3F61F4B3
:10D7E0000E94272ADC01CB0188199909AA09BB09E3
:10D7F000B7FDF1CF81E10DC08E3F51F4B701C801F3
:10D800000E94048D0E94FD8C0E94FD8C11E003C0DB
:10D810008FE0898310E0CE01B3DF812FDF91CF91BC
:10D820001F910F91FF90EF90BF90AF909F908F90BE
:10D830000895CF92DF92EF92FF926A017B010E94DE
:10D84000272AC60ED71EE81EF91E0E94FD8C8F3FA8
:10D8500061F00E94272ADC01CB018C199D09AE09D9
:10D86000BF09B7FDF2CF80E001C081E0FF90EF90EB
:10D87000DF90CF900895EF92FF921F93CF93DF93A5
:10D8800000D01F92CDB7DEB77C01162F29833A83D3
:10D890004B835C837DDF48E552E060E070E0C701C8
:10D8A000C8DF812F80640E94238D8C810E94238D8C
:10D8B0008B810E94238D8A810E94238D89810E9401
:10D8C000238D112311F087E801C085E90E94238D83
:10D8D0001C3011F40E94FD8C10E00E94FD8CF701B9
:10D8E000838387FF04C01F3F11F01F5FF6CF0F90A7
:10D8F0000F900F900F90DF91CF911F91FF90EF90BD
:10D9000008958F929F92AF92BF92CF92DF92EF9243
:10D91000FF920F931F93CF93DF93EC01162F1C827E
:10D92000198248830E94272A6B017C0120EDC20ED8
:10D9300027E0D21EE11CF11CA89561E088810E94BD
:10D940004C2C61E088810E94102C0E94F58C85E0AF
:10D950008A830E94E48C0AE08FEF0E94238D01509D
:10D96000D9F7A89520E030E0A90160E0CE0183DF7F
:10D970008B83813061F00E94272ADC01CB018C1956
:10D980009D09AE09BF09B7FDEDCF81E055C0A8954F
:10D990002AEA31E040E050E068E0CE016CDF8530FB
:10D9A00011F481E009C004E00E94FD8C8B830150DA
:10D9B000D9F78A3A51F482E08C83A8958C81823021
:10D9C00081F0812C912C540111C00E94272ADC0186
:10D9D000CB018C199D09AE09BF09B7FDD9CF82E0F3
:10D9E0002BC0812C912CA12C80E4B82E20E030E0BB
:10D9F000A90167E3CE013FDFA501940169E2CE01F1
:10DA00003ADF8B83882361F00E94272ADC01CB0157
:10DA10008C199D09AE09BF09B7FDE8CF8AE00CC09B
:10DA20008C818230D1F420E030E0A9016AE3CE019C
:10DA300022DF882329F088E08983CE01A1DE16C089
:10DA40000E94FD8C807C803C11F483E08C830E94DA
:10DA5000FD8C0E94FD8C0E94FD8CCE0191DE173062
:10DA600018F41A8381E003C088E1898380E0DF91A4
:10DA7000CF911F910F91FF90EF90DF90CF90BF90CB
:10DA8000AF909F908F9008950F931F93CF93DF9344
:10DA9000EC0189018C81833039F089E0440F551FF6
:10DAA000661F771F8A95D1F79A01AB0161E1CE011C
:10DAB000E2DE811109C040E052E0B801CE01DF9101
:10DAC000CF911F910F9170CE84E08983CE0158DEF3
:10DAD00080E0DF91CF911F910F910895CF93DF9355
:10DAE000EC01862FBA010E94288D8FEF0E94238DB2
:10DAF0008FEF0E94238D0E94FD8C8B83982F9F7146
:10DB0000953031F083E18983CE013ADE80E001C0B7
:10DB100081E0DF91CF9108950F931F93CF93DF930F
:10DB2000EC0189018C81833039F089E0440F551F65
:10DB3000661F771F8A95D1F79A01AB0168E1CE0184
:10DB40009ADE81111EC0A8016EEFCE01C7DF8823C7
:10DB5000E1F048E552E060E070E0CE016ADE882343
:10DB600071F020E030E0A9016DE0CE0184DE81118A
:10DB70000AC00E94FD8C811106C011E007C087E138
:10DB800003C086E001C086E1898310E0CE01F8DDA4
:10DB9000812FDF91CF911F910F910895CF93DF9344
:10DBA0001F92CDB7DEB72091FC153091FD15CE0147
:10DBB00001962115310519F0821B930B02C082508A
:10DBC00096410F90DF91CF910895FC01238121119F
:10DBD0000C94907E089580914F08847F8B7F809372
:10DBE0004F0810920606109207061092080610922F
:10DBF000090610920A0610920B0610920C0610925B
:10DC00000D0610927B061092BA068EE091E0EBEBC7
:10DC1000F6E0DF019C011D9221503040E1F78FEFCB
:10DC20008093FF070895FC0120E03EE2DB014C9168
:10DC3000403241F0283011F430833196DB014C91B1
:10DC4000408331962F5F6F5F7F4F2B3079F71082C3
:10DC500008952F923F924F925F926F927F928F9290
:10DC60009F92AF92BF92CF92DF92EF92FF920F936B
:10DC70001F93CF93DF93CDB7DEB7C356D1090FB64D
:10DC8000F894DEBF0FBECDBF8C015B014A014DB6DB
:10DC90005EB6312C7E0187E5E80EF11C9BE1292E52
:10DCA00040E058E0BE016F5F7F4FC5010E94007DDC
:10DCB00018160CF005C18C85282F2871203109F029
:10DCC00074C0909105069150923008F46EC06DB604
:10DCD0007EB6BE016F5F7F4FC701A5DF011511053D
:10DCE00021F0F8018081811173C021E081E090E092
:10DCF000F70101900020E9F73197EE19FF09E80FCD
:10DD0000F91F32968DB79EB78E1B9F0B0FB6F894F6
:10DD10009EBF0FBE8DBFEDB7FEB731966F012111CB
:10DD200002C0B80102C06BE773E0C6010F94672F11
:10DD3000B701C6010F94512F6BE773E0C6010F9432
:10DD4000512F1CAE1FAE21E0A701B501CE01CC962C
:10DD50000E948C8081110DC080910506811109C03F
:10DD60000E94FC8884EE91E30E94EE88C7010E9425
:10DD7000BA8BFE01FC96DE019196822D01900D92E8
:10DD80008A95E1F740E050E0BE016F5D7F4FC6012C
:10DD900060DFCE01819619DFCE01CC9616DF0FB67B
:10DDA000F8947EBE0FBE6DBE7BCF9981992309F496
:10DDB00087C0953E09F474CF9E3209F471CF9091DB
:10DDC00000089E3209F46CCF8A7009F069CF0AC04E
:10DDD000F80101900020E9F73197CF01801B910BEA
:10DDE00020E086CF81E0203109F080E090914F085B
:10DDF00080FB94F990934F08811108C0898587347E
:10DE000009F04ECF8A858E3709F44ACF80910506F6
:10DE1000813021F068F08230B9F142CF8091030661
:10DE2000909104060196909304068093030638CFE0
:10DE3000BE016F5F7F4F82E498E0F5DE01151105AA
:10DE400011F0680105C082E4C82E88E0D82E08C011
:10DE5000F60181916F018823B1F30E94638BF8CFA3
:10DE6000F60181916F01882319F00E94638BF8CF2E
:10DE700080E20E94638B6D8D7E8D8F8D98A14AE02C
:10DE800050E00E94708C0CCFBE016F5F7F4F82E428
:10DE900098E0C9DE8114910441F062E478E0C401A5
:10DEA0000F943E2F892B51F40BC0832D90E02091CD
:10DEB0000106309102068217930711F03394F0CED9
:10DEC0000FB6F8945EBE0FBE4DBECD59DF4F0FB6F4
:10DED000F894DEBF0FBECDBFDF91CF911F910F91A0
:10DEE000FF90EF90DF90CF90BF90AF909F908F907A
:10DEF0007F906F905F904F903F902F900895CF93B9
:10DF0000DF93CDB7DEB76B970FB6F894DEBF0FBEC9
:10DF1000CDBF1092050640E050E0BA0184EE97E0D4
:10DF20000E94AF7D8BE1E4EEF7E0DE0111960190F7
:10DF30000D928A95E1F740E050E0BE016F5F7F4FA0
:10DF400080E090E086DECE0101963FDE6B960FB654
:10DF5000F894DEBF0FBECDBFDF91CF9108950F9330
:10DF60001F93CF93DF93CDB7DEB72D970FB6F894FD
:10DF7000DEBF0FBECDBF80917F06882391F0BE012A
:10DF80006F5F7F4F8CE796E00E94227B8E010F5FD0
:10DF90001F4FF80181918F01882339F00E94638B14
:10DFA000F8CF8AED91E30E94EE888AE00E94638BAD
:10DFB0002D960FB6F894DEBF0FBECDBFDF91CF9187
:10DFC0001F910F910895CF92DF92EF92FF920F93DE
:10DFD0001F93CF93DF93CDB7DEB7EDB6FEB6DC016E
:10DFE0000D900020E9F79D01281B390B2C5F3F4F56
:10DFF0004DB75EB7421B530B0FB6F8945EBF0FBE12
:10E000004DBF0DB71EB70F5F1F4F9F938F9384E9CE
:10E0100091E39F938F931F930F930F94962F680113
:10E0200054E0C50ED11C0F900F900F900F900F90E1
:10E030000F90F6018081882349F0082E000C990B7F
:10E040000F94C22EF60181936F01F3CFC8010F9494
:10E05000791680E991E30F9474160FB6F894FEBE1A
:10E060000FBEEDBEDF91CF911F910F91FF90EF900A
:10E07000DF90CF90089580914F0883FF03C08460A4
:10E0800080934F08089510921C0B80914F088F7D4C
:10E090008B7F80934F080E940F59882321F08CE7D3
:10E0A00096E00C94907E0895EEDF80914F08877F74
:10E0B00080934F0808950F931F93CF93DF938B01A5
:10E0C000EA01DB016D917C910E94227BD801ED91E8
:10E0D000FC919081888191110EC08936B0F48FE255
:10E0E0008083F8018081918101969183808388816A
:10E0F0008F5F88830AC0893680F73196D801ED9307
:10E10000FC9388818F5F8883E1CFDF91CF911F914E
:10E110000F9108950F931F93CF93DF9300D0CDB746
:10E12000DEB79C012F5F3F4F3B832A832FE2FC0128
:10E13000208381E0898310E00BE18091BA061817F3
:10E1400070F4019FC0011124AE014F5F5F4FBE010B
:10E150006E5F7F4F8554994FAEDF1F5FEECF898191
:10E160008B3570F4AE014F5F5F4FBE016E5F7F4F26
:10E170008CE796E0A0DF8A819B8101979B838A834D
:10E18000EA81FB8110820F900F900F90DF91CF9169
:10E190001F910F91089580914F0882FF1FC088E55D
:10E1A00090E30E94EE8860910606709107068091C8
:10E1B0000806909109064AE050E00E94658C8FE2C3
:10E1C0000E94638B60910A0670910B0680910C0689
:10E1D00090910D064AE050E00C94708C87E490E337
:10E1E0000C94EE88EF92FF920F931F93CF93DF93DF
:10E1F0008C01FC0101900020E9F73197EF01C81B69
:10E20000D90B10927C066EE470E00F945C2F7C01B9
:10E21000009729F4FE013197E00FF11F0EC060E274
:10E2200070E00F945C2F8C010F5F1F4F6AE270E06B
:10E23000C7010F945C2FFC0131978DE081838AE048
:10E2400082831382B8018CE796E00E941F8380913D
:10E250007C06882361F00E94FF8880E390E3DF91D1
:10E26000CF911F910F91FF90EF900C94EE88DF916A
:10E27000CF911F910F91FF90EF9008958CE796E05A
:10E280000E94457E8CE796E00E94907E80914F0828
:10E290008D7F8E7F80934F0810920606109207069E
:10E2A000109208061092090681E08093150B0895DC
:10E2B0000F931F93CF93DF93CDB7DEB76B970FB656
:10E2C000F894DEBF0FBECDBF8B0122E02093050680
:10E2D000909302068093010640E050E0BA0189EC79
:10E2E00097E00E94AF7D8BE1E9ECF7E0DE0111964B
:10E2F00001900D928A95E1F7A801BE016F5F7F4FF3
:10E3000080E090E0A6DCCE0101965FDC6B960FB654
:10E31000F894DEBF0FBECDBFDF91CF911F910F915B
:10E320000895CF93DF93CDB7DEB76B970FB6F89410
:10E33000DEBF0FBECDBF81E08093050610920406BC
:10E340001092030640E050E0BA0189EC97E00E9489
:10E35000AF7D8BE1E9ECF7E0DE01119601900D92C3
:10E360008A95E1F740E050E0BE016F5F7F4F80E0AB
:10E3700090E06FDCCE01019628DC8091030690913D
:10E3800004066B960FB6F894DEBF0FBECDBFDF91CB
:10E39000CF9108952F923F924F925F926F927F920A
:10E3A0008F929F92AF92BF92CF92DF92EF92FF92A5
:10E3B0000F931F93CF93DF93CDB7DEB76C970FB654
:10E3C000F894DEBF0FBECDBF5C014C8F2DB63EB6BC
:10E3D00019821C82FB0180819E012F5F3F4F490102
:10E3E0008F3239F089EC97E0F501918380838B01BE
:10E3F00060C084EE97E0F501918380838B010F5F0D
:10E400001F4F0115110509F454C04DB65EB66FE2F9
:10E4100070E0C8010F945C2F3C010817190708F041
:10E4200048C07C01E01AF10AFF24C70101962DB70C
:10E430003EB7281B390B0FB6F8943EBF0FBE2DBF59
:10E440008DB79EB701966C01A701B8010F947C2F80
:10E45000F601EE0DFF1D10823C8D332319F0C6012D
:10E460000E94BA8BF5016081718121E0A601C4018F
:10E470000E948C80811111C0B60183E190E30E945B
:10E48000028980E190E30E94EE880FB6F8945EBEA8
:10E490000FBE4DBE00E010E00CC0F50191828082FD
:10E4A00083010F5F1F4F0FB6F8945EBE0FBE4DBEC7
:10E4B000A8CFC4018ADBC8010FB6F8943EBE0FBED8
:10E4C0002DBE6C960FB6F894DEBF0FBECDBFDF91A8
:10E4D000CF911F910F91FF90EF90DF90CF90BF9061
:10E4E000AF909F908F907F906F905F904F903F90F4
:10E4F0002F9008950F931F93CF93DF931F921F9236
:10E50000CDB7DEB720914F0823FF28C0BC0140E003
:10E51000CE0101963FDF8C01009701F1BC0189819A
:10E520009A810E946681B801882381F085E890E392
:10E530000E9402898AE00E94638B10920606109264
:10E540000706109208061092090608C08DE690E3AF
:10E550000E9402898AE690E30E94EE880F900F9055
:10E56000DF91CF911F910F910895EF92FF920F933A
:10E570001F93CF93DF9300D0CDB7DEB720914F0824
:10E5800023FF12C1F42EE62E8C010E940F5988231E
:10E5900009F457C0FF2009F461C080917B068823ED
:10E5A00059F00E94FF888BE491E30E94EE8880E09E
:10E5B00090E00F949D24F8C08EE096E0ABDDE091F2
:10E5C0007B0684E0E89FF0011124E958F94F80911F
:10E5D000060690910706A0910806B091090680836F
:10E5E0009183A283B3830E94FC88B80182E391E304
:10E5F0000E9402898AE00E94638B80917B0699E6E3
:10E60000899FB0011124625F794F87E291E30E94F4
:10E6100002898AE00E94638B4091060650910706AA
:10E62000609108067091090681E291E30E94638976
:10E630008AE00E94638B80917B068F5F80937B06CC
:10E6400025C0FF2039F00E94FC8881E191E30E94FF
:10E65000EE881CC010927B0622E001C021E02B83D3
:10E660000E94FC888CE091E30E94EE882B8121308F
:10E6700009F497C080E091E30E94EE88B80188EF2A
:10E6800090E30E9402898AE00E94638BFCDC40E0F8
:10E69000B801CE0101967EDE8C01009709F484C09A
:10E6A00069817A81EE2009F452C021E0AC018CE747
:10E6B00096E00E948C80882309F441C080918D06E9
:10E6C00090918E06A0918F06B091900680930A06D5
:10E6D00090930B06A0930C06B0930D0610920606BD
:10E6E000109207061092080610920906B8018AEEE9
:10E6F00090E30E9402898AE00E94638B40910A069F
:10E7000050910B0660910C0670910D0682EE90E31D
:10E710000E9463898AE00E94638B83ED90E30E94EC
:10E72000EE88B80180E090E0C3DD8091000881119F
:10E7300002C0C80102C080E098E060E02FC0B801CC
:10E740008FEB90E30E9402898CEB90E30FC026E5EB
:10E75000AC018CE796E00E948C8081110AC0B80160
:10E7600088EA90E30E94028985EA90E30E94EE889D
:10E770001BC080914F08816080934F08B80180E0F2
:10E7800090E096DD1092150BB80183E990E30E94AA
:10E7900002898AE00E94638B60E0C8010E946B6876
:10E7A00003C086E091E368CF0F900F900F90DF9148
:10E7B000CF911F910F91FF90EF90089520914F08F6
:10E7C000226020934F0840E060E0CFCE0F931F936C
:10E7D000CF93DF93CDB7DEB76B970FB6F894DEBF5C
:10E7E0000FBECDBF8C0119821C828091CC07811194
:10E7F00003C064EE77E002C069EC77E021E0A80195
:10E80000CE0101960E948C808823F1F08BE1FE01FD
:10E810003196A9ECB7E001900D928A95E1F7A091AD
:10E82000BA06AA30D8F481E08A0F8093BA068BE149
:10E830008A9FD0011124A554B94FE9ECF7E001906B
:10E840000D928A95E1F70AC00E94FC88B8018AEF10
:10E850009FE20E9402898AE00E94638BCE010196AA
:10E86000B4D96B960FB6F894DEBF0FBECDBFDF9163
:10E87000CF911F910F9108958091BA068823C9F016
:10E8800081508093BA06882359F090E001972BE1DC
:10E89000289FF001299FF00D1124E554F94F02C083
:10E8A000E4EEF7E08BE1A9ECB7E001900D928A95D8
:10E8B000E1F78091BA0608958BE1E4EEF7E0A9EC68
:10E8C000B7E001900D928A95E1F7089580914F0885
:10E8D000877F80934F088091E707882321F084EE9B
:10E8E00097E00E94907E45E360E085EB96E009D8D2
:10E8F000811105C00E94FC888CEC91E32AC041E0A4
:10E9000065EB76E087E996E07DD481110DC040E0AB
:10E9100065EB76E087E996E075D4811105C00E9429
:10E92000FF8888EB91E315C067E976E084EE97E015
:10E93000E5D6811105C00E94FF8887EA91E309C0EE
:10E9400080914F08886080934F080E94FC888BE973
:10E9500091E30E94EE88B0DF83E080931F02089568
:10E96000AF92BF92CF92DF92EF92FF921F93CF931D
:10E97000DF93CDB7DEB7A8970FB6F894DEBF0FBE12
:10E98000CDBF8091FF0787FD61C080914F0882FD58
:10E990005DC083FF9BDF80914F0883FF54C080914F
:10E9A000FF07082E000C990BC0969F938F9387E268
:10E9B00090E39F938F936E0181E2C80ED11CDF928A
:10E9C000CF920F94962F40E050E0BA0184EE97E08A
:10E9D0000E94AF7D0F900F900F900F900F900F90AF
:10E9E000FE0131967F0140E050E0B70184EE97E0F0
:10E9F0000E94007D18163CF5F70101900020E9F710
:10EA000031971E2F1E19115068F05701A10EB11C2D
:10EA100017FDBA94F501808190E00F94C22EF501A4
:10EA20008083F1CF8A858E37F1F245E050E0B60160
:10EA3000C7010F946E2F892BB1F6C601C4DA8091FD
:10EA4000FF078F5F01C08FEF8093FF07A8960FB677
:10EA5000F894DEBF0FBECDBFDF91CF911F91FF9025
:10EA6000EF90DF90CF90BF90AF9008951092FF0786
:10EA700023CF57CC0E9443D58CE796E00E94907E2E
:10EA800080917B06882329F1815080937B0629E6BB
:10EA9000829FC001112441E061E0825F994F65DDF2
:10EAA000E0917B0684E0E89FF0011124E958F94FDA
:10EAB000408151816281738140930606509307061D
:10EAC00060930806709309068CE796E00E94AF7D7C
:10EAD000D2CAD9DA0E941DD50F94AD210F94F2212C
:10EAE0006D3371058105910520F086EF9FE20F944B
:10EAF00074161092E8050C94996B1092E40710922A
:10EB0000E7071092C9071092CC0780E090E0FC0163
:10EB1000E554F94F108213824B968E3021E0920714
:10EB2000B1F789E18093B6061092B9061092AE064D
:10EB300010927C0610927F060895CF93DF938CE7A6
:10EB400096E043D8C9ECD7E06B97CE013ED886E07B
:10EB5000CB3BD807C9F789EC97E037D884EE97E02C
:10EB6000DF91CF9132C8CF93809154088823B9F1B7
:10EB70004091570A5091580A6091590A70915A0A67
:10EB800027E538E080915508909156080E948C6DD9
:10EB9000C82F811102C0C0E023C04091500850919D
:10EBA0005108609152087091530841155105610553
:10EBB000710591F027E538E080915508909156084D
:10EBC0000E948C6D882339F31092500810925108DE
:10EBD00010925208109253081092540801C0C1E0DC
:10EBE0008C2FCF910895CF92DF92EF92FF92CF9327
:10EBF0006B017C01C42F8091570A9091580AA09113
:10EC0000590AB0915A0A8C159D05AE05BF05C9F089
:10EC1000AADF811102C080E018C027E538E0B70103
:10EC2000A60180915508909156080E94446D882352
:10EC300091F3C092570AD092580AE092590AF09282
:10EC40005A0A81E0C11180935408CF91FF90EF9050
:10EC5000DF90CF900895CF92DF92EF92FF920F93C3
:10EC60001F93CF93DF93FC0181859285A385B485A3
:10EC70000196A11DB11D84179507A607B70710F4CB
:10EC800080E060C08789803149F4BB27A72F962F89
:10EC9000852FC388D488E588F6880FC0803281F735
:10ECA00083899489A589B6896A017B01C7E0F694B6
:10ECB000E794D794C794CA95D1F78C0D9D1DAE1DCE
:10ECC000BF1DE9016A017B018F014091570A5091F4
:10ECD000580A6091590A70915A0A84179507A60735
:10ECE000B70731F040E0BC01CD017DDF882341F260
:10ECF000F8018789803179F4B701A6015527662785
:10ED00007727440F551FFA01E95AF74F8081918107
:10ED1000A0E0B0E012C0B701A6014F7755276627E3
:10ED20007727440F551F440F551FFA01E95AF74F33
:10ED300080819181A281B381BF7088839983AA83E6
:10ED4000BB8381E0DF91CF911F910F91FF90EF90F6
:10ED5000DF90CF9008954F925F926F927F92AF9223
:10ED6000BF92CF92DF92EF92FF920F931F93CF93B8
:10ED7000DF9300D01F92CDB7DEB78C0149835A8351
:10ED80006B837C835901C12CD12C7601412C82E00C
:10ED9000582E612C712C49815A816B817C819E0196
:10EDA0002F5F3F4FC80157DF882341F1D301C201D4
:10EDB000F801058404C0880F991FAA1FBB1F0A947D
:10EDC000D2F7C80ED91EEA1EFB1E49815A816B81FB
:10EDD0007C818789803139F481E0483F5F4F61054C
:10EDE000710538F4D8CF81E0483F5F4F6F4F7F40C7
:10EDF00090F2F501C082D182E282F3820F900F90EF
:10EE00000F900F90DF91CF911F910F91FF90EF9096
:10EE1000DF90CF90BF90AF907F906F905F904F90BA
:10EE200008954F925F926F927F928F929F92AF92CE
:10EE3000BF92CF92DF92EF92FF920F931F93CF93E7
:10EE4000DF93EC016A017B01280139014230510551
:10EE50006105710510F480E064C089859A85AB85F1
:10EE6000BC850196A11DB11D84179507A607B7079C
:10EE700090F38F89803149F48D2C9E2CAF2CBB24CC
:10EE80008B899C89AD89BE890FC0803221F78B8820
:10EE90009C88AD88BE88DB01CA0157E0B695A7956E
:10EEA000979587955A95D1F7880E991EAA1EBB1E75
:10EEB00041E0C501B40197DE882369F29F89903152
:10EEC00061F4DD24EE24FF249601220F331FF901A3
:10EED000E95AF74F5182408211C0E894C7F8DD2407
:10EEE000EE24FF249601220F331F220F331FF90156
:10EEF000E95AF74F40825182628273829A89923036
:10EF000080F04D815E816F817885840E951EA61EEE
:10EF1000B71E8092500890925108A0925208B09269
:10EF20005308DF91CF911F910F91FF90EF90DF90E9
:10EF3000CF90BF90AF909F908F907F906F905F9099
:10EF40004F9008952F923F924F925F926F927F92CF
:10EF50008F929F92AF92BF92CF92DF92EF92FF92E9
:10EF60000F931F93CF93DF93CDB7DEB72F970FB6D5
:10EF7000F894DEBF0FBECDBF1C014D835E836F834F
:10EF800078873B872A87FC0181859285A385B48594
:10EF90008C019D010F5F1F4F2F4F3F4F0C871D8727
:10EFA0002E873F87AA85BB85CD90DD90ED90FC90A4
:10EFB000C114D104E104F10431F0BFEFCB1ADB0A34
:10EFC000EB0AFB0A10C0F101C080D180E280F3801F
:10EFD000F1E0F9870D811E812F81388501301105FF
:10EFE0002105310509F0198646015701412C512CA4
:10EFF0003201F10181859285A385B48548165906B1
:10F000006A067B0608F04EC00C851D852E853F855F
:10F01000081519052A053B0550F482E0882E912C2D
:10F02000A12CB12C92E0C92ED12CE12CF12C9E0107
:10F030002F5F3F4FB501A401C1010DDE882391F17F
:10F0400049815A816B817C81D501C4010196A11D42
:10F05000B11D452B462B472B19F06C017D010FC0CC
:10F06000AC01BD014C195D096E097F090D811E813E
:10F070002F813885401751076207730741F01FEF52
:10F08000411A510A610A710A4C015D01B2CF0FEFBA
:10F090001FEF2FEF3FE0B501A401C101C2DE8D8358
:10F0A000811113C01D823DC02401350121E0421AA7
:10F0B00051086108710895018401B301A201C101E1
:10F0C000B0DE882379F353014201C814D904EA045D
:10F0D000FB0450F3AA85BB854D915D916D917C91A8
:10F0E0004115510561057105A9F4EA85FB85C082CA
:10F0F000D182E282F382F985FF2399F00FEFC01AE3
:10F10000D00AE00AF00AD101CD92DD92ED92FC9294
:10F11000139707C097018601C10183DE8111E5CFF6
:10F12000C1CF8D812F960FB6F894DEBF0FBECDBF35
:10F13000DF91CF911F910F91FF90EF90DF90CF90D3
:10F14000BF90AF909F908F907F906F905F904F9007
:10F150003F902F900895AF92BF92CF92DF92EF929F
:10F16000FF920F931F93CF93DF9300D01F92CDB7E1
:10F17000DEB75C016A017B0182E090E0A0E0B0E0D4
:10F18000F50180839183A283B3839E012F5F3F4F5C
:10F19000B701A601C5015FDD882321F100E010E081
:10F1A0009801B701A601C5013CDE8823D9F0C980CA
:10F1B000DA80EB80FC80F5018789803149F481E0B9
:10F1C000F8EFCF16FFEFDF06E104F10460F4DDCFC6
:10F1D00081E098EFC9169FEFD906E9069FE0F9068E
:10F1E00010F4D3CF80E00F900F900F900F90DF912D
:10F1F000CF911F910F91FF90EF90DF90CF90BF9034
:10F20000AF9008954F925F926F927F928F929F92EC
:10F21000AF92BF92FF920F931F93CF93DF93EC01B6
:10F22000142F70935608609355081F8A82E090E06F
:10F23000A0E0B0E088839983AA83BB83109254082E
:10F2400010925008109251081092520810925308D0
:10F250008FEF9FEFDC018093570A9093580AA09399
:10F26000590AB0935A0A442371F1453008F0E0C0BE
:10F2700040E060E070E0CB01B6DC882309F4D8C040
:10F2800020E1129FA0011124495B574FFA01E2547B
:10F29000FE4F80818F7709F0CBC03C9680819181B1
:10F2A000A281B38184369105A105B10508F4C0C0DF
:10F2B000349780809180A280B38081149104A1044E
:10F2C000B10421F4B5C0812C912C540140E0C5015A
:10F2D000B40189DCF82E882309F4AAC08091620861
:10F2E000909163088115924009F0A2C0909167083F
:10F2F000992309F49DC02091650830916608232B5D
:10F3000009F496C080916408882309F491C09A8B0F
:10F310008C831D8690E061E070E02D85E22FAB01CB
:10F32000022E02C0440F551F0A94E2F78417950776
:10F3300031F031E0320F3D87283078F379C02091E9
:10F340006D0830916E082115310519F040E050E04C
:10F3500008C020917B0830917C0840917D08509135
:10F360007E082D833E834F83588780916508909156
:10F37000660824013501480E591E611C711C4B8A18
:10F380005C8A6D8A7E8A0091680810916908198FDD
:10F39000088FA0916708B0E00F94E82A460E571E28
:10F3A000681E791E4A8E5B8E6C8E7D8E85E0000F06
:10F3B000111F8A95E1F701501E4F012F1127069565
:10F3C000400E511E611C711C4E865F86688A798AC8
:10F3D00020916A0830916B082115310521F08901CF
:10F3E00020E030E008C00091770810917808209163
:10F3F000790830917A08B501A401441955096609C4
:10F400007709400F511F621F731F04C076956795DF
:10F4100057954795EA95D2F749875A876B877C8736
:10F42000453F8FE058076105710520F48CE08F8B14
:10F43000F12C15C0453F5F4F6105710510F480E167
:10F440000DC08091830890918408A0918508B091A7
:10F4500086088A8F9B8FAC8FBD8F80E28F8B8F2D1C
:10F46000DF91CF911F910F91FF90BF90AF909F9030
:10F470008F907F906F905F904F900895CF93DF9320
:10F48000EC019C012C5F3F4F41E050E060E070E0F8
:10F49000898D9A8D57DD882399F04D895E896F8912
:10F4A000788D452B462B472B59F44C815D816E811D
:10F4B0007F814D8B5E8B6F8B788F9981906899835C
:10F4C000DF91CF910895CF92DF92EF92FF920F9349
:10F4D0001F93CF93DF93DC0151964D915D916D9118
:10F4E0007C915497403E5F4F6F41710510F010E0E2
:10F4F00067C0EC01C3DF8823D1F335DB182F8823E5
:10F50000B1F3E98DFA8D8C819D81AE81BF81029727
:10F51000A109B109058404C0880F991FAA1FBB1F48
:10F520000A94D2F7C684D784E088F188C80ED91E21
:10F53000EA1EFB1E81E080935408C092570AD092C5
:10F54000580AE092590AF0925A0A80E092E0E7E500
:10F55000F8E0DF019C011D9221503040E1F701E00D
:10F56000E98DFA8D8481081798F427E538E0B70112
:10F57000A601400F511D611D711D8091550890918C
:10F5800056080E948C6D882309F4B1CF0F5FE8CF35
:10F5900040E052E060E070E0058404C0440F551F75
:10F5A000661F771F0A94D2F789899A89AB89BC892B
:10F5B000480F591F6A1F7B1F498B5A8B6B8B7C8BA3
:10F5C000812FDF91CF911F910F91FF90EF90DF90EE
:10F5D000CF900895CF93DF93EC0141E0611101C01A
:10F5E00040E06C857D858E859F85FDDA882341F01E
:10F5F000888920E2829FC0011124895A974F02C056
:10F6000080E090E0DF91CF910895FC0120E090E050
:10F610008EE23081303269F0283029F4DB01A90F05
:10F62000B11D8C939F5FDB01A90FB11D30813C930D
:10F630009F5F2F5F31962B3061F7FB01E90FF11DC2
:10F6400010820895CF93DF93FC012381211102C022
:10F6500080E010C02250223028F48FE2FB0180832A
:10F66000118207C0EB0160E0B5DF009789F3BE01AE
:10F67000CCDF81E0DF91CF9108952BE030E2215083
:10F68000FB01E20FF11D30832111F9CFDC0197E07E
:10F690003A2FEB2F8D9181110AC0DA013C9311961C
:10F6A000EC9381E0FB019081903239F525C08F32D7
:10F6B000A1F38E3229F49A30F9F028E09AE0E8CFED
:10F6C000E8EFF1E33491332321F031963813FACF88
:10F6D00013C0921788F0813278F08F3769F031E0EB
:10F6E000320FFB01E20FF11D2FE9280F2A3108F438
:10F6F00080528083232FCCCF80E008950F931F93F7
:10F70000CF93DF93FC012381222311F080E043C0DB
:10F710008B01EC01FB018789803131F18032B1F737
:10F7200083E08B83F801428D538D648D758D4D8BF5
:10F730005E8B6F8B788F9E012F5E3F4FC8010BDB76
:10F74000882321F31A8F098F81E08983188619860F
:10F750001A861B861C821D821E821F82188A1C86A6
:10F760001D861E861F8617C082E08B831D8A1E8A17
:10F770001F8A188EFB01808D918DA0E0B0E025E0FE
:10F78000880F991FAA1FBB1F2A95D1F7898B9A8BC7
:10F79000AB8BBC8BD7CFDF91CF911F910F91089589
:10F7A0002F923F924F925F926F927F928F929F9291
:10F7B000AF92BF92CF92DF92EF92FF920F931F937F
:10F7C000CF93DF9300D01F92CDB7DEB79C838B839E
:10F7D0004B015A01DC0113968C91811103C08FEF0C
:10F7E0009FEFE1C0EB81FC81818180FFF8CFEB814D
:10F7F000FC8181899289A389B4894085518562857C
:10F800007385841B950BA60BB70BA50160E070E018
:10F8100084179507A607B70708F45C0175018B816B
:10F820009C8104969A838983612C92E0792EE1145D
:10F83000F10409F48AC0AB81BC8118964D915D91A9
:10F840006D917C911B976A01B1E0DB22EB81FC8119
:10F8500023811A012B0189E0569447943794279409
:10F860008A95D1F7818D928D223061F4FC01828DD1
:10F87000938DA48DB58DBC01CD01620D731D841DCA
:10F88000951D49C0DC0114961C9111501221C11420
:10F89000D104F9F411111DC0452B462B472B59F407
:10F8A000EB81FC8185899689A789B08D84839583B6
:10F8B000A683B7830EC0AB81BC8114964D915D9138
:10F8C0006D917C91179729813A81C5D9882309F4D4
:10F8D00086CFEB81FC81218D328D84819581A6813B
:10F8E000B7810297A109B109F901058404C0880F05
:10F8F000991FAA1FBB1F0A94D2F7468557856089B6
:10F900007189840F951FA61FB71FBC01CD01610F20
:10F91000711D811D911D93012C193D0987012E1523
:10F920003F0508F489010115F2E01F0779F52091E0
:10F93000570A3091580A4091590A50915A0A621751
:10F9400073078407950719F421C0C5012CC09401E1
:10F95000AB01BC0180915508909156080E94446DFE
:10F96000882309F43CCF800E911EEB81FC818085B9
:10F970009185A285B385800F911FA11DB11D808740
:10F980009187A287B387E01AF10A51CF40E02BD9C3
:10F99000882309F424CFB601695A774FA801C4011E
:10F9A0000F94352FE0CF0F900F900F900F90DF91B5
:10F9B000CF911F910F91FF90EF90DF90CF90BF906C
:10F9C000AF909F908F907F906F905F904F903F90FF
:10F9D0002F900895CF93DF931F92CDB7DEB741E00C
:10F9E00050E0BE016F5F7F4FDBDE019719F4898124
:10F9F00090E002C08FEF9FEF0F90DF91CF910895BD
:10FA0000DF92EF92FF920F931F93CF93DF93FC014E
:10FA10002381223060F000851185228533850F71A6
:10FA2000112722273327012B022B032B11F08FEFF5
:10FA30005DC04115510511F0FA0110827A01EB0108
:10FA40008C018DE0D82E40E250E0BE01C801A8DE56
:10FA50008032910539F021E0892B09F420E0822FD2
:10FA6000819544C028812223C9F1253E11F02E3210
:10FA700031F4E114F10439F3F7011082E4CFE11419
:10FA8000F10441F13B853F733F3021F54A8D5B8D99
:10FA9000452B01F52F713FEF320F3530D8F430E0B0
:10FAA00021503109D29EC001D39E900D1124D7015F
:10FAB000A80FB91FFE0120E0AD01253088F4318187
:10FAC0003D932F5F32962D30C1F7288126FF02C06B
:10FAD000FA0115862B8523FDB6CF08C080E006C04D
:10FAE0002B3010F43481ECCF3681EACFDF91CF9107
:10FAF0001F910F91FF90EF90DF9008951F93CF9388
:10FB0000DF93FC012381223018F480E090E023C0D1
:10FB1000EC01408551856285738585E07695679512
:10FB2000579547958A95D1F7142F1F70CF0152DF53
:10FB300097FDEBCF88859985AA85BB854F96A11D3A
:10FB4000B11D88879987AA87BB87F0E21F9FC001F4
:10FB50001124895A974FDF91CF911F9108958F9269
:10FB60009F92AF92BF92CF92DF92EF92FF920F934C
:10FB70001F93CF93DF93EC018B81811102C080E052
:10FB800077C009891A892B893C890417150726072C
:10FB90003707A8F36A017B01823029F4C886D98629
:10FBA000EA86FB860DC0C114D104E104F10451F4CE
:10FBB000188619861A861B861C821D821E821F8249
:10FBC00081E056C088849984AA84BB84E98DFA8D2B
:10FBD000258530E0275F3F4FB501A4014150510911
:10FBE00061097109022E04C076956795579547956E
:10FBF0000A94D2F7D701C6010197A109B10904C03F
:10FC0000B695A795979587952A95D2F78417950766
:10FC1000A607B70720F089288A288B2849F44D8940
:10FC20005E896F89788D4C835D836E837F8304C08A
:10FC3000841B950BA60BB70B4C015D018E010C5F6D
:10FC40001F4F81149104A104B10409F4A7CF4C8182
:10FC50005D816E817F819801898D9A8D0E942B76BE
:10FC600091E0891A9108A108B1088111EACF87CFE4
:10FC7000DF91CF911F910F91FF90EF90DF90CF9088
:10FC8000BF90AF909F908F9008950F931F93CF9345
:10FC9000DF93EC018B818823D9F1898187FF32C002
:10FCA00061E0CE0197DC8C01009791F1FC0180812D
:10FCB000853E71F18B81823040F489899A89AB89C4
:10FCC000BC89848F958FA68FB78F8D899E89AF89C8
:10FCD000B88DF801938F828FB58BA48BE0915B0A6E
:10FCE000F0915C0A309759F0B8016A5E7F4FC80105
:10FCF00048961995F801808D918D938B828B89811F
:10FD00008F778983DF91CF911F910F910C94B375F9
:10FD100081E0888380E0DF91CF911F910F9108955A
:10FD2000CF93DF93EC01B1DF1B82DF91CF91089578
:10FD30004F925F926F927F928F929F92AF92BF92FB
:10FD4000EF92FF920F931F93CF93DF9300D01F92F8
:10FD5000CDB7DEB7FC0183818130E1F4818181FF81
:10FD600019C081899289A389B48984179507A60748
:10FD7000B70780F0892B8A2B8B2B09F474C04A01BA
:10FD80005B017F014084518462847384CF01E7DE8C
:10FD9000811102C080E068C0F701818D928D8114CD
:10FDA0009104A104B10469F4458956896789708D6D
:10FDB000D2D9882379F3F701158A168A178A108E0B
:10FDC00039C0F70144815581668177819E012F5F9B
:10FDD0003F4F0E942B768823E9F249815A816B813B
:10FDE0007C81F701818D928DFC012789203139F4C6
:10FDF000483FFFEF5F0761057105E0F407C0483F2A
:10FE00002FEF520762072FE07207A0F4A4D98823CE
:10FE100009F4C0CFF70144815581668177810FEFE6
:10FE20001FEF2FEF3FE0818D928D0E941177882385
:10FE300009F4B0CFF701818A928AA38AB48A8181BA
:10FE400080688183C70121DF882309F4A3CFB5012E
:10FE5000A401481459046A047B0410F4B301A201FC
:10FE6000C7017DDE01C081E00F900F900F900F90D1
:10FE7000DF91CF911F910F91FF90EF90BF90AF90C6
:10FE80009F908F907F906F905F904F9008951F93F9
:10FE9000CF93DF93EC01142F80E2689FF0011124CF
:10FEA0009F01295A374FD9011B968C91817121F0FE
:10FEB000842F827109F057C08091570A9091580A97
:10FEC000A091590AB0915A0A8C879D87AE87BF8747
:10FED000688BE95AF74F4489558960E070E0BA01B0
:10FEE000552744274D8B5E8B6F8B788F828D938D3A
:10FEF000A0E0B0E0482B592B6A2B7B2B4D8B5E8BFF
:10FF00006F8B788FD9011B968C91887151F4848DF9
:10FF1000958DA68DB78D898B9A8BAB8BBC8B81E031
:10FF20000CC0803101F59E012F5E3F4F898D9A8D67
:10FF30000E94AB768823B9F084E08B83812F8F7089
:10FF400089831C821D821E821F82188619861A864A
:10FF50001B8614FF0BC040E050E0BA01CE01E8DE82
:10FF6000811104C00FC01B8280E00CC015FF09C0C6
:10FF700049895A896B897C89CE01DF91CF911F9184
:10FF8000EECD81E0DF91CF911F910895BF92CF9286
:10FF9000DF92EF92FF920F931F93CF93DF938C0129
:10FFA000EB016A01E22E898D9A8DF801928F818F83
:10FFB00040E050E0BA01CE01D2DDF12C8885998570
:10FFC000AA85BB8549895A896B897C8984179507DD
:10FFD000A607B707C0F525E0B695A795979587952D
:10FFE0002A95D1F7F82FFF70BF2ECE0187DDDC01F7
:10FFF000892B09F486C08C91882319F0853EB9F4C9
:020000021000EC
:100000007DC0F1100EC04091570A5091580A60917E
:10001000590A70915A0AF80144875587668777878D
:10002000B08A8C91882369F0FF24F394C7CF4BE00A
:1000300050E0BD01C6010F94282F892B09F0BECFD7
:100040005AC0FF24F3948E2D8274823409F059C073
:10005000FF2049F0F801B08861E0C801BBDAEC018B
:10006000892B69F44EC08B81823009F44AC0CE01DD
:100070002ADA882309F445C0C7E5D8E0B12C80E22C
:10008000FE0111928A95E9F78BE0F601DE010190FD
:100090000D928A95E1F7E0915B0AF0915C0A309746
:1000A00039F0BE01625F7F4FCE014096199508C0BE
:1000B00081E298E2998B888B80E098E09F878E8719
:1000C000888999899B8B8A8B998F888F8E859F854C
:1000D0009F8B8E8B0E94B375882399F04E2D6B2DCC
:1000E000C801DF91CF911F910F91FF90EF90DF90AA
:1000F000CF90BF90CCCEE7FEF1CF03C0F11094CFEC
:1001000082CF80E0DF91CF911F910F91FF90EF9010
:10011000DF90CF90BF9008953F924F925F926F9281
:100120007F928F929F92AF92BF92CF92DF92EF9287
:10013000FF920F931F93CF93DF93CDB7DEB7C354D6
:10014000D1090FB6F894DEBF0FBECDBF5C016B01C5
:1001500024965FAF4EAF2497522E1C8E1F8E1982AD
:100160001C826115710511F410E074C0FC018381DB
:100170008111FACF2496EEADFFAD249780818F32A6
:10018000F1F4F60183818250823058F0618D728DD6
:10019000CE010196B3DA882339F38E010F5F1F4F2A
:1001A00001C086012496EEADFFAD249780818F3289
:1001B00039F431962496FFAFEEAF2497F3CF8B013D
:1001C0007E01FCE1EF0EF11C3701CE0101964C01DE
:1001D0004E2C3F2CAE014E5B5F4FBE01695C7F4FE2
:1001E00024968EAD9FAD249748DA882309F4BCCFBE
:1001F0002496EEADFFAD249780818F3231F4319695
:100200002496FFAFEEAF2497F3CF8823D9F021E0F7
:10021000AE01495C5F4FB801C701B8DE882309F41D
:10022000A3CF0C151D0511F0C8017ADDE614F70403
:1002300031F0942D832D8701E92EF82ECBCF982D08
:10024000892DF9CF252DAE01495C5F4FB801C5015D
:100250009DDE182FCE0101960E94E56DCE014C96D1
:100260000E94E56D812FCD5BDF4F0FB6F894DEBFA6
:100270000FBECDBFDF91CF911F910F91FF90EF90F7
:10028000DF90CF90BF90AF909F908F907F906F90B6
:100290005F904F903F900895CF93DF93EC0140E043
:1002A00050E0BA0145DD882369F061E0CE0192D9C2
:1002B000009741F025EEFC0120831B82DF91CF9156
:1002C0000C94B37580E0DF91CF9108951F93CF9385
:1002D000DF93CDB7DEB76B970FB6F894DEBF0FBED6
:1002E000CDBFAB0119821C8222E0BC01CE01019678
:1002F00013DF182F882321F0CE010196CDDF182FB0
:10030000CE0101960E94E56D812F6B960FB6F89491
:10031000DEBF0FBECDBFDF91CF911F9108952F9209
:100320003F924F925F926F927F928F929F92AF9285
:10033000BF92CF92DF92EF92FF920F931F93CF93D2
:10034000DF9300D01F92CDB7DEB78C014B013A018D
:10035000DC0113968C9113978130C1F411968C9126
:1003600081FF14C082FF18C0F80141895289638956
:10037000748980859185A285B38584179507A60722
:10038000B70751F0C801EBDB811106C081E0D8014D
:100390008C938FEF9FEF3CC1530184C0D8015996D5
:1003A0008D919C915A97FC0154805A946A017B016B
:1003B00029E0F694E794D794C7942A95D1F75C2066
:1003C0007A01F1E0FF22552009F478C080E092E044
:1003D0008E199F0965018A159B0508F46C01D801E7
:1003E00059962D913C915A9714968D919D910D900F
:1003F000BC91A02D0297A109B109F901058404C09F
:10040000880F991FAA1FBB1F0A94D2F746855785EC
:1004100060897189840F951FA61FB71F9C01AD01CC
:10042000250D311D411D511D19012A01C11432E054
:10043000D30609F08AC08091570A9091580AA0917A
:10044000590AB0915A0A82159305A405B50569F4B5
:10045000109254088FEF9FEFDC018093570A90931E
:10046000580AA093590AB0935A0A9401B201A10103
:1004700080915508909156080E948C6D882309F44C
:1004800085CFF80180859185A285B3858C0D9D1D52
:10049000A11DB11D80879187A287B3878C0C9D1CFD
:1004A000AC18BD08D80118964D915D916D917C9165
:1004B0001B97A114B10409F071CF7DC0E114F104C0
:1004C00009F084CF14964D915D916D917C911797B1
:1004D000411551056105710559F455968D919D9110
:1004E0000D90BC91A02D0097A105B10541F521C04B
:1004F0009E012F5F3F4F0E942B76882309F446CF41
:1005000089819A81AB81BC81F801218D328DF901FD
:100510002789203139F4883FFFEF9F07A105B105F6
:1005200040F40DC0883F2FEF9207A2072FE0B207DB
:1005300030F0C8010E943E7A811148CF27CFF801E0
:1005400084839583A683B78341CFE114F10419F521
:10055000D80118964D915D916D917C911B975196A4
:100560008D919D910D90BC91A02D481759076A0758
:100570007B0788F00E94B375882309F407CF81E0D8
:10058000809354082092570A3092580A4092590A90
:1005900050925A0A08C041E0C201B1010E94F375AD
:1005A000882309F4F3CEA601B401C701895A974FF5
:1005B0000F94352F66CF5196CD90DD90ED90FC9045
:1005C000549711968C91C416D506E606F70640F4AA
:1005D000F801418B528B638B748B806881830DC0D3
:1005E00020915B0A30915C0A232B39F0611471046D
:1005F00021F08068D80111968C93F801818183FDE8
:1006000002C0C30105C0C80140DB8111FACFBECED4
:100610000F900F900F900F90DF91CF911F910F913E
:10062000FF90EF90DF90CF90BF90AF909F908F9012
:100630007F906F905F904F903F902F900895FB01B7
:1006400001900020E9F73197AF01461B570B67CEA9
:10065000CF93C82F0E947EA9CC2389F024982C9A8E
:1006600065E070E080E090E00E94582A0898109AB7
:1006700065E070E080E090E0CF910C94582A249AD5
:100680002C98089A1098CF91089580E0E1CFCF92EE
:10069000DF92EF92FF926B017C0183E3C816D104D5
:1006A000E104F10470F082E3C81AD108E108F1080E
:1006B00062E370E080E090E00E94582A0E94B39CC0
:1006C000ECCFC701B6010E94582AFF90EF90DF904F
:1006D000CF900C94B39CDC01FB01460F571FE4172D
:1006E000F507C1F081912D913C911197382798E041
:1006F000B901660F771F37FF06C09B0181E22827EB
:1007000080E1382701C09B01915091F711963C93ED
:100710002E93E5CF0895282F843640F064E60F9499
:10072000602A6AE00F94602A905D01C090E2909385
:10073000610A2A3048F03AE0822F632F0F94602A32
:100740000F94602A905D01C090E29093620A822F1C
:100750006AE00F94602A905D9093630A81E69AE0C4
:1007600008959C0197FD0EC08436910584F064E6DF
:1007700070E00F94802ACB016AE070E00F94802A29
:10078000805D06C03195219531098DE201C080E27E
:100790008093610A2A30310564F0EAE0F0E0C90193
:1007A000BF010F94802ACB01BF010F94802A805D86
:1007B00001C080E28093620AC9016AE070E00F9490
:1007C000802A805D8093630A81E69AE00895AC01F7
:1007D000952F991F9927991F29F022273327241B2A
:1007E000350B01C09A01483E5340ACF0C90168EE98
:1007F00073E00F94802ACB01EAE0F0E0BF010F9490
:10080000802A805D8093600AC90164E670E00F94DD
:10081000802ACB0112C0243631050CF1911102C09F
:1008200080E201C08DE28093600AC90164E670E055
:100830000F94802ACB01EAE0F0E0BF010F94802AF8
:10084000805D8093610AC901BF010F94802ACB01AA
:10085000BF010F94802A805D8093620A16C080E2F7
:100860008093600A8093610A2A3031053CF091112F
:100870008DE28093610AEAE0F0E0E5CF911102C0D9
:1008800080E201C08DE28093620AC9016AE070E0F3
:100890000F94802A805D8093630A80E69AE0089531
:1008A0008F929F92AF92BF92CF92DF92EF92FF9280
:1008B000CF93FC01C080D180E280F38020E030E063
:1008C0004AE754E4C701B6010F9487294B015C0144
:1008D00020E030E0A901C701B6010F94492787FD48
:1008E00005C020E030E040EA50E404C020E030E001
:1008F00040EA50ECC501B4010F94702620E030E0CE
:1009000040E251E40F9450270F94B8276B017C010B
:1009100097FD10C020E137E240E050E00F94B52A87
:10092000CA01B9012AE030E040E050E00F94B52A56
:10093000605D09C0F094E094D094C094C11CD11CB7
:10094000E11CF11C6DE260935E0AC701B60128EE5E
:1009500033E040E050E00F94B52A8AE0882E912CD5
:10096000A12CB12CCA01B901A50194010F94B52A9B
:10097000605D60935F0AC701B60124E630E040E0A5
:1009800050E00F94B52ACA01B901A50194010F9452
:10099000B52A605D6093600A8EE28093610AC701A8
:1009A000B601A50194010F94B52AC62FCA01B90159
:1009B000A50194010F94B52A605D6093620AC05D41
:1009C000C093630A8EE59AE0CF91FF90EF90DF909D
:1009D000CF90BF90AF909F908F9008958F929F92ED
:1009E000AF92BF92CF92DF92EF92FF92FC01C08054
:1009F000D180E280F38020E030E048EC52E4C7018F
:100A0000B6010F9487294B015C0120E030E0A90179
:100A1000C701B6010F94492787FD05C020E030E0EB
:100A200040EA50E404C020E030E040EA50ECC50168
:100A3000B4010F94702620E030E040E251E40F94BE
:100A400050270F94B8279B0177FF06C02227332732
:100A5000261B370B8DE201C08BE280935E0AC90131
:100A600068EE73E00F94802ACB01EAE0F0E0BF016A
:100A70000F94802A805D80935F0AC90164E670E06C
:100A80000F94802ACB01BF010F94802A805D809350
:100A9000600AC901BF010F94802A282FCB01BF0132
:100AA0000F94802A805D8093610A8EE28093620AAF
:100AB000205D2093630A8EE59AE0FF90EF90DF902F
:100AC000CF90BF90AF909F908F9008958F929F92FC
:100AD000AF92BF92CF92DF92EF92FF92CF93C62F49
:100AE000FC01C080D180E280F38020E030E44CE162
:100AF00056E4C701B6010F9487294B015C0120E041
:100B000030E0A901C701B6010F94492787FD05C050
:100B100020E030E040EA50E404C020E030E040EA69
:100B200050ECC501B4010F94702620E030E040E2A3
:100B300051E40F9450270F94B8276B017C01611585
:100B400071058105910561F097FF0CC0F094E09468
:100B5000D094C094C11CD11CE11CF11C6DE203C0F7
:100B600060E201C06C2F60935E0AC701B60128EEF7
:100B700033E040E050E00F94B52A8AE0882E912CB3
:100B8000A12CB12CCA01B901A50194010F94B52A79
:100B9000605D60935F0A8EE28093600AC701B601D0
:100BA00024E630E040E050E00F94B52ACA01B901D4
:100BB000A50194010F94B52A605D6093610AC70195
:100BC000B601A50194010F94B52AC62FCA01B90137
:100BD000A50194010F94B52A605D6093620AC05D1F
:100BE000C093630A8EE59AE0CF91FF90EF90DF907B
:100BF000CF90BF90AF909F908F9008958F929F92CB
:100C0000AF92BF92CF92DF92EF92FF92FC01C08031
:100C1000D180E280F38020E030E0A901C701B60175
:100C20000F94492787FF08C0C701B601905820E0FC
:100C300030E040E251E406C020E030E040E251E420
:100C4000C701B6010F94872920E030E040EA50E464
:100C50000F94702620E030E040E251E40F945027DA
:100C60000F94B8276B017C016031F7E27F078105A3
:100C7000910584F020E137E240E050E00F94B52A7E
:100C8000CA01B9012AE030E040E050E00F94B52AF3
:100C9000605D01C060E260935F0A88EEC81683E081
:100CA000D806E104F10494F0C701B60128EE33E060
:100CB00040E050E00F94B52ACA01B9012AE030E0C3
:100CC00040E050E00F94B52A605D01C060E260939F
:100CD000600AE4E6CE16D104E104F10494F0C70101
:100CE000B60124E630E040E050E00F94B52ACA0196
:100CF000B9012AE030E040E050E00F94B52A605D91
:100D000001C060E26093610AFAE0CF16D104E10409
:100D1000F1049CF08AE0882E912CA12CB12CC70103
:100D2000B601A50194010F94B52ACA01B901A50124
:100D300094010F94B52A605D01C060E26093620A7D
:100D4000C701B6012AE030E040E050E00F94B52A38
:100D5000605D6093630A8FE59AE0FF90EF90DF900B
:100D6000CF90BF90AF909F908F9008958F929F9259
:100D7000AF92BF92CF92DF92EF92FF92CF93FC019E
:100D8000C080D180E280F38020E030E04AE754E484
:100D9000C701B6010F9487294B015C0120E030E0C8
:100DA000A901C701B6010F94492787FD05C020E0BE
:100DB00030E040EA50E404C020E030E040EA50EC8B
:100DC000C501B4010F94702620E030E040E251E408
:100DD0000F9450270F94B8276B017C0197FF0AC02E
:100DE000F094E094D094C094C11CD11CE11CF11C7F
:100DF0008DE201C08BE280935D0AC701B60120E15C
:100E000037E240E050E00F94B52A8AE0882E912C1A
:100E1000A12CB12CCA01B901A50194010F94B52AE6
:100E2000605D60935E0AC701B60128EE33E040E0E2
:100E300050E00F94B52ACA01B901A50194010F949D
:100E4000B52A605D60935F0AC701B60124E630E011
:100E500040E050E00F94B52ACA01B901A501940100
:100E60000F94B52A605D6093600A8EE28093610AF8
:100E7000C701B601A50194010F94B52AC62FCA0176
:100E8000B901A50194010F94B52A605D6093620ACF
:100E9000C05DC093630A8DE59AE0CF91FF90EF901B
:100EA000DF90CF90BF90AF909F908F9008958F92DA
:100EB0009F92AF92BF92CF92DF92EF92FF92CF9329
:100EC000FC01C080D180E280F38020E030E0A90105
:100ED000C701B6010F94492787FF08C0C701B601B3
:100EE000905820E030E04AE754E406C020E030E0CB
:100EF0004AE754E4C701B6010F94872920E030E0A7
:100F000040EA50E40F94702620E030E040E251E4E3
:100F10000F9450270F94B8276B017C01603AF6E8D4
:100F20007F07F1E08F07910584F020EA36E841E081
:100F300050E00F94B52ACA01B9012AE030E040E040
:100F400050E00F94B52A605D01C060E260935D0AD5
:100F500080E1C81687E2D806E104F10494F0C701E5
:100F6000B60120E137E240E050E00F94B52ACA0113
:100F7000B9012AE030E040E050E00F94B52A605D0E
:100F800001C060E260935E0AE8EECE16E3E0DE06A2
:100F9000E104F10494F0C701B60128EE33E040E02B
:100FA00050E00F94B52ACA01B9012AE030E040E0D0
:100FB00050E00F94B52A605D01C060E260935F0A63
:100FC000C701B60124E630E040E050E00F94B52AB6
:100FD0008AE0882E912CA12CB12CCA01B901A5015F
:100FE00094010F94B52A605D6093600A8EE280934D
:100FF000610AC701B601A50194010F94B52AC62F55
:10100000CA01B901A50194010F94B52A605D6093EE
:10101000620AC05DC093630A8DE59AE0CF91FF90AC
:10102000EF90DF90CF90BF90AF909F908F900895FA
:101030008F929F92AF92BF92CF92DF92EF92FF92E8
:10104000FC01C080D180E280F38020E030E04AE7FC
:1010500054E4C701B6010F9487294B015C0120E0DD
:1010600030E0A901C701B6010F94492787FD05C0EB
:1010700020E030E040EA50E404C020E030E040EA04
:1010800050ECC501B4010F94702620E030E040E23E
:1010900051E40F9450270F94B8276B017C0197FF00
:1010A0000AC0F094E094D094C094C11CD11CE11CFF
:1010B000F11C8DE201C080E280935D0AF0E1CF1661
:1010C000F7E2DF06E104F10494F0C701B60120E184
:1010D00037E240E050E00F94B52ACA01B9012AE096
:1010E00030E040E050E00F94B52A605D01C060E25E
:1010F00060935E0A88EEC81683E0D806E104F10426
:1011000094F0C701B60128EE33E040E050E00F94C0
:10111000B52ACA01B9012AE030E040E050E00F945E
:10112000B52A605D01C060E260935F0AC701B60145
:1011300024E630E040E050E00F94B52A8AE0882EA3
:10114000912CA12CB12CCA01B901A50194010F94D5
:10115000B52A605D6093600AC701B601A5019401DC
:101160000F94B52A6B017C01672B682B692B89F0E2
:101170008EE28093610ACA01B901A50194010F941E
:10118000B52A605D6093620A80E38C0D8093630AE8
:101190001AC0CA01B901A50194010F94B52A6115BD
:1011A00071058105910539F02EE22093610A605D99
:1011B0006093620A05C080E28093620A8093610AAC
:1011C00080E28093630A8DE59AE0FF90EF90DF90D4
:1011D000CF90BF90AF909F908F900895CF93DF9363
:1011E000FC018491EF012196882319F06CD2FE0155
:1011F000F8CFDF91CF9108958FE092E3EFCF85E1B3
:1012000092E3ECCF0F931F93CF93DF931F921F9224
:10121000CDB7DEB769837A83E1DF6981062F7A81F2
:10122000172FF80181918F01882311F04CD2F9CF4B
:101230000F900F90DF91CF911F910F910895CF9351
:10124000DF93EB01CBDF6AE070E0CE01DF91CF915D
:101250002DC3CF92DF92EF92FF926A017B01BEDF36
:101260004AE050E0C701B601FF90EF90DF90CF90C9
:101270000CC3CF92DF92EF92FF926A017B01AEDF47
:1012800042E050E0C701B601FF90EF90DF90CF90B1
:101290009AC3CF92DF92EF92FF926A017B019EDFA9
:1012A00042E050E0C701B601FF90EF90DF90CF9091
:1012B0008AC3CF93DF93EB0191DF6AE070E0CE0148
:1012C000DF91CF9108C3CF92DF92EF92FF926A0134
:1012D0007B0184DF4AE050E0C701B601FF90EF9048
:1012E000DF90CF90F2C2811103C088E092E302C088
:1012F0008CE092E373CFF7DF8AE0E5C10C94CE6D0A
:1013000081E0089581E008958F929F92AF92BF92FD
:10131000CF92DF92EF92FF920F931F93CF93DF93C1
:101320001F921F92CDB7DEB76C0159018B017B0173
:10133000E40EF51E0E151F0561F1F6018080918007
:10134000F80161918F016983C4016A830F949A3215
:101350006A81681779F0C4010F94A232C4010F9416
:101360009A329981891731F047DF8CE192E336DFB9
:1013700081E010C041E050E0BE016F5F7F4FC501CA
:10138000AAD9F601408151814F5F5F4F518340835D
:10139000D1CF80E00F900F90DF91CF911F910F91EF
:1013A000FF90EF90DF90CF90BF90AF909F908F9085
:1013B00008958F929F92AF92BF92CF92DF92EF9259
:1013C000FF920F93CF93DF931F92CDB7DEB75C01EF
:1013D0006B017A014901F501808191810F949A3264
:1013E0008983002311F0F601808341E050E0BE01C3
:1013F0006F5F7F4FC4016FD9F501408151814F5F0D
:101400005F4F51834083FFEFCF1ADF0A81E0E81A74
:10141000F10809F780E00F90DF91CF910F91FF90D5
:10142000EF90DF90CF90BF90AF909F908F900895F6
:1014300098E288E10FB6F894A895809360000FBEFB
:101440009093600008951F920F920FB60F9211248F
:101450000BB60F920F931F932F933F934F935F936E
:101460006F937F938F939F93AF93BF93CF93DF93AC
:10147000EF93FF9300918B0AD0918A0A11E01D0F20
:101480001F77C091C6009091660A492F092E000C63
:10149000550B660B770B4C30510508F046C0FA012E
:1014A0008827EF55FF4F8F4F0D94D12ACD3441F04F
:1014B000CE34B9F481E005C0CA3330F0CD3471F5D3
:1014C00082E08093660A4AC0C03308F047C0C03249
:1014D00009F444C0CD3211F541C0C13329F0C43301
:1014E00029F0C032D9F43AC083E0EBCF88E0E9CFED
:1014F000C03321F0C13391F486E0E3CF84E0E1CF43
:10150000C83361F485E0DDCFC23341F487E0D9CF41
:10151000C13321F489E0D5CFC03311F08BE0D1CFB6
:101520008AE0CFCFCA30D1F417C0CA30B9F4809165
:10153000150B882389F0973049F09A3059F095308F
:1015400059F4109277021092FA1506C081E0809348
:10155000160B02C00F9454241092660A101731F033
:10156000ED2FF0E0E657F54FC283D12FD0938A0AD2
:10157000FF91EF91DF91CF91BF91AF919F918F91AB
:101580007F916F915F914F913F912F911F910F919B
:101590000F900BBE0F900FBE0F901F9018951F92CB
:1015A0000F920FB60F9211240BB60F922F938F93B9
:1015B0009F93EF93FF938091690A2091680A2817FF
:1015C00091F0E82FF0E0E859F54F92818F5F8F712D
:1015D0009093C6008093690A9091C00090649093A4
:1015E000C000281305C08091C1008F7D8093C10089
:1015F000FF91EF919F918F912F910F900BBE0F90C4
:101600000FBE0F901F9018959B01AC011092C00067
:10161000211581EE380741055105C1F08091C000C8
:1016200082608093C00060E079E08DE390E00F94E9
:10163000B52ACA01B901615071098109910922E0F5
:1016400030E040E050E00F94B52A02C020E130E0E5
:101650003093C5002093C4008091C10080618093C5
:10166000C1008091C10088608093C1008091C10059
:1016700080688093C1008091C1008F7D8093C100FC
:101680001092670A089580918A0A90918B0A8917AF
:1016900059F0E92FF0E0E657F54F82819F5F9F7781
:1016A00090938B0A90E008958FEF9FEF0895EAE8FA
:1016B000FAE0808181830895EAE8FAE080819181EF
:1016C000891B8F77089591E09093670A9091C100EC
:1016D00095FD04C09091C00095FD40C02091680A1E
:1016E0002F5F2F710FB607FC34C09091690A291340
:1016F00022C09091C00095FF1DC09091690A409151
:10170000680A491791F0E92FF0E0E859F54F328166
:101710009F5F9F713093C6009093690A3091C0001B
:1017200030643093C000491305C09091C1009F7D83
:101730009093C100DACFE091680AF0E0E859F54FE4
:1017400082832093680A8091C10080628093C100E7
:1017500008959091690A2913EECFFBCF8093C600BC
:101760008091C00080648093C00008958DE0ABDF5D
:101770008AE0A9CFCF93DF93EC018991882311F000
:10178000A2DFFBCFDF91CF91F1CF8F929F92AF92EB
:10179000BF92EF92FF921F93CF93DF93CDB7DEB747
:1017A000A0970FB6F894DEBF0FBECDBF61157105CF
:1017B0008105910579F110E0842E912CA12CB12C9A
:1017C000EE24E394F12CEC0EFD1EE10EF11C17FD4E
:1017D000FA94A50194010F94932AF7016083B9014B
:1017E000CA011F5F611571058105910549F7115007
:1017F00010F1E1E0F0E0EC0FFD1FE10FF11D17FD2E
:10180000FA9580818A3010F097E301C090E3890F48
:101810005ADFEDCF80E3A0960FB6F894DEBF0FBE7F
:10182000CDBFDF91CF911F91FF90EF90BF90AF9010
:101830009F908F9048CFA0960FB6F894DEBF0FBE52
:10184000CDBFDF91CF911F91FF90EF90BF90AF90F0
:101850009F908F900895CF92DF92EF92FF926B014D
:101860007C0197FF0AC08DE22EDFF094E094D094C3
:10187000C094C11CD11CE11CF11C4AE0C701B60197
:10188000FF90EF90DF90CF9080CF4115510511F47C
:10189000862F19CF4A30510509F4DDCF76CFAB0141
:1018A000682F880F770B880B990BEFCFAB01BC012A
:1018B000990F880B990BE9CFAB01BC01990F880BED
:1018C000990BE3DF53CFE1DF51CF4115510511F4FF
:1018D000862FF9CE5ACFAB01BC0180E090E0F5CF66
:1018E000F4DF44CF8F929F92AF92BF92CF92DF925C
:1018F000EF92FF92CF936B017C01B42E20E030E099
:10190000A9010F94492787FF06C08DE2DCDEF7FAB4
:10191000F094F7F8F094C0E060E070E080E09FE3BE
:10192000CB1541F02DEC3CEC4CEC5DE30F9487299A
:10193000CF5FF6CF9B01AC01C701B6010F947026B3
:101940006B017C010F94BD274B015C014AE01DDF58
:10195000CC2379F1C501B4010F94E9279B01AC01B7
:10196000C701B6010F946F266B017C018EE2ABDEDE
:1019700020E030E040E251E4C701B6010F9487292E
:101980004B015C010F94B8276B01770FEE08FF083D
:10199000C701B60160DFC701B6010F94EB279B01B9
:1019A000AC01C501B4010F946F266B017C01C150DD
:1019B000F9F6CF91FF90EF90DF90CF90BF90AF906E
:1019C0009F908F9008958ECF909164009B7F90930D
:1019D0006400982F906A96959CBD80FD03C091E0AD
:1019E000863009F490E09DBD0895209A289A219AA6
:1019F0002398229A209A81E0E7CF8FEF8EBD0DB415
:101A000007FEFDCF8EB5089561157105D9F06150BF
:101A100071092FEF2EBDFC014FEF9F01281B390BE1
:101A20002617370738F40DB407FEFDCF2EB52193E6
:101A30004EBDF3CF0DB407FEFDCF2EB5FC01E60F72
:101A4000F71F208308958EBD0DB407FEFDCF0895C6
:101A50008EBD80E090E00DB407FEFDCFFB01E80FE6
:101A6000F91F20812EBD0DB407FEFDCF21812EBDB3
:101A70000296811522E0920771F70DB407FEFDCFA3
:101A80000895CF92DF92EF92FF920F931F930E94DF
:101A9000272A0091100B1091110B2091120B3091FD
:101AA000130B6B017C01C01AD10AE20AF30AF7FC9E
:101AB00055C08B019C010C53164F2F4F3F4F009385
:101AC000100B1093110B2093120B3093130B079BE9
:101AD0003CC0069B3AC0059B38C020919A0B21114F
:101AE00034C0049B32C000910C0B10910D0B20915F
:101AF0000E0B30910F0B011511052105310599F0E1
:101B0000DC01CB01801B910BA20BB30B80569A4ECC
:101B1000A109B1098827B7FD83959927AA27BB2773
:101B2000682F619501C060E06093140B662311F08B
:101B3000749A01C0749870E082E01F910F91FF9039
:101B4000EF90DF90CF900C94F32A60930C0B70937E
:101B50000D0B80930E0B90930F0BC5CF1F910F9120
:101B6000FF90EF90DF90CF90089581E08093150B68
:101B70000895AF92BF92CF92DF92EF92FF920F93B0
:101B80001F93CF93DF93F82E662351F010921B0B17
:101B90001092170B1092180B1092190B10921A0B2F
:101BA0000E94272A0091170B1091180B2091190BF6
:101BB00030911A0B5B016C01A01AB10AC20AD30A58
:101BC000D7FC44C020911B0BF7FC16C04F2D0F2CE7
:101BD000000C550B4C5F5F4FE22F022E000CFF0BE9
:101BE0004E175F079CF12F153CF044EFC42EDD2407
:101BF000D394E12CF12C06C038EEC32E33E0D32E63
:101C0000E12CF12CDC01CB018C0D9D1DAE1DBF1D07
